:020000040800F2
:1000000000040020A51F0008F71F0008F71F0008C4
:10001000F71F0008F71F0008F71F00080000000086
:10002000000000000000000000000000F71F0008B2
:10003000F71F000800000000F71F00088DF90108F5
:1000400019FB01081BFB01081DFB010821FB01082E
:1000500041FB010843FB010845FB010869FB01085E
:100060008DFB0108B1FB0108D5FB0108F9FB010874
:10007000FBFB0108FDFB0108FFFB010801FC010877
:1000800003FC010805FC010807FC0108F71F000834
:10009000F71F0008F71F0008F71F000809FC0108F8
:1000A00055FC010857FC010859FC01085BFC0108DC
:1000B0005DFC010861FC01088DFC0108FDFC0108E4
:1000C000FFFC010801FD010803FD010805FD010811
:1000D00009FD010879FE0108A1FD01083DFF0108A5
:1000E00001000208C5000208C7000208C900020892
:1000F000CD00020835010208370102083901020863
:100100003B0102083D0102083F01020841010208CB
:1001100045010208190202081B0202081D0202081A
:10012000290302082B0302082D0302082F030208EB
:1001300000000000000000000000000000000000BF
:1001400000000000000000000000000000000000AF
:10015000000000000000000000000000000000009F
:10016000000000000000000000000000000000008F
:10017000000000000000000000000000000000007F
:10018000000000000000000000000000000000006F
:10019000000000000000000000000000000000005F
:1001A000000000000000000000000000000000004F
:1001B000000000000000000000000000000000003F
:1001C000000000000000000000000000000000002F
:1001D000000000000000000000000000000000001F
:0401E0005FF8E0F1F3
:1001E800032A70B404460D4626D941EA000313F0E9
:1001F800030F13D020782B78984208BF294606D0E1
:100208001EE014F8010F11F8013F984218D1012A95
:1002180002F1FF32F5D1002070BC70470B4604464E
:1002280051F8045B50F8046BAE4204D1043A04461A
:10023800032A0B46F2D81D461046002ADAD1EBE70E
:10024800C01AE9E7032A2DE9F00109D82AB10023E9
:10025800CC5CC45401339342FAD1BDE8F001704735
:100268000B468218014603E02478013301F8014B5C
:1002780011F0030F1C46F7D113F003055DD06E4251
:10028800C5F1040CED009B594FEACC0C08E004348E
:10029800A7593B4607FA0CF748EA070741F8047BD9
:1002A800571A23FA05F8032FF1DC03E014F8013B91
:1002B80001F8013B8A42F9D8CFE753F8404C41F89E
:1002C800404C53F83C4C41F83C4C53F8384C41F8FE
:1002D800384C53F8344C41F8344C53F8304C41F80E
:1002E800304C53F82C4C41F82C4C53F8284C41F81E
:1002F800284C53F8244C41F8244C53F8204C41F82E
:10030800204C53F81C4C41F81C4C53F8184C41F83D
:10031800184C53F8144C41F8144C53F8104C41F84D
:10032800104C53F80C4C41F80C4C53F8084C41F85D
:10033800084C53F8044C41F8044C561A1D460C4618
:10034800403340313F2EB8DC2B460FE053F8101CE9
:1003580044F8101C53F80C1C44F80C1C53F8081CE7
:1003680044F8081C53F8041C44F8041C161B2146C6
:100378001D46103410330F2EE8DC2B4602E02468AB
:1003880041F8044B551A1C46032D03F10403F6DC0F
:1003980090E700BF032AC9B270B408D82AB103464F
:1003A800121803F8011B9342FBD170BC70478218E6
:1003B800044601E004F8011B14F0030FFAD14FF0D2
:1003C800013303FB01F31FE044F8403C44F83C3C94
:1003D80044F8383C44F8343C44F8303C44F82C3C6D
:1003E80044F8283C44F8243C44F8203C44F81C3C9D
:1003F80044F8183C44F8143C44F8103C44F80C3CCD
:1004080044F8083C44F8043C161B254640343F2E6B
:10041800DADC2C4607E044F8103C44F80C3C44F87D
:10042800083C44F8043C161B254610340F2EF2DC19
:1004380001E045F8043B541B032CFADC01E005F805
:10044800011B9542FBD3B0E710F0030F38B5044603
:1004580012D10368A3F1013222EA030313F0803FAB
:100468000AD1031D184653F8042BA2F1013525EAD9
:10047800020212F0803FF5D003782BB1431C1846D6
:1004880013F8012B002AFAD100F076F9204638BD7E
:10049800C9B2F0B4002950D010F0030F10D003787F
:1004A800002B79D0994246D0431C05E013F8012B64
:1004B800002A3FD091423ED013F0030F1846F5D1E1
:1004C800036841EA01270646A3F1013247EA0747D4
:1004D80022EA030212F0803F1DD187EA0303A3F149
:1004E800013222EA030313F0803F14D1043002E002
:1004F80012F0803F0FD1064650F8043BA3F10135B6
:1005080087EA030225EA0303A2F1013413F0803FCE
:1005180024EA0202ECD033783046002B3CD09942D2
:1005280009D0731C01E0914205D0184613F8012B3D
:10053800002AF8D11046F0BC704710F0030F0CD019
:100548000378002BF7D0431C03E013F8012B002A93
:10055800F1D013F0030F1846F7D102680346A2F151
:10056800013121EA020212F0803F0AD10430034629
:1005780050F8042BA2F1013121EA020212F0803F67
:10058800F5D01A781846002AD5D00133184613F842
:10059800012B002AFAD1CEE71846CCE780EA0102FF
:1005A80012F0030F3AD110F0030220F0030021F0FB
:1005B800030150F804CB08BF51F8043B0DD082F07A
:1005C80003024FEAC2026FF07F4323FA02F251F8A6
:1005D800043B4CEA020C43EA020300BFACF10132CF
:1005E8009C4501BF22EA0C0212F0803F50F804CB70
:1005F80051F8043BF2D04FEA0C604FEA1C2C01285A
:1006080028BFB0EB036F08BF1B0AF4D003F0FF0349
:100618004FEA1060A0EB0300704700BF10F0030F13
:100628000AD010F8012B11F8013B012A28BF9A4281
:10063800F4D0A2EB030070474DF8045D4DF8044D6B
:100648004FF0010242EA022242EA024201F0030CA0
:1006580021F0030150F8044B51F8045BBCF1020F80
:1006680026D04BD824F07F4CBCEB152FA4EB02030B
:1006780023EA04030DD113EAC21308BF51F8045B3F
:100688000AD18CEA040CBCEB056F0CD150F8044B72
:10069800E8E74FEA15255CE033F07F4352D10D7847
:1006A8004FEA146C55E04FEA146C05F0FF0550E072
:1006B8004FEA044CA4EB02034FEA1C4C23EA040360
:1006C800BCEB154F17D113EAC21308BF51F8045BEE
:1006D80007D18CEA040CBCEB054F08D150F8044B49
:1006E800E6E71B042ED10D884FEA144C31E04FEA9F
:1006F80005454FEA144C4FEA15452AE004F0FF0C73
:10070800BCEB156FA4EB020323EA04030DD113EA33
:10071800C21308BF51F8045B0AD18CEA040CBCEB85
:10072800052F0AD150F8044BE8E74FEA156510E0A9
:1007380014F0FF0F06D051F8045B4FEA142C25F093
:100748007F4506E04FF000005DF8044B5DF8045B60
:1007580070470CF0FF0205F0FF00012828BF904207
:1007680004BF4FEA1C2C2D0AF3D0A2EB00005DF861
:10077800044B5DF8045B704780EA0102844612F07E
:10078800030F4FD111F0030F32D14DF8044D11F082
:10079800040F51F8043B0BD0A3F101329A4312F035
:1007A800803F04BF4CF8043B51F8043B16D100BF0E
:1007B80051F8044BA3F101329A4312F0803FA4F19F
:1007C80001320BD14CF8043BA24312F0803F04BF26
:1007D80051F8043B4CF8044BEAD023460CF8013B93
:1007E80013F0FF0F4FEA3323F8D15DF8044B70473D
:1007F80011F0010F06D011F8012B0CF8012B002A7B
:1008080008BF704711F0020FBFD031F8022B12F069
:10081800FF0F16BF2CF8022B8CF8002012F47F4F24
:10082800B3D1704711F8012B0CF8012B002AF9D12C
:10083800704700BF20F0030110F00300C0F1000072
:1008480051F8043B00F1040C4FEACC0C6FF00002A5
:100858001CBF22FA0CF213434FF0010C4CEA0C2C8B
:100868004CEA0C4CA3EB0C0222EA030212EACC126B
:1008780004BF51F8043B0430F4D013F0FF0F1FBF3E
:10088800013013F47F4F013013F47F0F18BF01308C
:10089800704700BFF0B4002A46D041EA000313F0C5
:1008A80003032CD1032A07460E4643D904680D6872
:1008B800AC423FD1043A37D0A4F1013525EA04040B
:1008C80014F0803F18BF18462CD1041D0D1D0EE0F2
:1008D80054F8043B55F8041BA3F101308B4220EA7D
:1008E800030027D1043A1FD010F0803F1ED1032AFD
:1008F80027462E46ECD820462946002A1DD00478E3
:10090800013A0D78AC420CD172B18CB1002302E0EF
:1009180093420BD064B1013310F8014FCD5CAC4267
:10092800F6D0601BF0BC70471046FBE70020F9E7E3
:100938002046F7E738463146E1E724782D78F0E796
:1009480041EA000313F0030F0B4670B414BF0024F0
:100958000124032A94BF002404F001040546D4B9F5
:10096800BAB10E782B46013A03F8016B56B1AC1CAC
:100978007AB111F8015F2346013A04F8015C0134A9
:10098800002DF5D12AB19A18002103F8011B9342D2
:10099800FBD170BC7047194653F8044BA4F10136DB
:1009A80026EA040616F0803FDAD1043A45F8044BEB
:1009B800032A1946EFD8D3E701232DE9F0071D468E
:1009C80000264FF0FF37AC1900EB070C8C420DD214
:1009D8001CF805C010F80480E0452ED201252646F3
:1009E800E31BAC198C4200EB070CF1D34FF0010963
:1009F80000264D464FF0FF3C1360AC1900EB0C0885
:100A0800A1420ED918F8058010F804A0C2451AD9D9
:100A180001252646CCEB0409AC19A14200EB0C08D1
:100A2800F0D80CF101000137B8423CBF994638466E
:100A3800C2F80090BDE8F00770470BD00123374695
:100A48001D46F618BFE709D04FF00109B4464D46D8
:100A58004E44D2E79D4205D00135B4E74D4505D057
:100A68000135CAE72B4626460125ACE7A9462646A6
:100A78000125C2E72DE9F04FADF5826D81B014462E
:100A8800074610460DF580628B460C3219461D4606
:100A9800FFF792FF03AE04A901F57E72331F0090A1
:100AA80043F8045F9342FBD14DB1681E0023E25C1A
:100AB800C11A013303AEAB4246F82210F7D1DDF874
:100AC8000C142046009A6118FFF78AFB002877D19A
:100AD8000099814605F1FF380646C1F101020192ED
:100AE8005A46AB4609EB0B0501F1FF3AB81800214D
:100AF800AA1A00F0E5F900284FD1002D00F0C080B7
:100B08007B1903A913F8013C51F82330002B4CD171
:100B1800009B9E4228BF334698450FD903EB090135
:100B2800E05C7A18795C884205D038E012F8011F39
:100B3800E05C884233D101339845F7D8009A964251
:100B480080F0A48007EB090214F80A10534612F843
:100B58000A20914204BF0AEB0901791807D095E0F1
:100B680014F802C011F8010D844503D113465A1E2A
:100B7800B342F5D101369E4200F28D80DDF80C6457
:100B88002A46B144C6EB0B0609EB0B05B818002141
:100B9800AA1A00F095F90028AFD0002071E0019A58
:100BA8000026914499442A46EEE7002EFAD0DDF853
:100BB8000C2493423CBFC2EB0B0306469944F2E770
:100BC800009E4FF000080099AB1BB34238BF334674
:100BD800C1F101026E1E019201F1FF3A5A4689469F
:100BE800AB460133CDF80C3408EB0B05B8180021DF
:100BF800AA1A00F065F90028CFD1002D40D07B1942
:100C080003A913F8013C51F82330002B30D1B1452A
:100C180013D208EB090314F80910FA18FB5C99427F
:100C280018BF4B4627D14B4604E012F8011FE05C81
:100C3800884220D10133B342F7D3BAF1FF3F53467C
:100C48002CD007EB080C14F80A101CF80A20914263
:100C58000CD10AEB0802BA1804E0E05C12F8011D96
:100C6800884203D1013BF8D260460AE0DDF80C3433
:100C780098442A46B8E701992A4688449844B3E735
:100C8800284605B00DF5806DBDE8F08F009B013654
:100C98009E427FF673AF07EB0900F2E707EB080CFB
:100CA8006046EEE72DE9F04F8346037885B00C46A1
:100CB800002B00F0F9800A78A2B106460131012024
:100CC80002E011F8012B8AB1934214BF002000F012
:100CD800010016F8013F0D46002BF2D12B782BB1FD
:100CE8004FF0000B584605B0BDE8F08F0028F9D149
:100CF8000BF101002178FFF7CBFB2D1BA5F10102B9
:100D0800534243EB0203002808BF43F001030746A0
:100D180083B90BEB0508404594BFC0EB08084FF0BA
:100D280001081F2D08D9414622462B46FFF7A2FE8F
:100D38008346D7E78346D5E7294603AA2046FFF727
:100D48003BFE03996118814620464A46FFF748FA58
:100D580000284FD109F1FF33C9F10102064601927B
:100D680082464246C84699460AEB050BB818002148
:100D7800C2EB0B0200F0A4F80028B1D1BBF1000FC0
:100D8800B0D046452CBF334643469D420FD903EBAE
:100D98000A01E05C7A18795C884205D075E012F89F
:100DA800011FE05C884270D101339D42F7D1B04504
:100DB8007DD907EB0A0214F809104B4612F80920EE
:100DC800914202BF09EB0A01AC46791806D06EE0E1
:100DD800A55C11F8010D854203D113465A1EB34292
:100DE800F6D1654601369E4267D8039E5A46B244FC
:100DF800AE1BB9E7C9F10101C9EB0503424600265C
:100E080009F1FF3A88464B4538BF4B4601330393F7
:100E180006EB050BB8180021C2EB0B0200F050F8E6
:100E280000287FF45DAFBBF1000F3FF45BAF4D4589
:100E380012D906EB090314F80910FA18FB5C994259
:100E480008BF4B4605D026E012F8011FE05C884237
:100E580022D101339D42F7D1BAF1FF3F534628D042
:100E680007EB060C14F80A101CF80A20914217D157
:100E78000AEB0602BA1804E0E05C12F8011D884289
:100E88000ED1013BF8D2E3462CE7019A00269244A2
:100E98005A469A4468E74B4646445A46F618B7E716
:100EA800039B5A46F618B3E70D46012016E743465A
:100EB80098E707EB060CE34614E707EB0A0B11E784
:100EC80010F0030F034670B4C9B211D0002A22D023
:100ED80003788B421DD0013A013005E0DAB110F8F1
:100EE800014B013A8C4218D010F0030F0346F5D19C
:100EF800032A14D87AB1187888420ED0541E5D1C83
:100F080003E015F8016B8E4203D0013C2846F8D265
:100F1800002070BC70471046FBE71846F9E741EA25
:100F2800012646EA0646184653F8044B86EA0404A6
:100F3800A4F1013525EA040414F0803F03D1043AF2
:100F48001846032AEFD80346D4E700BF0000000084
:100F5800C1F30A5C0246ACF57E7C2DE9F84FACF192
:100F68000704132C0B4606460F468946804627DCA5
:100F7800002C52DB4FF6FF7CC0F20F0C4CFA04FA3F
:100F88000AEA0105054317D037A3D3E9002300F087
:100F980075F80022002300F0B3FC002856D0002F7B
:100FA80005DD4FF4801353FA04F407EB040929EA2A
:100FB8000A0900264B46324610461946BDE8F88F06
:100FC800332C07DDB4F5806FF6D100F057F80246F0
:100FD8000B46F1E74FF0FF3BACF11B0C2BFA0CFB77
:100FE8001BEA000FE8D020A3D3E9002300F046F85D
:100FF8000022002300F084FC40B3002F0ADD142CEB
:1010080006D00126C4F13404A64016EB080601D325
:1010180007F1010926EA0B0619E013A3D3E9002317
:1010280000F02CF80022002300F06AFC78B1002FB1
:1010380013DB46EA07054FF000094D45C3F6F07982
:101048000CBF2E46002608BFA94600E0B9464B460D
:10105800324610461946BDE8F88F00264FF0004981
:10106800F5E700BFAFF300809C7500883CE4377E4D
:1010780081F0004102E000BF83F0004330B54FEA41
:1010880041044FEA430594EA050F08BF90EA020FAE
:101098001FBF54EA000C55EA020C7FEA645C7FEA41
:1010A800655C00F0E2804FEA5454D4EB5555B8BF64
:1010B8006D420CDD2C4480EA020281EA030382EAD5
:1010C800000083EA010180EA020281EA0303362D67
:1010D80088BF30BD11F0004F4FEA01314FF4801C3A
:1010E8004CEA113102D0404261EB410113F0004F4C
:1010F8004FEA03334CEA133302D0524263EB430303
:1011080094EA050F00F0A780A4F10104D5F1200EA0
:101118000DDB02FA0EFC22FA05F2801841F10001FB
:1011280003FA0EF2801843FA05F359410EE0A5F1CF
:1011380020050EF1200E012A03FA0EFC28BF4CF000
:10114800020C43FA05F3C01851EBE37101F00045B6
:1011580007D54FF0000EDCF1000C7EEB00006EEBC3
:101168000101B1F5801F1BD3B1F5001F0CD349084D
:101178005FEA30004FEA3C0C04F101044FEA4452A4
:1011880012F5800F80F09A80BCF1004F08BF5FEA2B
:10119800500C50F1000041EB045141EA050130BD0B
:1011A8005FEA4C0C404141EB010111F4801FA4F1AE
:1011B8000104E9D191F0000F04BF01460020B1FA03
:1011C80081F308BF2033A3F10B03B3F120020CDA3B
:1011D8000C3208DD02F1140CC2F10C0201FA0CF019
:1011E80021FA02F10CE002F11402D8BFC2F1200C7E
:1011F80001FA02F120FA0CFCDCBF41EA0C01904034
:10120800E41AA2BF01EB0451294330BD6FEA04047C
:101218001F3C1CDA0C340EDC04F11404C4F1200267
:1012280020FA04F001FA02F340EA030021FA04F379
:1012380045EA030130BDC4F10C04C4F1200220FAD0
:1012480002F001FA04F340EA0300294630BD21FA0E
:1012580004F0294630BD94F0000F83F4801306BFD4
:1012680081F480110134013D4EE77FEA645C18BFC8
:101278007FEA655C29D094EA050F08BF90EA020F5F
:1012880005D054EA000C04BF1946104630BD91EA57
:10129800030F1EBF0021002030BD5FEA545C05D15A
:1012A8004000494128BF41F0004130BD14F5800499
:1012B8003CBF01F5801130BD01F0004545F0FE410D
:1012C80041F470014FF0000030BD7FEA645C1ABF42
:1012D800194610467FEA655C1CBF0B46024650EA79
:1012E800013406BF52EA033591EA030F41F40021A5
:1012F80030BD00BF90F0000F04BF0021704730B52B
:101308004FF4806404F132044FF000054FF00001FF
:1013180050E700BF90F0000F04BF0021704730B5C0
:101328004FF4806404F1320410F0004548BF404295
:101338004FF000013EE700BF42004FEAE2014FEAEA
:1013480031014FEA02701FBF12F07F4393F07F4FC5
:1013580081F06051704792F0000F14BF93F07F4FF7
:10136800704730B54FF4607401F0004521F000413A
:1013780020E700BF50EA010208BF704730B54FF0C0
:1013880000050AE050EA010208BF704730B511F0C5
:10139800004502D5404261EB41014FF4806404F1FD
:1013A80032045FEA915C3FF4DCAE4FF003025FEA7F
:1013B800DC0C18BF03325FEADC0C18BF033202EB07
:1013C800DC02C2F1200300FA03FC20FA02F001FA61
:1013D80003FE40EA0E0021FA02F11444C1E600BF00
:1013E80070B54FF0FF0C4CF4E06C1CEA11541DBFB3
:1013F8001CEA135594EA0C0F95EA0C0F00F0DEF87E
:101408002C4481EA030621EA4C5123EA4C5350EA62
:10141800013518BF52EA033541F4801143F48013B3
:1014280038D0A0FB02CE4FF00005E1FB02E506F044
:101438000042E0FB03E54FF00006E1FB03569CF099
:10144800000F18BF4EF0010EA4F1FF04B6F5007F9F
:1014580064F5407404D25FEA4E0E6D4146EB060611
:1014680042EAC62141EA55514FEAC52040EA5E509A
:101478004FEACE2EB4F1FD0C88BFBCF5E06F1ED844
:10148800BEF1004F08BF5FEA500E50F1000041EB7B
:10149800045170BD06F0004646EA010140EA020028
:1014A80081EA0301B4EB5C04C2BFD4EB0C0541EA4A
:1014B800045170BD41F480114FF0000E013C00F35F
:1014C800AB8014F1360FDEBF002001F0004170BD83
:1014D800C4F10004203C35DA0C341BDC04F114049C
:1014E800C4F1200500FA05F320FA04F001FA05F228
:1014F80040EA020001F0004221F0004110EBD370F5
:1015080021FA04F642EB06015EEA430E08BF20EA20
:10151800D37070BDC4F10C04C4F1200500FA04F3C3
:1015280020FA05F001FA04F240EA020001F0004155
:1015380010EBD37041F100015EEA430E08BF20EAC8
:10154800D37070BDC4F1200500FA05F24EEA020E10
:1015580020FA04F301FA05F243EA020321FA04F03F
:1015680001F0004121FA04F220EA020000EBD370F6
:101578005EEA430E08BF20EAD37070BD94F0000FF6
:101588000FD101F00046400041EB010111F4801F2A
:1015980008BF013CF7D041EA060195F0000F18BFDB
:1015A800704703F00046520043EB030313F4801F17
:1015B80008BF013DF7D043EA0603704794EA0C0FD1
:1015C8000CEA135518BF95EA0C0F0CD050EA4106E7
:1015D80018BF52EA4306D1D181EA030101F0004164
:1015E8004FF0000070BD50EA410606BF104619468C
:1015F80052EA430619D094EA0C0F02D150EA013698
:1016080013D195EA0C0F05D152EA03361CBF1046D8
:1016180019460AD181EA030101F0004141F0FE4177
:1016280041F470014FF0000070BD41F0FE4141F4FB
:10163800780170BD70B54FF0FF0C4CF4E06C1CEAFB
:1016480011541DBF1CEA135594EA0C0F95EA0C0FB0
:1016580000F0A7F8A4EB050481EA030E52EA03356B
:101668004FEA013100F088804FEA03334FF080558C
:1016780045EA131343EA12634FEA022245EA1115B9
:1016880045EA10654FEA00260EF000419D4208BF6A
:10169800964244F1FD0404F5407402D25B084FEA17
:1016A8003202B61A65EB03055B084FEA32024FF4C3
:1016B80080104FF4002CB6EB020E75EB030E22BF20
:1016C800B61A754640EA0C005B084FEA3202B6EBE0
:1016D800020E75EB030E22BFB61A754640EA5C008F
:1016E8005B084FEA3202B6EB020E75EB030E22BF1F
:1016F800B61A754640EA9C005B084FEA3202B6EB20
:10170800020E75EB030E22BFB61A754640EADC00DE
:1017180055EA060E18D04FEA051545EA16754FEA40
:1017280006164FEAC30343EA52734FEAC2025FEA5E
:101738001C1CC0D111F4801F0BD141EA00014FF0ED
:1017480000004FF0004CB6E711F4801F04BF0143BE
:101758000020B4F1FD0C88BFBCF5E06F3FF6AFAEDA
:10176800B5EB030C04BFB6EB020C5FEA500C50F16A
:10177800000041EB045170BD0EF0004E4EEA1131ED
:1017880014EB5C04C2BFD4EB0C0541EA045170BDF4
:1017980041F480114FF0000E013C90E645EA060E38
:1017A8008DE60CEA135594EA0C0F08BF95EA0C0F66
:1017B8003FF43BAF94EA0C0F0AD150EA01347FF4AE
:1017C80034AF95EA0C0F7FF425AF104619462CE785
:1017D80095EA0C0F06D152EA03353FF4FDAE1046E8
:1017E800194622E750EA410618BF52EA43067FF439
:1017F800C5AE50EA41047FF40DAF52EA43057FF4C9
:10180800EBAE12E74FF0FF3C06E000BF4FF0010CD3
:1018180002E000BF4FF0010C4DF804CD4FEA410C37
:101828007FEA6C5C4FEA430C18BF7FEA6C5C1BD004
:1018380001B050EA410C0CBF52EA430C91EA030F85
:1018480002BF90EA020F0020704710F1000F91EAE2
:10185800030F58BF994208BF90422CBFD8176FEAB0
:10186800E37040F0010070474FEA410C7FEA6C5C7E
:1018780002D150EA013C07D14FEA430C7FEA6C5C85
:10188800D6D152EA033CD3D05DF8040B704700BFB1
:101898008446104662468C461946634600E000BFFF
:1018A80001B5FFF7B7FF002848BF10F1000F01BDD1
:1018B8004DF808EDFFF7F4FF0CBF012000205DF89C
:1018C80008FB00BF4DF808EDFFF7EAFF34BF012021
:1018D80000205DF808FB00BF4DF808EDFFF7E0FFBA
:1018E80094BF012000205DF808FB00BF4DF808ED0B
:1018F800FFF7CEFF94BF012000205DF808FB00BF72
:101908004DF808EDFFF7C4FF34BF012000205DF853
:1019180008FB00BF4FEA4102B2F1E04324BFB3F530
:10192800001CDCF1FE5C0DD901F0004C4FEAC0024E
:101938004CEA5070B2F1004F40EB830008BF20F032
:101948000100704711F0804F21D113F13872BCBFEC
:1019580001F00040704741F480114FEA5252C2F141
:101968001802C2F1200C10FA0CF320FA02F018BF8A
:1019780040F001004FEAC1234FEAD32303FA0CFCDD
:1019880040EA0C0023FA02F34FEA4303CCE77FEA6C
:10199800625307D150EA01331EBF4FF0FE4040F4B6
:1019A8004000704701F0004040F0FE4040F4000065
:1019B800704700BF80F0004002E000BF81F00041A6
:1019C80042001FBF5FEA410392EA030F7FEA226CDD
:1019D8007FEA236C6AD04FEA1262D2EB1363C1BF6D
:1019E800D218414048404140B8BF5B42192B88BFDC
:1019F800704710F0004F40F4000020F07F4018BFFF
:101A0800404211F0004F41F4000121F07F4118BF1E
:101A1800494292EA030F3FD0A2F1010241FA03FCC6
:101A280010EB0C00C3F1200301FA03F100F00043AE
:101A380002D5494260EB4000B0F5000F13D3B0F176
:101A4800807F06D340084FEA310102F10102FE2AE5
:101A580051D2B1F1004F40EBC25008BF20F0010055
:101A680040EA03007047490040EB000010F4000F03
:101A7800A2F10102EDD1B0FA80FCACF1080CB2EB96
:101A88000C0200FA0CF0AABF00EBC25052421843F5
:101A9800BCBFD0401843704792F0000F81F400019A
:101AA80006BF80F400000132013BB5E74FEA41036D
:101AB8007FEA226C18BF7FEA236C21D092EA030FD9
:101AC80004D092F0000F08BF0846704790EA010F53
:101AD8001CBF0020704712F07F4F04D1400028BF80
:101AE80040F00040704712F100723CBF00F5000062
:101AF800704700F0004343F0FE4040F40000704798
:101B08007FEA226216BF08467FEA23630146420243
:101B180006BF5FEA412390EA010F40F48000704756
:101B28004FF0000304E000BF10F0004348BF4042FC
:101B38005FEA000C08BF704743F0964301464FF038
:101B480000001CE050EA010208BF70474FF0000394
:101B58000AE000BF50EA010208BF704711F00043D5
:101B680002D5404261EB41015FEA010C02BF8446A5
:101B78000146002043F0B64308BFA3F18053A3F504
:101B88000003BCFA8CF2083AA3EBC25310DB01FA4B
:101B980002FC634400FA02FCC2F12002BCF1004FCF
:101BA80020FA02F243EB020008BF20F00100704760
:101BB80002F1200201FA02FCC2F1200250EA4C00B4
:101BC80021FA02F243EB020008BF20EADC707047FA
:101BD8004FF0FF0C1CEAD0521EBF1CEAD15392EA08
:101BE8000C0F93EA0C0F6FD01A4480EA010C4002E4
:101BF80018BF5FEA41211ED04FF0006343EA50103E
:101C080043EA5111A0FB01310CF00040B1F5000F7F
:101C18003EBF490041EAD3715B0040EA010062F12E
:101C28007F02FD2A1DD8B3F1004F40EBC25008BF18
:101C380020F00100704790F0000F0CF0004C08BF36
:101C480049024CEA502040EA51207F3AC2BFD2F103
:101C5800FF0340EAC250704740F400004FF0000311
:101C6800013A5DDC12F1190FDCBF00F0004070474B
:101C7800C2F10002410021FA02F1C2F1200200FA89
:101C880002FC5FEA310040F1000053EA4C0308BF50
:101C980020EADC70704792F0000F00F0004C02BFA1
:101CA800400010F4000F013AF9D040EA0C0093F01C
:101CB800000F01F0004C02BF490011F4000F013B76
:101CC800F9D041EA0C018FE70CEAD15392EA0C0FE4
:101CD80018BF93EA0C0F0AD030F0004C18BF31F04F
:101CE800004CD8D180EA010000F00040704790F025
:101CF800000F17BF90F0004F084691F0000F91F0C9
:101D0800004F14D092EA0C0F01D142020FD193EA8E
:101D18000C0F03D14B0218BF084608D180EA010016
:101D280000F0004040F0FE4040F40000704740F0F2
:101D3800FE4040F4400070474FF0FF0C1CEAD052C0
:101D48001EBF1CEAD15392EA0C0F93EA0C0F69D01C
:101D5800A2EB030280EA010C49024FEA402037D087
:101D68004FF0805343EA111143EA10130CF000407E
:101D78008B4238BF5B0042F17D024FF4000C8B426E
:101D880024BF5B1A40EA0C00B3EB510F24BFA3EB4E
:101D9800510340EA5C00B3EB910F24BFA3EB91031E
:101DA80040EA9C00B3EBD10F24BFA3EBD10340EA78
:101DB800DC001B0118BF5FEA1C1CE0D1FD2A3FF6BE
:101DC80050AF8B4240EBC25008BF20F00100704773
:101DD8000CF0004C4CEA50207F32C2BFD2F1FF0316
:101DE80040EAC250704740F400004FF00003013A47
:101DF80037E792F0000F00F0004C02BF400010F4EB
:101E0800000F013AF9D040EA0C0093F0000F01F0FE
:101E1800004C02BF490011F4000F013BF9D041EA20
:101E28000C0195E70CEAD15392EA0C0F08D1420253
:101E38007FF47DAF93EA0C0F7FF470AF084676E726
:101E480093EA0C0F04D14B023FF44CAF08466EE7FF
:101E580030F0004C18BF31F0004CCAD130F00042CD
:101E68007FF45CAF31F000437FF43CAF5FE700BF25
:101E78004FF0FF3C06E000BF4FF0010C02E000BF4E
:101E88004FF0010C4DF804CD4FEA40024FEA4103F0
:101E98007FEA226C18BF7FEA236C11D001B052EAA6
:101EA800530C18BF90EA010F58BFB2EB030088BF6C
:101EB800C81738BF6FEAE17018BF40F001007047DB
:101EC8007FEA226C02D15FEA402C05D17FEA236CBD
:101ED800E4D15FEA412CE1D05DF8040B704700BF04
:101EE800844608466146FFE70FB5FFF7C9FF00289B
:101EF80048BF10F1000F0FBD4DF808EDFFF7F4FFD4
:101F08000CBF012000205DF808FB00BF4DF808ED6C
:101F1800FFF7EAFF34BF012000205DF808FB00BF8F
:101F28004DF808EDFFF7E0FF94BF012000205DF8B1
:101F380008FB00BF4DF808EDFFF7D2FF94BF012062
:101F480000205DF808FB00BF4DF808EDFFF7C8FF5B
:101F580034BF012000205DF808FB00BF42000ED20C
:101F6800B2F1FE4F0BD34FF09E03B3EB126209D4CC
:101F78004FEA002343F0004323FA02F070474FF082
:101F88000000704712F1610F01D1420202D14FF0F7
:101F9800FF3070474FF00000704700BF00F026F890
:101FA8000C4880F30888002103E00B4B5B58435032
:101FB80004310A480A4B42189A42F6D3094A02E009
:101FC800002342F8043B084B9A42F9D317F0ACF9C6
:101FD8007047000000C00020D42D03080000002036
:101FE800600E0020600E0020584200207047FEE777
:101FF80010B586B0002301244FF46022114801A9CE
:1020080001938DF80930039204938DF808408DF8F8
:10201800144020F037FF0B48214620F059FF0948AB
:1020280020F060FF074820F062FF0028FAD1054839
:1020380020F061FF034820F063FF0028FAD106B0C2
:1020480010BD00BF00240140014610B50D48012213
:10205800032320F063FF0B48012120F055FF7F2068
:1020680021F092FD0748022120F0A2FF0028F6D0B7
:102078000448022120F0A2FF0248BDE8104020F0E9
:1020880094BF00BF002401400C4A0C2303FB01232A
:1020980010B59C880CB9588010BD5B8803F11304F7
:1020A800844204DA142B07D9133B834204DC0C2343
:1020B80003FB012102238B8010BD00BFB425002043
:1020C8000A4B10B500241C7021464FF4E0720848F2
:1020D800FEF760F9074B4FF474501C70064B1C70E8
:1020E8000EF09AFD054B187010BD00BFD4100020EB
:1020F800A0120020EB140020681400206A140020AD
:10210800074B1978013101F01F011970054B1A7836
:102118008A4203D1013202F01F021A70704700BFD1
:1021280068140020EB14002010B50E4A0E2303FBA0
:1021380000200D4A014614780C4A03FB042300F1E1
:102148000C0251F8044B914243F8044BF9D10A8828
:1021580000211A800E22FEF71DF9BDE81040FFF796
:10216800CFBF00BFD810002068140020A0120020A4
:10217800084B1A5C002352FA03F111F0010FD8B290
:1021880002D00130C0B270470133042BF3D10120D3
:10219800704700BF9515002000F07F0000F57450CF
:1021A8002DE9F84305300C46154698460EF034FDE7
:1021B80000284ED043F63837002638460EF02CFD5E
:1021C800C0B25FFA86F988B120280FD04FEA5909C2
:1021D8004AF20B5048440EF01FFDC0B208B1022865
:1021E80004D10123B34022781343237011370136F9
:1021F800B7F56F5FE1D14AF2B2300EF00DFDC0B213
:1022080080B120280ED02B784AF2A13043F0010388
:102218002B700EF001FDC0B220B1202802D001239E
:1022280088F800304AF2E3300EF0F6FCC0B280B114
:1022380020280ED02B784AF2A13043F002032B70ED
:102248000EF0EAFCC0B220B1202802D0012388F8A1
:102258000030BDE8F8830000034610465A1E10B54A
:10226800032A1CD8DFE802F00E0E0207114A527842
:1022780002F0100203E00F4A527802F00802D2B2CC
:1022880072B10BE00C4A927802F04002D2B23AB135
:102298000A4A127802F003029A4200D140B10022A1
:1022A8000748105C984203D00132052AF8D1002172
:1022B800084610BD68400020B0310020633400207B
:1022C80098120020F8B5064643F63835002428460B
:1022D8000EF0A2FCC0B2E7B268B120280BD07F088C
:1022E8004AF20B5038180EF097FC012803D1A04091
:1022F80033781843307001341135082CE7D1F8BD14
:1023080003780E2202FB0313084AD3189978002396
:1023180051FA03F010F00100DAB202D0501CC0B23A
:1023280070470133082BF3D1704700BFA01200207B
:102338002DE9F04101248C40284A29490346E4B29A
:10234800107891F800C019E0264F0E2606FB00769B
:10235800F178A9B996F80680B8F1000F10D196F86F
:102368000580B8F1000F0BD196F80480B8F1000F82
:1023780006D1F67926B9013000F01F00054626E09F
:10238800FBB1012B05D0022B06D10E2101FB0077F2
:1023980039790C4218D014E0042B04D10E2101FB2A
:1023A8000077B9790CE0032B04D10E2101FB0077EB
:1023B800797905E0052B07D10E2101FB0077F97922
:1023C80011B11570BDE8F081013000F01F006045C3
:1023D800BAD11570FF20BDE8F08100BFEB140020D2
:1023E80068140020A01200202DE9F043434D444B0F
:1023F8002A780E2101FB0232917A85B0044698466C
:1024080031B101390523594301F56F5189B201E012
:102418004FF46F51204604220EF00FFC2B780E2546
:1024280005FB038393F80B80354E344FB8F1000F4A
:1024380025D131232371073363713B7801A86B439E
:102448000422F15E06F00CFA3B7802A805FB036350
:102458000222997A06F004FA3B780DF10A0005FB8E
:1024680003650322697A06F0FBF9A01D01A9092278
:10247800FEF766FA4FF00F0984F8108012E0B8F101
:10248800010F0FD132232371053363713B784FF06D
:10249800080905FB036393F90130E3713B785D4359
:1024A800735BA371002320461A4612E010F8011B43
:1024B800A1F13005EDB2092D04D8EB183029DBB2B3
:1024C80003D004E037395B1800E00A33DBB201328D
:1024D800D2B24A45EAD10F21B3FBF1F10801411A02
:1024E8005B1AC3F10F03DBB2092BA35401D83033B5
:1024F80000E03733A35405B0BDE8F0839E120020F6
:10250800A0120020024B1A7842F001021A7070479C
:10251800CD17002008B50C4B0C4A1B780E2101FB87
:102528000323D97A21B101290CBF0921002100E038
:10253800102140221346064805F0B6FF054B1A78CD
:1025480042F002021A7008BD9E120020A01200205C
:102558006B140020CD170020034B1A7802F0F80204
:102568006FF3C3021A707047CD170020024B1A7818
:1025780042F004021A707047CD170020024B1A78F7
:1025880042F008021A707047CD17002038B5114B79
:102598001C7814F0010502D1FFF7B4FF05E004F040
:1025A8000405EDB21DB9FFF7E1FF284638BD04F078
:1025B8000805EDB215B9FFF7E1FFF6E704F00204EC
:1025C800E4B21CB9FFF7A6FF204638BDFFF7C4FFE9
:1025D800012038BDCD170020014B1878704700BF87
:1025E800D410002030B51E4B85B01B780446002B54
:1025F80034D11C4D2B78034113F0010F2ED01A4B08
:102608001A4A1B780E2101FB0323DA78024112F0E3
:10261800010F1CD11B79034113F0010317D110F0EE
:10262800010001F1F1014FEA540206D00132009194
:10263800019302926D20FE3905E00132009101906C
:1026480002923C20012103220B460EF063FB01237A
:1026580013FA04F42B7823EA04042C7005B030BD77
:102668006A14002061140020EB140020A01200203E
:10267800037830B513F0010F144A4FF00E0419D146
:1026880004FB01210133012212FA03F3CD7825EA74
:102698000303CB7004780D79A41812FA04F425EA20
:1026A80004040C7103789B189A408B7823EA020281
:1026B8008A7030BD04FB0121013B012212FA03F3A9
:1026C8008A7822EA03038B7030BD00BFA012002075
:1026D80010B500230278590052FA01F404F00304FB
:1026E800022C05D1013414FA01F122EA0102027028
:1026F8000133042BEED110BD2DE9F04F85B00192C6
:10270800BDF838201C46734B0092DA78054612F063
:1027180020028B4640F0D8808DF80E208DF80F20CF
:102728008DF80D20DCB99B7803F04003DBB21BB1B8
:1027380001238DF80F3020E0674B5B7803F002032C
:10274800DBB21BB101238DF80E3016E00DF10F013D
:102758000DF10E020DF10D03FFF71EFD0DE0012C2A
:102768000BD19B7803F04003DBB223B90DF10F00C6
:10277800FFF7A8FD01E08DF80F409DF80F3023B951
:102788009DF80E00002800F0A28044B905F07F01F2
:10279800490001F574510DF10A00623109E0012C7C
:1027A8000AD1E90101F50C413C310DF10A0001EBB8
:1027B8004B0102220EF041FABDF90A3013B9002C80
:1027C80000F08480009B33B9444B454F93F8008058
:1027D800FFF796FC08E0434B434F93F8008008F15D
:1027E800010202F01F021A700DF10F00FFF770FFCF
:1027F800002C44D1BDF80A3069B240F6B83212EA6A
:10280800210238BF4FF47A72D2180E2303FB08F363
:10281800ADF80A20FA529DF80F9022464946012049
:10282800FE18FFF719FD4946F07022460220FFF70F
:1028380013FD86F8029030719DF80E9022464946A5
:102848000420FFF709FD4946B0718246224603205D
:10285800FFF702FD05F07F0570713572BAF1000FC0
:1028680000D128B1214B1B7813B99DF80D3000E039
:102878000023F37186F809B0019AB2721CE0012CAA
:102888001AD10E2303FB08F3BDF80A202046FA529A
:102898009DF80F6000223146FD18FFF7DDFC314638
:1028A800E87000220220FFF7D7FC00232871AE70E1
:1028B800AB716B71EB71AB720E2303FB0877FC7283
:1028C800009B0120BB8102E0002000E0204605B00B
:1028D800BDE8F08FB0310020684000206814002067
:1028E800A0120020D3100020D8100020B21700201A
:1028F80073B5154B04461B780E46D3B113482146D1
:102908001FF067FC0546A0B9012E04F1010606D1A7
:102918002046FFF72DFC00950246812005E0204661
:10292800FFF726FC00950246982031462B46FFF714
:10293800E3FE214605481FF036FC0548214602B053
:10294800BDE870401FF03ABC69140020D016002082
:10295800F81400202DE9F7437B4B04461B7843B15C
:102968007A4B1B7803F02403042B02D1002900F0D2
:10297800E880774B774F1B78002B00F0C7807648AC
:1029880021461FF026FC002840F0C08007F5C470DF
:1029980021461FF01EFC8046002840F0B7803B19F6
:1029A80093F880302D2B01D0532B3AD16B4E3578CC
:1029B80045B30EF0A5FC04F10108054650B12046C8
:1029C800FFF7D6FB337802461E3300939320414627
:1029D800002307E02046FFF7CBFB0095024641465F
:1029E80093202B46FFF788FE0EF08AFC014628B19B
:1029F800337813201E330093002101E00090132048
:102A08000A4680E02046FFF7B3FB611C02462B46CE
:102A180093200095FFF770FE0095132029462A465B
:102A280071E0542B09D12046FFF7A2FBCDF80080B6
:102A38000246611C9420434666E0462B474D20D150
:102A48002E78BEB10EF05CFC04F10109064648B1CF
:102A58002046FFF78DFB2B7802461E3300939A2001
:102A6800494622E02046FFF783FB00960246494686
:102A78009A2025E02046FFF77BFB009602469A2025
:102A880039E02E78002E2CD00EF03AFC04F11C0907
:102A9800064660B12046FFF76BFB2B7802461E33D3
:102AA80069F07F000093C0B2611C434609E02046EC
:102AB800FFF75EFB024669F07F000096C0B2611C1A
:102AC8003346FFF719FE0EF01BFC21B2024628B16F
:102AD8002B7803201E330093002214E0009003207B
:102AE80011E02046FFF744FB024604F11C0060F0A9
:102AF8007F000096C0B2611C3346FFF7FDFD0096CB
:102B08000320214632460123FFF7F6FD12482146ED
:102B18003F191FF048FB97F880302D2B0AD0532B14
:102B280008D0542B06D0462B04D00D4821461FF060
:102B380050FB30B10B48214603B0BDE8F0431FF00D
:102B48003DBB03B0BDE8F083D6100020BE160020C0
:102B580069140020E0230020D01600202817002048
:102B680068250020C8160020002302780E2101FBEA
:102B78000232044901338A180021062B9170F4D1DE
:102B8800704700BFA0120020064B00201870064BAB
:102B98001A78064B1B789A4202D00146FFF7C8BB49
:102BA800FF207047D410002068140020EB14002088
:102BB8000121814038B5114BC9431A78104BC9B26D
:102BC80002F0030203F5E074012A04D1DD7801EA7A
:102BD8000505DD7005E0022A03D11D7901EA050526
:102BE8001D710E33A342EFD1FFF7FCFC4FF4745074
:102BF8000EF012F8034B187038BD00BF6334002084
:102C0800A01200206A1400202DE9F743A34D8DF887
:102C180007002B78A24C1BB12378C2B29A4204D089
:102C28004FF474500DF0F8FF28709DF807302370AA
:102C38009C4C2278072A00F22D81DFE812F0080068
:102C48002400360054005D0072008D00BA00964AD8
:102C58003C211170954A1946107800F00300FFF7DF
:102C680067FB934BFF28187000F036811DF0E6FFD4
:102C7800904B002093F8742042F0010283F87420EE
:102C88008D4B187064E0884B1B78002B00F0248172
:102C98001EF09CF9012840F04D812378142201335D
:102CA8002370864B01381A7047E17F4B1B78002B45
:102CB80000F01281814E307808B901234AE01EF0F5
:102CC80085F9022804D01EF081F9032840F03281EA
:102CD8001DF0B4FF23780422013323701D233370C1
:102CE800774B1A7026E1704B3C221A707548FFF733
:102CF8007BFB2378013323706B4B1B78002B00F090
:102D0800EB806E4B1D78002D40F014811020FFF7EA
:102D18003DFC002800F011812378284601332370F8
:102D28000BE1614B1B78002B00F0D68005F026FCE8
:102D3800002800F00281614B7D221A705E4B002052
:102D480018705C4B93F8742042F0010283F87420E9
:102D5800237801332370F0E0534B1B78002B00F0ED
:102D6800BB801EF033F90128544E03D01EF02EF913
:102D780003280FD19DF80720012111FA02F2524BC6
:102D8800197821EA02021A70642333702378013318
:102D98002370CFE03078002840F0CC80484A0323E5
:102DA80023701378013BDBB21370002B00F0948082
:102DB800C3E0404A414E92F86A201AB13278002A9C
:102DC80040F0B88000223270013212FA03F3DFF8C3
:102DD800E0803E4F98F800104FF00E0909FB017291
:102DE800DB4392F803E0DBB203EA0E0E907882F838
:102DF80003E092F804E003EA0E0E0340937082F8B1
:102E080004E00DF10700FFF733FC98F8003009FBE8
:102E18000372D278DFF894902AB999F8002002F06A
:102E28000302012A0AD00E2202FB03721279B2B9F8
:102E380099F8002002F00302022A10D10E2202FBA8
:102E48000377BA785AB9224F3A789A4207D1184884
:102E5800FFF78AFE3B78013303F01F033B7099F8B4
:102E680000009DF8071000F00300FFF761FA144B0B
:102E78000422FF281A7088F80000164B42D0987870
:102E880000F04000C0B200283CD1032323701A335D
:102E9800337052E0002020704FE000BF6A14002019
:102EA800D7100020D41000206214002063340020C2
:102EB8009E120020E8330020D5100020D2100020F8
:102EC800601400206B14002061140020A012002060
:102ED800EB140020B0310020FFF73EFB00232370E5
:102EE8001DF0ACFE2B78013BDBB22B702BB1144BE1
:102EF8009B7803F04003DBB2F3B19DF80700FFF7BE
:102F080057FE19E09B780E4A03F04003DBB22BB161
:102F1800136843F400031360FFF7D2F8FFF71CFBB4
:102F28001DF08CFE002323704FF474500DF074FED6
:102F3800287001E0002000E0FF20BDE8FE8300BF0C
:102F4800B0310020044B1A780AB1013A1A701B7884
:102F58000BB9FFF72DBE70476A140020044A054BD1
:102F680010781B7803EA501000F00100704700BF8A
:102F7800B031002097160020044B054A1B781078C2
:102F8800C3F3400303EA1010704700BF97160020F0
:102F9800B0310020034B044A1B78D078C3F3800378
:102FA8001840704797160020B0310020044B054A9E
:102FB8001B78D078C3F3C00303EA5000704700BF02
:102FC80097160020B0310020044B054A1B78D078B2
:102FD800C3F3001303EA9000704700BF9716002060
:102FE800B0310020044B1878044BDB785B005BB2EF
:102FF800DB1103EAD010704797160020B03100208B
:103008002DE9F041154E0024B04620E0204629461F
:103018001AF0ECFD90B1F35DFF2B0FD04FF4A073C5
:1030280063430A2202FB053318F80330DB0905D095
:103038000B4B1878C0F30010BDE8F08101350A3752
:10304800202DE3D10134022C06F5A07602D000270A
:103058003D46DBE70020BDE8F08100BF35350020A4
:103068009716002008B51AF0D1F9034B1B7800EA2F
:10307800931000F0010008BD97160020044B054A84
:103088001B78D078C3F3401303EAD000704700BF21
:1030980097160020B03100202DE9F84FFFF75EFFAA
:1030A8008146FFF769FF8246FFF774FF8346FFF703
:1030B8007DFF8046FFF788FF0446FFF7A1FF05461E
:1030C800FFF7DCFF0746FFF7CDFF0646FFF78AFF4D
:1030D8004FEA8B0343EA4A0343EA090343EAC80376
:1030E80043EA471343EA861345EA040443EAC01354
:1030F800E0B243EA0010BDE8F88F0000044B98786E
:1031080000F00F00A0F10203584240EB03007047A3
:1031180035150020044B987800F00F00A0F101024B
:10312800504240EB0200704735150020044B987858
:1031380000F00F00A0F10301484240EB0100704786
:1031480035150020054B987800F00F00A0F1060C0B
:10315800DCF1000040EB0C00704700BF3515002083
:10316800514AF0B513781446012B29D003D3022B0A
:1031780040F098805EE04D484D4B047819786FF325
:10318800C304047001F0F80158786FF3C301197093
:1031980000F08001C9B2002900F08480012111707B
:1031A8009C78062204F00F04544302464148005D0F
:1031B80060F306025A701A7861F302021A70F0BDC1
:1031C8003B494D780B4625F07F00002838D00A7817
:1031D80002F00802D2B222B9344A117841F008014B
:1031E80011709A7802F00F02012A04D12F4A11783F
:1031F80041F00101117015F07F0F53D119789E78B5
:1032080001F00700062206F00F0602FB0606294F0A
:103218005D78BE5D013066F3060500F007005D705D
:1032280090FBF2F502FB150262F30201197002230A
:103238002370F0BD1E494D780B4625F07F0028B954
:103248008B7860F303038B701070F0BD174A117808
:103258006FF3C3011170997801F00F01012903D1AF
:1032680011786FF30001117015F07F0F1AD11978DA
:103278009E7801F00700062206F00F0602FB0606FC
:103288000C4F5D78BE5D013066F3060500F007005F
:103298005D7090FBF2F502FB150262F302011970F2
:1032A80001232370F0BD00BF84150020F71400200F
:1032B80035150020303C020810B51F4A1F4B92F903
:1032C800031009B1002231E008B1032119701978FF
:1032D800032930D8DFE801F00209192C11780029F8
:1032E80029D0154881700121197092F902001249FC
:1032F80020B1134B1A786FF3861217E0487808B993
:10330800032213E088700221197092F902100A480A
:1033180089B90B4A147861F386141470026861F352
:103328000F22D1B261F31742026001221A7010BD58
:1033380000211160197010BD2C170020F514002011
:103348004033002038B5044643F6EF2343F6F02017
:10335800012A08BF18460D460DF05EFC2378C0B25E
:103368001842104C09D043F6EE200DF055FC2368A6
:1033780060F307036FF30F230CE02B7818420AD091
:1033880043F6EE200DF048FC2368C0B260F3070353
:1033980060F30F23236094F9003013B1014B0F221F
:1033A800DA7038BD2C17002008B543F6F7200DF069
:1033B80033FC014B187008BDF6140020014B18703F
:1033C800704700BFA0160020024B1A5C6FF303027F
:1033D8001A547047DE15002070B50C46C10001F57F
:1033E800CE411B488B3108220DF027FC00251848D8
:1033F8002946EEB21EF0EDFE08B9237823BB154B23
:103408002278EB5C1A421FD13046FFF7DDFFF60841
:103418004AF2B34030180DF0FFFB05F00703C0B2C5
:10342800184110F0010F0FD10B4829461EF0D1FEAC
:1034380050B1294608481EF0C1FE074B06F5CC409E
:10344800CA30995D0DF0DEFB0135402DCFD170BD3E
:10345800A2160020951500203815002038B546F230
:10346800127540242046FFF7AFFFA5F5CC43094A63
:10347800D23BD15C11F0100F06D06FF30411D15478
:10348800284600210DF0BEFB0134E4B20135B92C09
:10349800E8D138BDDE1500203F287FB5054607D89E
:1034A80000F5E2400D300DF0B7FBC3B22BB92AE1AD
:1034B800994A1478002C00F02B81984E725D02F026
:1034C8000F014C1C04F00F0464F303023F2D7255E6
:1034D80033D8002C00F01C8101339C4240F0158148
:1034E8008F4B5A1992F88020522A725D03D161F3EA
:1034F8000302725509E16FF30302EC081B197255B8
:1035080093F8902105F0070352FA03F313F0010F23
:1035180040F0FD80294683481EF045FE814B04F5A6
:10352800CC40195DCA3001240DF06CFB2D19022323
:103538000093019402951820CEE0002C00F0E8805A
:10354800754B1B7801339C4240F0DF80735D05F5B5
:10355800CC406FF30303D230012173550DF052FBB9
:10356800735D43F010037355A5F14003DBB2032BE1
:1035780007D80422009201330232019202931920E3
:103588002FE0A5F14803DBB2032B07D804220092F1
:1035980001330332019202931A2060E0A5F150032F
:1035A800DBB2012B07D804220092013303320192C7
:1035B80002931B2053E0572D07D1042300930124C5
:1035C800033301930294212086E0A5F15B03DBB26B
:1035D800012B09D80422009201330232019202938E
:1035E80022200121033A8AE05D2D06D104230093AD
:1035F8000193043B029328467FE05E2D07D1042304
:10360800009301330193053B02935E2075E0A5F119
:103618005F03DBB21F2B09D80422009201339218F2
:103628000192029333200121053A68E005F1610314
:10363800DBB2032B07D80422009201330332019234
:1036480002935F200BE005F15903DBB2012B09D887
:103658000422009201330332019202936020012177
:10366800043A4CE0AA2D07D1042300930124043B1B
:103678000194029361202FE0A92D07D10423009320
:10368800023B0193023B0293622036E0AD2D08D144
:10369800042300930322043B019202936320012137
:1036A8002DE0AB2D06D104230093043B0193029334
:1036B800642022E0AC2D06D104230093043B01933F
:1036C8000293702019E0AE2D0CD10423009301243D
:1036D80002330193029468202146032223460DF009
:1036E80019FB15E04E35EDB2012D10D804230093D7
:1036F80001350233019302956A20012103220B460A
:103708000DF008FB03E01C4602E0002400E0012461
:10371800204604B070BD00BF00000020DE15002068
:10372800E023002038150020024B185CC0F300107D
:10373800704700BFDE150020F8B508220E460021AC
:103748000746FCF727FE46F28B75002433782341A1
:1037580013F0010F08D02946064808220DF06DFA2B
:10376800384604491EF0EDFC01340835042CEDD12F
:10377800F8BD00BFAC160020024846F2CA61082214
:103788000DF05BBA3815002070B5044600F56A5094
:1037980044300DF041FA0B4D06462B7813F0010F1B
:1037A80002D1CC201FF002FB2B8843F001032B80B1
:1037B800054B1E55054B13F8242042F0010203F86F
:1037C800242070BDBE160020191500200815002001
:1037D800024B185C084100F0010070479515002065
:1037E80070B505460024094BE0B2E618E35C4BB11E
:1037F8002946FFF7EDFF28B100233370044821461E
:103808001EF0DCFC0134402CEDD170BDE016002028
:103818002515002038B5054600242846E1B2FFF7F3
:10382800D7FF10B1044BE35C23B90134042CF4D165
:10383800002038BD012038BD1915002038B50546CF
:103848000DF05EFDA0B100242846E1B2FFF7C0FFED
:1038580040B1084B13F8243013F0010F02D0064B87
:10386800E35C23B10134042CEED1002038BD0120E3
:1038780038BD00BF0815002019150020F8B51148FB
:1038880000214022FCF786FD46F28B7500240127B3
:103898000D4829460822A7400DF0CFF9FFB20026AF
:1038A800094831461EF095FC20B1064BF25C47EA08
:1038B8000202F2540136402EF2D101340835042CAC
:1038C800E5D1F8BD95150020AC1600202DE9FF4183
:1038D80000263446B0461A4B1B78234113F00102E8
:1038E800184B23D0184F1D5D17F82430A84538BF52
:1038F800A84613F0010F1AD0CDB965F3000307F8F5
:10390800243023B20122F71902935B2029462B4663
:10391800009201950DF0FEF97B78B878F978184394
:10392800621C2B460095FEF7E7FE00E01A550134AD
:103938000436042CCFD1054B83F80080BDE8FF8105
:10394800F61400201915002008150020F414002092
:1039580010B50C4B1B78A3B10B4B1B788BB1002413
:103968000A4821461EF035FC40B1094821461EF0A0
:1039780030FC18B920460121FEF7ECFF0134402C39
:10398800EED110BD69140020D6100020C816002002
:10399800461E00202DE9F043324C334A2388002686
:1039A8006FF386136FF3C4032380304B304F85B019
:1039B80016701E709146984617F8013B5BB3227843
:1039C800D20052B243EAA2122388402E62F3C40303
:1039D80043F0400323801ED000253046E9B2FFF7AC
:1039E800F7FEA8B117F8013C13F0010F06D0012229
:1039F800AA4099F800100A4389F8002013F0020F32
:103A080006D00123AB4098F80020134388F8003013
:103A18000135042DE1D10136F6B2412ECCD12378FF
:103A280003F04005EDB2D5B903F02403042B0BD104
:103A3800FFF78EFFFF2300934020294602222B46E2
:103A4800019502950DF066F9238800226FF345135E
:103A58006FF382036FF3C4032380064B1A7005B01B
:103A6800BDE8F083BE160020DC320020F9320020C9
:103A780043150020A116002010B500240548214652
:103A88001EF0A7FB08B9044BE0540134402CF5D1D3
:103A980010BD00BF981600204315002010B51278FD
:103AA80004469DF80810DAB1D3B111B10D491EF0E2
:103AB8003DFBACB1082246F2CA610B480DF0BDF8D7
:103AC800214609481EF03DFB0749082246F2CA6014
:103AD8000DF0ADF805480449BDE810401EF047BB9D
:103AE80010BD00BF78250020EC14002038150020F8
:103AF80030B5064B04781D7824EA05040C7001786B
:103B08001B7823EA0103137030BD00BFF6140020B0
:103B180038B50A4D002415F8013F2D2B09D0532B39
:103B280007D0542B05D0462B03D0054821461EF05C
:103B380045FB0134402CEED138BD00BF5F24002086
:103B4800C816002010B50F481EF0E8FA00240E48E9
:103B580021461EF03EFB80B10C4BE31893F88030F1
:103B6800482B06D003D82D2B03D0462B00E0542B2E
:103B780003D1044821461EF016FB0134402CE6D13F
:103B880010BD00BF85150020C8160020E0230020C6
:103B9800094A0A4B117831B1997801F00F01814235
:103BA80001D0002111709A7860F303029A705A7854
:103BB80042F080025A7070478415002035150020A5
:103BC8007FB5604B154604461A780E4600235E49B9
:103BD80011F8231011F0010F05D001219940C1F10E
:103BE8000F0101EA02020133042BF0D1574B1A707E
:103BF800002C6FD014F0010F0AD0FF23012100938D
:103C0800FF3B0193029352200A460B460DF082F8BF
:103C180014F0020F0AD0FF2301210093FF3B019308
:103C2800029353200A460B460DF074F814F0040F63
:103C38000AD0FF2301210093FF3B019302935420F4
:103C48000A460B460DF066F814F0080F0AD0FF2359
:103C580001210093FF3B0193029355200A460B462E
:103C68000DF058F814F0100F0AD0FF23012100932B
:103C7800FF3B0193029356200A460B460DF04AF883
:103C880014F0200F0AD0FF2301210093FF3B01937A
:103C9800029357200A460B460DF03CF814F0400FEB
:103CA8000AD0FF2301210093FF3B01930293582080
:103CB8000A460B460DF02EF814F0800F0AD0FF23A9
:103CC80001210093FF3B0193029359200A460B46BA
:103CD8000DF020F8CEB10024284621461EF079FACE
:103CE80060B1FF230093FF3B0193631C1BB20121CA
:103CF80002935A200A460B460DF00CF82146284636
:103D080001341EF05BFA402CE6D110481049114AE4
:103D1800FFF7EEFE104B00221A70013200920632B5
:103D28000192083202920A490A4A08480AF058FBE6
:103D38000A4B3C2251201A7004B0BDE870400DF0C7
:103D4800C5BB00BFF6140020081500203818002055
:103D58000E19002002190020FD1700201815002058
:103D680010B5FFF799F9044607481EF005FAD0F197
:103D7800010138BF002104B929B1034A2046BDE832
:103D88001040FFF71DBF10BDD6150020054B03EBF3
:103D9800D00393F8903100F0070053FA00F000F0D8
:103DA80001007047E023002010B50F4B04461B7834
:103DB80013F0010315D0FFF72DFD28B90B4B1B1984
:103DC80093F88030462B0DD10DF09AFA18B9204699
:103DD800FFF7DCFF30B1064821461EF0E4F9012068
:103DE80010BD184610BD00BFBE160020E0230020FD
:103DF800D6150020024B1878003818BF01207047EC
:103E08001815002010B5034C04EB83035870997003
:103E1800DA7010BD0815002010B5002409480021EB
:103E280000190E220E34FCF7B5FAB4F5E07FF5D18F
:103E3800054A00231370054A002199520233AA2B20
:103E4800F9D110BDD8100020D3100020821900200D
:103E58007FB5474B04461B780E46AA2B78D04548B9
:103E680021461EF0B6F90546002871D12046FFF715
:103E78009BFF00286DD1404821461EF0AAF950B991
:103E88003E4821461EF0A5F9054620B92046FFF711
:103E980003FB00285DD13A4B1B7823B9394B1B78BB
:103EA80013F0010F09D1384BDB7803F02003DBB2A4
:103EB8001BB9364B032283F84020012E05D82E4823
:103EC80021461EF086F940B142E0022E07D12B4868
:103ED80021461EF07EF910B13AE0274800E0274855
:103EE80021461EF060F92A4821461EF067F9022E85
:103EF80015D10125294603222B4600964A2066192A
:103F0800019502960CF006FF2046FEF731F90023D2
:103F18000246314618200093FEF7EEFB19E0012E09
:103F280009D102230093631C0293019612203146A3
:103F38000322334609E07EB9012102230093631866
:103F480002930191112003220B460CF0E3FE03E0DB
:103F58000025284604B070BD2046FEF709F9024640
:103F680001200023211800930125FEF7C5FBF0E787
:103F7800A016002038150020F81400202017002073
:103F8800F61400207E190020B031002043150020CF
:103F9800D01600202DE9FF4704460D4675482146F6
:103FA8001EF017F98146002840F0DF80214671484D
:103FB8001EF0F9F8704821461EF000F96F4E0DBB4F
:103FC80001274FF00208E3190293424603203946BD
:103FD8003B46CDF8008001970CF09CFE327862B128
:103FE8000DF08EF9024630B1337840461E33009307
:103FF80021462A4604E0009000E00092404621460F
:104008003B4628E0012D2BD15D4B04F5E2400D30F5
:104018001F5D0CF001FE07F00F07874209DA631CE9
:10402800022202930E2029462B46009201950CF09D
:1040380071FE327892B10DF063F9024638B14F4BF8
:104048000D201B7821461E330093002202E00090C9
:104058000D2021460123FEF74FFB5EE00092F7E7B3
:10406800022D0BD101230193E31802931420494632
:104078002A464B4600950CF04DFE4EE0032D4CD1E0
:1040880001272A464FF0020804EB070A4D2039465B
:104098003B46CDF800800197CDF808A00CF03AFE19
:1040A80035783DB30DF02CF9024630B133784046EF
:1040B8001E33009321464A4602E0009021464046BE
:1040C8003B46FEF719FB0DF01BF9671C054648B186
:1040D8002046FEF74DF8337802461E3300931A2027
:1040E80039462CE02046FEF743F80095024639464B
:1040F8001A202DE021462A463B4640460095FEF709
:10410800FBFA2046FEF734F8514602462B461A20A1
:104118000095FEF7F1FA384628E03578EDB10DF054
:10412800EFF804F11C06054658B12046FEF720F8C2
:10413800124B02461B7830461E330093611C002345
:1041480007E02046FEF714F8009502463046611C49
:104158002B46FEF7D1FA012008E02046FEF708F8C2
:104168000095024604F11C00F1E7002004B0BDE808
:10417800F08700BFC8160020D0160020281700209E
:10418800DE150020064B1B1893F84001492804D07F
:10419800452814BF0320022070470120704700BF44
:1041A800E02300202DE9F041244F00243C702448EE
:1041B80021461EF00EF8E5B2224B002837D01E5DCE
:1041C8003B789E4200D303B93E70002E30D1314671
:1041D8001C484022FCF7DEF81B4B1C4803EBD503B8
:1041E80093F8888104F0070348FA03F8214608F099
:1041F80001081DF0EEFF68B9B8F1000F02D028469B
:10420800022101E028463146FFF7C4FE28460DF09A
:104218005DF90DE0B8F1000F0AD12846FFF7B2FFAB
:104228000B4BDB7803F02003DBB20BB9094B1855B5
:104238000134402CBBD1BDE8F08100BF2817002015
:1042480025150020E0160020E0230020C8160020D5
:10425800B0310020431500202DE9F04F914B89B073
:104268001B7813F0010F06D08F4B1A786FF3861264
:104278001A7001F022BA8D498D4A0B7810788D4D4D
:10428800984218BF8C49137018BF0B706B7803F0F5
:104298000803DBB24BB143F6CF200CF0BDFC864BD4
:1042A80018702B886FF3CB232B80844B1B78AA2B99
:1042B80008D18349AA3B0B702B8843F080032B80DD
:1042C80000F076BE6A787B4B02F01002D2B27D4CC9
:1042D800A2B11A886FF30C321A807B4B1B7823B972
:1042E8007A4B1B7813F0010F08D1E37803F0200311
:1042F800DBB21BB9764B032283F840202368754F45
:104308006FF3186323603A7802F00202D2B232B92E
:104318006B494A781AB16B4A43F080731360E678A8
:1043280016F0010648D05D20FFF7FEF900285AD1A3
:104338006B78DFF8808103F00203DBB22BBB5D30C2
:10434800FFF7AAF8064600BBB8F80030012143F48D
:104358000073A8F80030042303220093019302900D
:104368000B460D200CF0D6FC45200DF0AFF8314679
:10437800012233460D200096FEF7BEF9092031468A
:10438800324601230096FEF7B7F96B7803F0020373
:10439800DBB243B34C4B1B7823B94C4B1B7813F05F
:1043A800010F20D1E37803F02003DBB2DBB9484BDF
:1043B800032283F8402016E06B7803F00203DBB297
:1043C8006BB13146324601230A200096FEF794F974
:1043D8008D203146012233460096FEF78DF92B8851
:1043E8006FF349232B802368354A6FF359632360A1
:1043F80093787BB1D37823B93B7813F00C0F05D1B0
:1044080008E03B7803F00C03042B03D0236843F047
:1044180000732360E17801F00201C9B200295BD082
:104428005E20FFF781F9002865D16B78214F03F0F2
:104438000403DBB2EBB95E30FFF72EF80646C0B9CD
:104448003B88012143F480633B80042300930133BC
:104458000322019302900B4617200CF05BFC4520C9
:104468000DF034F80D203146012233460096FEF750
:1044780043F96B7803F00403DBB2002B3BD0124BFB
:104488001B7823B9114B1B7813F0010F33D1E37854
:1044980003F02003DBB273BB0D4B032283F84020EB
:1044A80029E000BF3918002040330020AA16002058
:1044B800AB160020BE16002029170020A0160020E9
:1044C800600E0020B0310020F61400207E19002074
:1044D80043150020DE2300206B7803F00403DBB2D1
:1044E8002BB18D2001220B460091FEF705F92B8890
:1044F8006FF38A232B802368DFF8DCB26FF3DF7356
:1045080023605F2306930026D94696E03046394655
:1045180019F06CFB002871D01BF80A30FF2B6DD006
:104528004FF4A0727243A8F15E03DBB207930A232B
:1045380003FB072219F802E009EB02035FEADE1E1B
:1045480050D02268404642F0004222600593FFF7AF
:10455800EBF8059B00285CD11A7912F0040F24D1DE
:104568004046FEF799FF059B8446F0B91A79322038
:1045780042F004021A710799042300930291DB1890
:104588000121032201930B46CDF814C00CF0C2FBA5
:104598004A200CF09BFFDDF814C00C20079901227B
:1045A8006346CDF800C0FEF7A7F84FF4A073734335
:1045B8000A2202FB07334B441B7913F0040F28D05F
:1045C800804B1B7823B9804B1B7813F0010F20D147
:1045D800E37803F02003DBB2DBB97C4B032283F8DA
:1045E800402016E01B7913F0040F07D08C200799A0
:1045F80001227346CDF800E0FEF77EF84FF4A07371
:1046080073430A2202FB07334B441A796FF3820281
:104618001A71013708F10108202F5FFA88F80AF1AA
:104628000A0A7FF473AF069A013602F12003DBB25F
:10463800022E0BF5A07B069305D04FF0000ADDF89B
:104648001880574662E72368614923F080636FF357
:104658009E7323600B79002B00F017845D4ADFF806
:104668007CB106924FF09F0800271BF8011F3E46B9
:104678000137002952D02368A8F15F0A43F080630C
:104688005FFA8AFA23605046FFF74EF800285CD19B
:1046980017237343DFF8489119F8032012F0100F1D
:1046A80023D150460593FEF7F7FE059B8246E0B9F5
:1046B80019F80320012142F0100209F8032004230D
:1046C8000093023301933BB2032202930F200B465F
:1046D8000CF020FB45200CF0F9FE0D20514601227C
:1046E8005346CDF800A0FEF707F81723734319F8CF
:1046F800033013F0100F28D0324B1B7823B9324BFC
:104708001B7813F0010F20D1E37803F02003DBB20C
:10471800DBB92E4B032283F8402016E0172373439E
:10472800DFF8BC9019F8033013F0100F05D08D2076
:1047380001220B460091FDF7DFFF1723734319F899
:1047480003206FF3041209F80320069A12F8011FD8
:104758000692002946D02368404643F080432360F0
:10476800FEF7E2FF002854D14FF0170909FB06F9BC
:10477800DFF86CA01AF8093013F0200F49D1404631
:10478800FEF78AFE0646002843D11AF809300121AF
:1047980043F020030AF809300423009303330193FC
:1047A8003BB2032202934B200B460CF0B3FA502085
:1047B8000CF08CFE19203146012233460096FDF795
:1047C8009BFF26E0F61400207E19002043150020E8
:1047D800600E002050320020353500207532002050
:1047E8007D32002017237343DFF8FC9219F8033059
:1047F80013F0200F05D0992001220B460091FDF7F8
:104808007BFF17235E4319F806306FF3451309F849
:10481800063008F10108042F5FFA88F87FF425AF05
:10482800AA4ADFF8C8B206924FF05008043F1BF8B6
:10483800011F3E460137002950D0236808F1620A5B
:1048480043F080635FFA8AFA23605046FEF76CFFF4
:10485800002858D1DFF89892330119F8032012F094
:10486800400F23D150460593FEF716FE059B82465E
:10487800E0B919F80320012142F0400209F80320A9
:1048880004230093023301933BB20322029369206D
:104898000B460CF03FFA45200CF018FE0D2051464F
:1048A80001225346CDF800A0FDF726FF330119F881
:1048B800033013F0400F26D0854B1B7823B9854B66
:1048C8001B7813F0010F1ED1E37803F02003DBB24D
:1048D800CBB9814B032283F8402014E0DFF8109213
:1048E800330119F8033013F0400F05D08D20012251
:1048F8000B460091FDF700FF330119F803206FF311
:10490800861209F80320069A12F8011F0692002958
:1049180033D02368404643F080432360FEF704FF0A
:1049280000283FD1DFF8C8A14FEA06191AF8093064
:1049380013F0200F36D14046FEF7AEFD064688BB81
:104948001AF80930012143F020030AF8093004233A
:104958000093033301933BB20322029310200B46CA
:104968000CF0D8F950200CF0B1FD19203146012285
:1049780033460096FDF7C0FE14E0DFF8749133016A
:1049880019F8033013F0200F05D0992001220B46A7
:104998000091FDF7B1FE360119F806306FF34513A3
:1049A80009F8063008F10108022F5FFA88F87FF449
:1049B8003EAF4A4B1978002946D02368AE2043F011
:1049C80080632360FEF7B0FE00284CD1444B1A7870
:1049D800984612F0400F20D1AE30FEF75DFD074635
:1049E800D8B998F80030012643F0400388F8003021
:1049F8000423009302333146032201936720334690
:104A080002960CF087F945200CF060FD0D20394620
:104A180032463B460097FDF76FFE98F8003013F0DA
:104A2800400F20D02A4B1B7823B92A4B1B7813F050
:104A3800010F18D1E37803F02003DBB29BB9264BB2
:104A4800032283F840200EE0254E337813F0400F00
:104A580005D08D2001220B460091FDF74DFE3378DD
:104A68006FF3861333701F4B1978002942D02368DF
:104A7800572043F080432360FEF756FE002848D1B4
:104A8800174E337813F0200F43D15730FEF704FD4B
:104A9800074600283DD13378032243F020033370C2
:104AA8000423012600930333314601931F20334624
:104AB80002960CF02FF950200CF008FD1920394609
:104AC80032463B460097FDF717FE22E0B33100203F
:104AD800F61400207E19002043150020EC31002038
:104AE80000320020F13100207D32002040320020C9
:104AF800213200209E4E337813F0200F05D09920E4
:104B080001220B460091FDF7F7FD33786FF345134B
:104B180033704FF000094FF0A70AC8464E46954B30
:104B280008F10108F15C00294ED02368AAF14C0B6A
:104B380043F080635FFA8BFB23605846FEF7F4FD71
:104B4800002854D1182373438B4FFA5C12F0200FBE
:104B580022D158460593FEF79FFC059B8346D8B99A
:104B6800FA5C012142F02002FA5404230093023334
:104B780001930FFA88F30322029320200B460CF0CE
:104B8800C9F845200CF0A2FC0D20594601225B46CD
:104B9800CDF800B0FDF7B0FD18237343FB5C13F0AC
:104BA800200F24D0754B1B7823B9754B1B7813F055
:104BB800010F1CD1E37803F02003DBB2BBB9714BC2
:104BC800032283F8402012E0182373436A4FFB5CEA
:104BD80013F0200F05D08D2001220B460091FDF720
:104BE8008BFD18237343FA5C6FF34512FA54664B36
:104BF800F15C002936D02368504643F08043236097
:104C0800FEF792FD002842D15B4B4FF0180B0BFBCF
:104C1800063B9BF8013013F0200F38D15046FEF7C1
:104C28003BFC0746002832D19BF80130012143F0B4
:104C380020038BF8013004230093033301930FFA08
:104C480088F3032202934C200B460CF063F85020A3
:104C58000CF03CFC1920394601223B460097FDF731
:104C68004BFD14E0444F182303FB06735B7813F0E5
:104C7800200F05D0992001220B460091FDF73CFD3D
:104C8800182303FB06777B786FF345137B703F4B44
:104C98001B78002B00F090803D4B374FF35C1822B7
:104CA800002B77D002FB06F3FA5C07EB0901C2F38D
:104CB800801BBBF1000F1BD142F04002FA5478224E
:104CC80004234A800093DB18012101930FFA88F32B
:104CD800032202932E200B460CF01CF846200CF001
:104CE800F5FBCDF800B00920414601225B4661E0A2
:104CF800B1F9021029BB5FEAD21B22D143F6DE20AC
:104D080005930BF089FF059BD8B1FA5C012142F0AD
:104D18008002FA5404230093DB1801930FFA88F3F6
:104D2800032202932F200B460BF0F4FF47200CF0D0
:104D3800CDFB0920414601225B46CDF800B0FDF7C6
:104D4800DBFC18237343FB5CDB0935D00B4B1B786A
:104D580023B90B4B1B7813F0010F2DD1E37803F027
:104D68002003DBB243BB074B032283F8402023E038
:104D7800003200204E320020BC310020F614002002
:104D88007E1900204315002044320020F93100200C
:104D9800F33100207243B95C11F0400F0CD063F37B
:104DA800861163F3C711B9544F447B80892000935F
:104DB80041460122FDF7A0FC01360AF1010A022E44
:104DC80009F118095FFA8AFA7FF4A9AEDFF8C4A3DB
:104DD8004827023E1AF8011FB0460136002937D08D
:104DE8002368384643F080432360FEF79DFC002883
:104DF80047D14FF01D0909FB08F9DFF884B31BF808
:104E0800093013F0200F3CD13846FEF745FB8046A9
:104E1800002836D11BF80930012143F020030BF894
:104E28000930042300930333019333B2032202931E
:104E380013200B460BF06EFF50200CF047FB192097
:104E4800414601224346CDF80080FDF755FC18E0A5
:104E58001D2303FB08F3DFF8289319F8033013F038
:104E6800200F05D0992001220B460091FDF744FC44
:104E78001D2303FB08F819F808306FF3451309F8E8
:104E880008300137042EFFB2A4D1A37803F0080339
:104E9800DBB2002B40F08C8048F6F234A4F50A47C8
:104EA800A7F5F977A14839461DF093F928B9A04824
:104EB80039461DF08EF9002874D09E4839461DF0F9
:104EC80088F900286ED139469A481DF06CF92046B9
:104ED8000BF0A2FE984EC0B23070002862D00138A4
:104EE800C0B230700BF002F800285BD13078934ED6
:104EF80000F56A5078300BF08FFE914BC0B214F871
:104F08000380307000EA0808394688481DF061F9C6
:104F1800DFF87CA2DFF82C9238B1854839461DF0BD
:104F280058F910B99AF8003014E0814839461DF054
:104F380050F938B17D4839461DF04BF910B99AF847
:104F4800003004E09AF8003018EA030F02D023EA90
:104F5800080801E048EA03087A487B4989F8008094
:104F68007A4AFEF7C5FD7848794911F0EDFF68B136
:104F78000CF0C6F950B9764809F09CFA30B901230B
:104F880073487449704A0093FEF788FD0023009324
:104F98000133019333786B4802936B496B4A6D4B2D
:104FA80009F01EFA013448F632439C427FF476AF8A
:104FB800694C63786FF3C71363702B7803F0800232
:104FC800D2B2002A00F0F08064490E78002E40F03A
:104FD800EB8003F02403042B0BD1FEF7B9FCFF236D
:104FE80000934020314602223346019602960BF088
:104FF80091FE2B8800266FF3C7136FF3820366F3C5
:10500800451366F3410366F30003554A66F34923E3
:1050180066F38A2316702B80524B1A7842F0C0022E
:105028001A705A7866F3C3025A70FEF771FD4E483B
:105038001DF074F84D481DF071F84D481DF06EF8DC
:1050480041224C483146FBF7A5F94B4B1A7802F040
:10505800DF0266F304121A70DA7D02F0DF0266F3EB
:105068000412DA7593F82E2002F0DF0266F30412B8
:1050780083F82E2093F8452002F0DF0266F304122D
:1050880083F845203D4B1A7802F0DF0266F386125A
:105098001A701A7C02F0DF0266F386121A74384B13
:1050A8001A7866F345121A705A7F66F345125A77D2
:1050B80093F83A2066F3451283F83A2093F857207C
:1050C80066F3451283F857202E4B1A7802F0DF0258
:1050D80066F386121A702C4B5A7866F345125A708A
:1050E8001A7802F07F0266F345121A705A7E66F348
:1050F80045125A761A7E02F07F0266F345121A7636
:1051080011E04FF4A07272430A2101FB03221F49E8
:1051180001338A181179202B6FF382011171F0D1B4
:105128000136022E38D00023EBE700BFC42300204D
:10513800CC230020D4230020D5150020CE18002031
:10514800AE98FF1F381800200E1900200219002001
:1051580000150020FD17002035150020600E0020E6
:10516800A11600204033002020170020F81400204A
:1051780025150020431500207D3200202132002013
:105188005B33002000320020BC3100203535002080
:10519800F61400201C32002004226F480021FBF77F
:1051A800F9F86E4B00221A706D4F3878002846D1F6
:1051B8002A786C4B02F00202D2B2CAB16A4A51781C
:1051C80060F3C30151701A88CA3042F080021A8015
:1051D8001DF0ECFDC6201DF0E9FD1DF035FE634A0B
:1051E80013780BB90CF0FEF9FEF738F9FEF714FE48
:1051F8005F4A2B8811786FF341036FF300016FF357
:10520800000311705B48002140222B80FBF7C2F895
:1052180059481CF083FF59481CF080FF58481CF07F
:105228007DFF58481CF07EFF04224B480021FBF705
:10523800B1F84A4A00231370534A137067E02E7876
:1052480006F00203DBB293B916F001060FD14A4803
:105258001CF064FF3B78F0B2334113F0010F03D028
:10526800FEF792FA0CF042F80136042EF2D12B78B0
:105278003C4E13F0010F22D0FEF772FD338843F045
:1052880002033380FEF722FB344B1F78A7B9CA20EC
:105298001DF08CFDCD201DF089FD33883B4867F358
:1052A80000033380324B1A7842F001021A701CF066
:1052B80035FFFEF7D3F802E00120FEF769FC2B78F2
:1052C80003F00202D2B212B32F4A12782AB113F0B5
:1052D800010F02D10220FEF75BFCFEF763FF2C49A9
:1052E80026481CF039FF254925481CF01FFFFEF70A
:1052F80029FC224927481CF019FF274925481CF09A
:1053080020FFFEF7B9FB1F481C491CF030FF20495D
:1053180022481CF00BFF15490B780BB9FEF73AFB36
:10532800637803F08003DBB2002B3FD12B7803F0C6
:105338002403042B06D143F6EC200BF06DFC08B1D6
:10534800062031E0FEF756FD08B105202CE00CF0F0
:1053580033FA28B3032027E019150020F41400209D
:10536800F6140020BE16002040330020600E0020F6
:10537800F7140020E01600202529002098160020A8
:1053880025150020D816002028170020D615002043
:1053980038150020C8160020851500201D1500208E
:1053A80001F056F810B10420FEF7F2FB654B1B78AC
:1053B8001BB163786FF3C7136370634A137813B133
:1053C800624B1B78CBB12B78614C03F04403402B24
:1053D80013D10021BF3300933F200B4602220191D5
:1053E80002910BF097FC238843F6CE2043F0040388
:1053F80023800BF011FC574B18705349564E0B780D
:105408009BB1524B197881B92A78514B02F040026E
:10541800D2B252B11A8861F382021A80337823B962
:1054280043F6CE200BF0F8FB30702A78484F02F094
:105438000400C0B2494B002872D002F02000C0B26C
:10544800444C80B11A78002042F0C0021A70FDF76F
:1054580033FF2378002B69D13A8863F3820263F320
:1054680045123A8062E0D20052B219789211D2B253
:1054780041F0C00112F0010F197003D0C9B260F3F6
:10548800C711197012F0020F03D01A786FF3861241
:105498001A701B78314A03F04003DBB21BB953780A
:1054A80043F0080353700120FDF706FF43F6CD20B3
:1054B8000BF0B2FBC0B20128307002D1264B022299
:1054C8001A702478002C31D1FEF742FAFF23022209
:1054D8000093402021462346019402940BF01AFCC5
:1054E8002B8843F6CD2043F020032B800BF094FB50
:1054F800184B1B4A1870154B14701A780AB1013AE8
:105508001A70197891B9104A13787BB1FF23009368
:10551800412002220B46019102910BF0FBFB05E0B2
:105528001A7842F0C0021A70FDF7C6FE0CF0F4F8C3
:105538000C481CF021FE0C4BC0B91A7860F38202AB
:1055480017E000BF4E3A0020AA16002029170020B5
:10555800BE160020A116002042150020403300206E
:10556800600E00208D150020F71400201A7842F0F4
:1055780004021A706A78524812F001011A780CBFB6
:1055880061F3410242F002021A704E491CF0EFFD2D
:105598004D494B481CF0D5FD49484C491CF0D1FDFC
:1055A8003378012B40F089802B8800246FF349233E
:1055B8006FF38A232B80464B41221C7021464548B5
:1055C800FAF7E8FE44481CF0A9FDFEF7A1FA3E48A8
:1055D8001CF0A4FD3D481CF0A1FD404B1A7802F0D8
:1055E800DF0264F304121A70DA7D02F0DF0264F35A
:1055F8000412DA7593F82E2002F0DF0264F3041225
:1056080083F82E2093F8452002F0DF0264F3041299
:1056180083F84520324B1A7802F0DF0264F38612D1
:105628001A701A7C02F0DF0264F386121A742D4B8A
:105638001A7864F345121A705A7F64F345125A7740
:1056480093F83A2064F3451283F83A2093F85720E8
:1056580064F3451283F85720234B1A7802F0DF02CF
:1056680064F386121A70214B5A7864F345125A7003
:105678001A7802F07F0264F345121A705A7E64F3B6
:1056880045125A761A7E02F07F0264F345121A76A2
:1056980011E04FF4A07262430A2101FB032214496E
:1056A80001338A181179202B6FF382011171F0D11F
:1056B8000134022C01D00023EBE709B0BDE8F08FDC
:1056C800A22D0020C8160020F81400202017002062
:1056D8004215002043150020251500207D320020AA
:1056E800213200205B33002000320020BC31002032
:1056F800353500202DE9FF4104460D460CF036F8FB
:105708009E4B1A1992F880709D4A98461278AA2AD8
:105718000AD1A7F14F03DAB20B2A00F2A981994AFC
:105728005BB29A4040F1A481974B0C2202FB0433F0
:105738005A7A0833AA42C0F09B81FF2A00F0988168
:10574800FF229A70914808EBD403214693F88851B8
:105758001CF03FFD0646002840F08A8104F007034C
:105768001D41502F05F0010500F0228114D8462F65
:1057780000F0EE8009D8412F00F09A80452F00F004
:1057880017812D2F40F0728134E0482F00F0C1803E
:105798004F2F40F06B810EE0542F63D006D8522F64
:1057A80000F08680532F40F061811CE0A7F1590377
:1057B800012B00F25B81764821461CF00AFD064663
:1057C800002840F055815A2F01D1724802E0592F24
:1057D80004D1714821461CF0E6FC50E121466D4891
:1057E8001CF0E1FCF5E76D4821461CF0F2FC0028AE
:1057F80000F03E816A4821461CF0EBFC0746002871
:1058080040F03681214666481CF0CDFC65482146AB
:105818001CF0D4FC012602224DB1A41914203946EB
:105828003B460092019602940BF074FA27E1294650
:105838003346671C0A200092019602970BF06AFA19
:105848002046FCF795FC394602462B461320009566
:10585800FCF752FF122029462A4633460095FCF7EA
:105868004BFF0CE14E4821461CF0B3FC07460028CC
:1058780040F005810126022231463346A5193E2013
:105888000092019602950BF045FA2046FCF770FC51
:10589800294602463B4614200097FCF72DFF214677
:1058A8003F481CF080FC21463E481CF087FCE6E09F
:1058B8003A4821461CF08DFC0646002800F0DF809F
:1058C800374821461CF085FC064628B92046FDF7D6
:1058D800E3FD002840F0D380002D40F08E80204664
:1058E800FEF762FA002840F0C5802046FEF74AFC21
:1058F8002D4BDB7803F02003DBB20BB92B4B18558B
:10590800412F00F08880522F40F0B08020460121BE
:1059180083E0234821461CF05CFC28B92046FDF7AB
:10592800BBFD002840F0A480002D66D12046FEF77C
:105938003BFA002840F09E801B4BDB7803F02003E5
:10594800DBB2002B67D1194B032283F8402062E0B9
:10595800134821461CF03DFC064628B92046FDF7B1
:105968009BFD002840F08B802046FEF71DFA00289A
:105978007ED1002D41D1204603214EE0E0230020B6
:10598800A016002000003080B42500203815002023
:10599800D4230020C4230020CC2300209816002004
:1059A800C8160020D0160020B03100204315002072
:1059B800354821461CF00DFC064600285FD02046DD
:1059C800FDF73CFF20B1214630481CF0ECFB4FE0CE
:1059D800502F28D12E4B1B782BBB2046FDF71AFFE2
:1059E80008BB2C4821461CF0F4FB064620B920468B
:1059F800FDF752FD002842D115B1204602210CE0E6
:105A08002046FEF7BFFB244BDB7803F02003DBB214
:105A18000BB9224B185520460021FEF7BBFA061E8B
:105A280018BF01262BE02046FDF7F4FE0546F8B91D
:105A38001B4821461CF0CDFB0646D8B92046FDF789
:105A48002BFD0746D8B9164821461CF0ACFB154A71
:105A5800135D8BB910494E7806F02006F6B26EB980
:105A680008EB040393F80031135508E0012606E01B
:105A7800002604E02E4602E03E4600E01E46304680
:105A880004B0BDE8F08100BF98160020D6150020AC
:105A980028170020C8160020B03100204315002028
:105AA80025150020E0160020032210B505490648F8
:105AB800FAF746FF054806490222BDE81040FAF702
:105AC8003FBF00BF1E210020040200200902002061
:105AD8001C21002070B5804C237813F0010F0AD0E8
:105AE8000BF016FC38B100207C4902F093FE7C4B89
:105AF8007C48197849E07C4D2B78002B4AD00BF074
:105B08000DFC002846D0794B1B7873B9784B5B782D
:105B180013F0010F09D00BF0F3FB30B9237803F031
:105B28002403042B01D10330B6E0724C207870B105
:105B38000020714902F06EFE217801226F4802F0C0
:105B48008FFE00201021621C08F044F802E06C4926
:105B580002F060FE6B4C644808F08CF82378002B48
:105B680000F00F810BF0D4FB002800F00A81664991
:105B780066481022FAF7E4FE64485B21FAF788FCCD
:105B8800002800F0FE80217801308322BDE87040B3
:105B980002F066BE5E4C237803F00503012B5DD14D
:105BA80000205C4902F036FE202110225A48FAF7FC
:105BB800F1FB601D59490322FAF76CFE40BBE01C5B
:105BC80057490222FAF766FE30B95648FAF732FE0C
:105BD8005449024650480BE0E01C53490222FAF7A8
:105BE80059FE40B95148FAF725FE504902464A483D
:105BF800FAF7A6FE0EE0E01C4D490222FAF74AFE2B
:105C080030B94C48FAF716FE4A4902464248EFE7CF
:105C1800FFF74AFF6278303AD3B2092B00F2B1801D
:105C28003B4B9B78303BDBB2092B00F2AA800A2160
:105C380001FB0231C9B2002900F0A380334BFF22D7
:105C48000C291A7740F29D8010295A7740F29980E2
:105C580013299A7740F29580DA7770BD234E33780E
:105C6800F3B9234B5B7813F0010F19D00BF048FB05
:105C7800B0B931481CF080FA68B1304C304B22681A
:105C880002EA03033BB917F0C1FB20B9E37803F03C
:105C98004003DBB223B10020BDE8704009F00ABC24
:105CA800337863B90BF02CFB48B1264B1B7803F013
:105CB8000603042B03D02B780BB90120ECE7FEF781
:105CC80099F810B10020204957E0204B1C78002C8F
:105CD80040D01F4951E000BFBE160020C1CF0208C6
:105CE800F414002000020020F6140020CC18002034
:105CF8007E1900201A180020DCA5020805020020E1
:105D08009AA5020828170020BBA50208F401002064
:105D180019210020E3AA020804020020242B03080A
:105D2800282B030846AB02082B2B030825AB0208D7
:105D38002E2B030804AB02088D150020B03100207B
:105D48003000000FF71400206CB80208650E002020
:105D5800FDA502080B4802F00CFD0A4802F000FD00
:105D6800094802F0FDFC1AF0E7FE084BDB7803F067
:105D78002003DBB22BB106492046BDE8704002F093
:105D880049BD70BD1019002044180020B031002012
:105D9800F5A40208054B1B78D8019B015BB2DB1107
:105DA80040B243EAE070C0B2704700BFBE160020A0
:105DB80070B50E4686B041000122054601F5E9712D
:105DC80005A80AF03AFF0021012E8DF815104FF0B2
:105DD800FF0205F1010305D1009201910293092008
:105DE800FB3A04E00092019102931E2004220B4624
:105DF8000AF090FF05A84249FAF7D0FB50B105A870
:105E08004049FAF7CBFB28B105A83F49FAF7C6FB8A
:105E1800002872D105A83C49FAF7C0FB3B4B044661
:105E2800F8B95A78214642F010025A70FF2302222C
:105E380000930190FE3B02903D200AF06BFF4D203D
:105E48000BF044FB691C0122234612200094FCF746
:105E580053FC12202146224601230094FCF74CFCF7
:105E680003E05A786FF304125A700024284BE35C5D
:105E7800552B07D12846214615F021F810B12046A8
:105E880015F00CF80134082CF0D1002E32D121483D
:105E98002149224AFDF72CFE1F48214911F054F8E8
:105EA800C0B10BF02DFAA8B91D4808F003FB88B95A
:105EB80005A81349FAF772FB012320B90093184883
:105EC8001849154A04E016481649134A0093334600
:105ED800FDF7E4FD144B10491D70002300930533B2
:105EE8000193124B0D4A1B780A4802930D4B08F098
:105EF80077FA02E00E4B00221A7005A806B070BDB2
:105F0800A12B0308312B0308772D03084033002009
:105F1800DD320020381800200E1900200219002058
:105F280000150020FD170020CF330020CE180020D8
:105F38001815002007B54100012201A801F5E971F3
:105F48000AF07BFE002301A804498DF80530FAF712
:105F580025FBD0F1010038BF00200EBDA12B03089E
:105F680007B54100012201A801F5E9710AF065FEB3
:105F7800002301A804498DF80530FAF70FFBD0F18A
:105F8800010038BF00200EBD342D030870B5154B35
:105F980004461B1893F88050B1B1134821461CF0F1
:105FA80018F988B9114821461CF0FDF8A5F15903E4
:105FB800DBB2012B0CD94F2D0AD0542D08D0214625
:105FC8000B481CF0F0F807E0084821461CF0F6F8EA
:105FD800074821461CF0F2F804480649BDE870401D
:105FE8001CF0A4B8E0230020381500208D150020EF
:105FF8002D150020D8160020024B1878C0F3800019
:10600800704700BFF7140020024B1A8860F308227B
:106018001A807047BE160020034B5878C00140B262
:10602800C011C0B2704700BFBE160020014B1878DF
:10603800704700BFF614002030B5457800230021D2
:10604800C218917055FA03F111F0010F08D00649F2
:1060580059188C7C017804EA0101A14208BF9170AB
:106068000133042BEBD130BD1A18002046F67531E8
:1060780004220AF0E2BD000070B5104C054611225A
:1060880020460021FAF786F9002004F8010C2A7846
:10609800103414F8011FC3B291420BD152B1084910
:1060A800013301F8013B112246F6C553BDE87040A3
:1060B80002F0FCBA01300428EBD170BD1B18002097
:1060C8001A1800201FB520B1134B1A8842F48052C9
:1060D8001A80124B00245A78214642F010025A7056
:1060E800FF23022200933D20FE3B019402940AF014
:1060F80011FE4D200BF0EAF920210122234612203F
:106108000094FCF7F9FA1220214622460123009454
:10611800FCF7F2FA1FBD00BFBE1600204033002076
:106128002DE9F3412D4C0722E37848F6883702FB26
:10613800003348F6A930DBB218180AF06DFD25794E
:1061480064795FFA80F8002648FA06F313F0010F25
:106158003AD03946042201A80AF06FFD9DF80400E0
:106168009DF805309DF806109DF8072000282BD0D3
:10617800002929D0002B27D0002A25D0934204D10A
:106188009C4221D185421FD30FE09A4210D99C42EC
:106198001AD3944218D89C4201D994421AD39C42EB
:1061A80001D1854216D294420ED18D420CD811E00D
:1061B8009C4201D185420DD2944201D18D4209D928
:1061C8009C4207D8944205D301360437082EBBD128
:1061D800002000E00120BDE8FC8100BFBC370020A2
:1061E80010B5044648F6E13000EBD4000AF014FD7F
:1061F80004F00704C0B2204100F0010010BD70B5E2
:10620800C30848F6E1355D19044628460E460AF0EB
:1062180003FD04F00704C0B2012126B9A14040EAF9
:106228000101C9B202E0A14020EA01012846BDE807
:1062380070400AF0E7BC0000F0B57C4B8DB0DE780A
:10624800042200EBC606F6B2F10001F5F04104A8FD
:1062580010310AF0F2FC764B764C1A78002304A928
:10626800C95C312905D13039994041EA0202D2B2DC
:1062780005E0302903D12F39994022EA0102013380
:10628800042BECD122706B486B496C4AFDF730FC4B
:10629800694B1B7813B9694B1B78F3B16648684999
:1062A80010F052FE68B10BF02BF850B9644808F0B2
:1062B80001F930B90123624862495F4A0093FDF74A
:1062C800EDFB0023009302330193FD3302935948F9
:1062D80059495A4A5B4B08F083F806EB061100252A
:1062E80001F5F241257004A8D03108220AF0A5FC76
:1062F8002C462F46544B0135E35C542B36D104AB66
:106308001B5D312B03D1204614F0D0FC38B104AB0F
:106318001B5D302B2AD1204614F0C8FC30B34FB98E
:10632800FF2300933420394604223B460197029705
:106338000AF0F0FC04AF385D2146303814F0C4FC94
:106348003B5D0127312B4FF0030305D100932BB29E
:1063580001970293352004E000932BB20197029332
:106368003620002104220B460AF0D4FC0134082C04
:10637800C0D1B10101F5FA4104A8883120220AF000
:106388005CFC083C04AD274615F8013BE6B2013435
:10639800302B03D13046FFF723FF38B115F8013C05
:1063A800312B2CD13046FFF71BFF40B34FB9FF23E9
:1063B80000933420394604223B46019702970AF09D
:1063C800A9FC15F8011C30463039C9B2FFF717FF90
:1063D80015F8013C0021302B4FF0FF0305D1009345
:1063E80023B201910293372004E0009323B2019174
:1063F8000293382004220B460AF08CFC0127202C3B
:10640800C2D1124D6B7803F00403DBB263B1203CB8
:106418002046FFF7E5FE38B90134E4B2202CF7D165
:106428006B7860F382036B700DB0F0BDBC37002051
:10643800F6140020381800200E1900200219002038
:1064480000150020FD170020DD3200204033002019
:10645800014B1878704700BF650E00202DE9F04FFA
:106468004E4B00221A704E4A85B01678002E40F026
:1064780091804C4B4FF4B468DA78997808FB02F2B3
:106488004FF03C0808FB01285A78474F90441FFA00
:1064980088F8BA466CE03AF815303C24DAB254432E
:1064A80004EB13244C44A4B2042CEEB207D842F2F5
:1064B8005A73984503D904F51C546034A4B2444572
:1064C80011D948F6A8300AF0A7FBC8EB04038342A9
:1064D80009DC364B1A787B1993F83830934302D08D
:1064E8002E4901230B702F4AD378B34232D142F29E
:1064F8006073B4FBF3F203FB12439BB2434523D111
:106508002B4B9B7813F0090F44D12A4B5B7803F08F
:106518008003DBB2002B3DD1274B5B7803F00203ED
:10652800DBB2002B36D1254B1A781BEA020F11D1AA
:106538000199009841EA02021A70FFF7F1FD48B983
:106548000098FFF779FE05E01C4B02991A7801EADA
:1065580002021A70013509F5B469072D1FFA89F985
:1065680099D1039E07370136042E0AF10E0A11D07D
:106578004FF0010B0BFA06FB5FFA8BF301936FEAFE
:106588000B03F2B2DBB24FF00009009202934D46C2
:10659800039680E705B0BDE8F08F00BF650E0020C8
:1065A80031170020BC37002032170020F6140020D5
:1065B800B03100204F3300209A2B002030170020E4
:1065C80073B50C4601EBC001C9B2C90001F5F04131
:1065D8000546042201A810310AF02FFB104B0020B9
:1065E80003EBC402121B521982F8380001AA125C8C
:1065F800312A0AD10121814003EBC402121B52192E
:1066080092F83860314382F8381001300428EDD10F
:1066180001A9312230231BF0E4FDC0B27CBD00BFCC
:106628003217002000B501EBC001C9B2890189B059
:1066380001F5FA418831202268460AF0FEFA202046
:106648006946312230231BF0CCFDC0B209B000BD31
:1066580007B501EBC001C9B201EB011101F5F24127
:10666800D031082268460AF0E8FA08206946312243
:1066780030231BF0B6FDC0B20EBD00002DE9F84373
:10668800002634462BE021462846FFF799FF21468D
:1066980081462846FFF7C6FF214640EA09092846F1
:1066A800FFF7D6FF5FFA89F949EA000010F0FF0FFB
:1066B80005D04046394602220AF0BFFA03E04FF0FF
:1066C800FF33A8F800300135EDB20237072D08F185
:1066D8000208D8D10134E4B20E3E042C07D0054B91
:1066E800C6F5EE47C6EB0308A0370025CBE7BDE8A3
:1066F800F88300BF3217002010B51CF0D9FD4FF405
:1067080080301CF0F5FD1CF00DFF0128044628D14F
:1067180010201CF0EFFC02201CF0E0FC00201CF014
:1067280027FE00201CF038FE4FF480601CF02AFE83
:106738004FF440401CF03AFE4FF480304FF4E01123
:106748001CF0F2FD20461CF0FBFD39201CF0D6FEA3
:106758000028FAD002201CF0F9FD1CF001FE0828E0
:10676800FBD17C2001211CF093FE46F6012001217B
:106778001CF08EFE0C4801211CF096FE0B480121EE
:106788001CF092FE042001211CF08EFE7E201CF0DD
:10679800B5FE38B11CF0DCFE054B04211A7861F314
:1067A80044021A7010BD00BF0340060020080818F4
:1067B800313A002010B50C46014620B110220C4891
:1067C800FAF7BEF804E00A4820211022F9F7E2FDA2
:1067D80034B1084821461022BDE81040FAF7B0B895
:1067E800044820211022BDE81040F9F7D3BD00BFAE
:1067F800F40100200402002010B5FF2B1446029A71
:1068080003D0421802F8013C08E06FF07F439A4237
:1068180004D01314437013128370C27019F09CF8DB
:1068280002E07F201DF0B0F919F082F80028F8D1B5
:10683800ACB10B4890F82010163001F00F0119F098
:106848008BF802E07F201DF09FF919F071F80028FD
:10685800F8D1044B93F8693013F0010FE9D110BD5A
:10686800900C00204C39002010B50A4B002203EB95
:10687800C003013B1046084951184C7813F8011F12
:106888008C4205D10130C0B20C320828F3D1F73060
:1068980010BD00BF5A3C0208B425002070B50D4C4D
:1068A80005460E464FF4007200212046F9F772FDA6
:1068B8002A46314604F50070F9F7C4FC642024F830
:1068C800035C1AF00BFC0023A4F82D33024B64225E
:1068D8001A6070BDB53A00202421002010B5054C7F
:1068E800002120464FF40072F9F754FD0023A4F864
:1068F8002D3310BDB53A0020164B2DE9F0415D8AC5
:1069080007462846FBF70CF91349FBF715FA134B12
:10691800134E1860D723B5FBF3F5EDB28222294652
:106928000446F01901F09CFF2846FBF7FDF80146E4
:106938002046FBF743F80B49FBF74AF9FBF70EFB38
:106948000337BE19C1B281223046BDE8F04101F0DB
:1069580087BF00BFF0280020000057438817002099
:10696800F40100200000204170B54B4D2868FAF76B
:10697800E3FC45A3D3E90023FAF77EFBFAF7CAFF45
:10698800FAF7DAFC42A3D3E90023FAF729FD3EA37C
:10699800D3E90023FAF74EFEFAF7BCFFFAF7CCFC6E
:1069A800FAF7D6FAFAF7B6FF3C4906462860FBF72D
:1069B800B7FA20B13046FBF7D1FAC4B25EE03046F0
:1069C8003649FBF7C1FA50B130463549FBF7A8FA0A
:1069D80028B13046FBF7C2FAC0B2441C4EE030463C
:1069E8002F49FBF7B1FA50B130462E49FBF798FA18
:1069F80028B13046FBF7B2FAC0B2841C3EE03046FC
:106A08002849FBF7A1FA50B130462749FBF788FA25
:106A180028B13046FBF7A2FAC0B2C41C2EE03046BB
:106A28002149FBF791FA50B130462049FBF778FA33
:106A380028B13046FBF792FAC0B2041D1EE030467A
:106A48001A49FBF781FA50B130461949FBF768FA41
:106A580028B13046FBF782FAC0B2441D0EE030463A
:106A68001349FBF771FA48B130461249FBF758FA57
:106A780020B13046FBF772FAC0B2841D0A202146C5
:106A8800BDE870400AF0BEB8736891ED7CFF7F40A6
:106A98000000000080842E418C1700200000104167
:106AA8000000F0410000484200008E420000B84259
:106AB8000000E0420000F2422DE9F04F9DB018F0CE
:106AC800E1FE09201AF0A6FC1AF08CFA4FF4614096
:106AD8001AF0DCFC09201AF059FD0022A3484FF4F3
:106AE80080411CF06CFBA24800211CF035FFA14935
:106AF80004224B78DFF8A0E26FF300034B709E4B43
:106B08009E4C1A705A715A709A70DA701A719A718A
:106B1800DA719B4B033A1A709A4B00201F328EF899
:106B2800000020705A7105900546069006467F20A1
:106B38001DF02AF823780E2B01F2B681DFE813F056
:106B48000F004F009500E0007902DE033004850451
:106B5800EA06DC07EF075808B108D00882098A4E10
:106B68008A48317801F00F01013149014118FFF7D6
:106B780021FE337813F00F0308D1854A92F80123D8
:106B8800012A41F09181834A138024E0012B03D12B
:106B98007F4B93F819330BE0022B04D17C4B93F80D
:106BA8000D33032B05E0032B06D1794B93F80D33F6
:106BB800012B41F079810EE0774901220A7077486C
:106BC8004FF400711CF0FBFA754BC8221A60337839
:106BD8006FF30303BFE333785A1C01F05FB8704BBF
:106BE8001A6822B96D484FF400711CF0E8FADFF812
:106BF80098816C4898F8001001F00F0101314901A3
:106C08004118FFF7D7FD36B198F800305A1C62F3E7
:106C1800030388F800305F4B00221A8098F80010B0
:106C280001F00F02022A03D11A7842F010020AE09A
:106C3800042A03D11A7842F0040204E0052A05D197
:106C48001A7842F040021A7001F02EB9062A04D1CF
:106C58004D4B6FF3030119707EE301F00F01012220
:106C680012FA01F1198001F01FB9474E4E483178E8
:106C780001F00F01013149014118FFF79BFD96F81A
:106C8800008008F00F08B8F1070F27DC18F0010F93
:106C9800464B02D00020588002E04FF0FF31598067
:106CA8004FEA6809062209F1010902FB09394FF088
:106CB800FF32A9F802204046FFF7D6FDFF2806D08C
:106CC8003B4B03EB40005823437401F0EDB800231D
:106CD800A9F8023008F1010801F08AB80021102251
:106CE80013A8F9F757FB0FA800211022F9F752FB58
:106CF80023780133237033786FF3030301F07BB8F3
:106D0800DFF884A09AF8008018F00F0840F03F815F
:106D1800284E337803F04003DBB2F3B926486FF00E
:106D28007F43817A0122009301F00F01FF23FFF7CF
:106D380063FD224B93F8692012F0400F08D093F8B6
:106D48006C3013F0040F03D0337843F040033370F2
:106D58007378142262F3C7037370737813F0F80F13
:106D680030D0174800F12001A7E300BF0018014008
:106D7800002C014012290020E02300209217002057
:106D8800630E00207D320020911700209A3C0208F3
:106D9800B42500204033002054210020000C01407D
:106DA800242100203A3D02081A3E0208FA32002047
:106DB800F40100209B310020900C00204C39002069
:106DC8003A3F0208BC4B1B7803F04003DBB2002BB0
:106DD80000F0D980DFF80483DFF8049398F80030D6
:106DE80013F00C0B30D1B54E6FF07F4396F82B1093
:106DF80006F12100009301F00F0101220523FFF79E
:106E0800FBFC96F84C104FF4860A06F1420001F09C
:106E18000F010122FF23CDF800A0FFF7EDFC96F843
:106E28004110FF2306F1370001F00F015A46CDF853
:106E380000A0FFF7E1FC042389F8003098F800303F
:106E480043F0080301F02EB803F00803DBB2002B6F
:106E580039D099F800A0BAF1000F03D0984800F192
:106E6800400138E0954E6FF07F4B717D06F10B00C5
:106E780001F00F010122FF23CDF800B0FFF7BCFCA1
:106E880096F82B1006F1210001F00F0101220723CB
:106E9800CDF800B0FFF7B0FC96F836104FF4860333
:106EA800009306F12C00FF2301F00F015246FFF773
:106EB800A3FC98F800306AF3C303DBB243F0040381
:106EC80088F800305AE099F800C0BCF1000F08D0EB
:106ED8007B4800F16001FFF76DFC99F80020303223
:106EE80008E2764E6FF07F40717DFF23009001F03D
:106EF8000F0106F10B000122CDF80CC0FFF77CFC56
:106F08009AF80030DFF8C4B103F0100A5FFA8AFA81
:106F1800DDF80CC0BAF1000F0CD098F800206CF323
:106F2800820288F800205A1C62F303038BF80030B1
:106F380000F0BABF96F82B106FF07F42009206F16E
:106F4800210001F00F0101220C23FFF755FC96F8F0
:106F580036104FF4860300935246FF2306F12C00A7
:106F680001F00F01FFF748FC9BF8003083F0100296
:106F7800C2F3001262F304138BF80030042389F87B
:106F8800003000F091BF4E4800F1800195E2B8F161
:106F9800010F3CD14A4800F1A001FFF70BFC002E7D
:106FA80000F082879AF80030444E5A1C62F30303BB
:106FB8008AF8003096F82B106FF07F4906F121000F
:106FC80042460F2301F00F01CDF80090FFF714FCA3
:106FD80096F82B1006F1210042460E2301F00F010E
:106FE800CDF80090FFF708FC96F82B1006F1210069
:106FF800424601F00F010F23CDF80090FFF7FCFB8C
:107008003048802142461CF0DAF800F04DBF2C4889
:1070180000F1C001FFF7CEFB002E00F045872A4B98
:1070280096221A609AF800306FF303038AF800304A
:1070380092E1264E317811F00F0A16D1244800F15A
:107048002001FFF7B7FB204B1B68002B40F02C8773
:1070580013A8F9F7EFFB40221346014613A801F0E5
:1070680023FA3378012200F019BEBAF1010F39D1A1
:1070780012486FF07F4390F82010002200931630DA
:1070880001F00F01FF23FFF7B7FB01F077FA0028A3
:1070980000F00A873378022262F3030333700D4B42
:1070A8001A7842F080021A700B4B5A7842F00202AA
:1070B8005A7000F0F9BE00BF9B310020900C0020F0
:1070C8003A3F0208001001402421002091170020B7
:1070D8001A400208A03100205E340020D040002071
:1070E8005742002001F00F0101F10E0303F00F03D6
:1070F800012B44D89B4849014118FFF75BFB9A488C
:107108006FF07F4390F8201000221630009301F0B2
:107118000F01FF23FFF770FB19F0ACFD337803F084
:107128000F03022B13D116F03DF9002800F0BC869E
:107138008E4B1A7842F040026FF304121A705A7894
:107148006FF345125A703378032200F0A7BD16F08A
:1071580013F978B116F0B2F916F06AF8844B0020EA
:107168001A7858816FF3C7121A703378042262F3C1
:10717800030333707F4B1A786FF3000263E5BAF1AB
:10718800040F4DD1DFF8DC914901DFF81082494442
:107198004846FFF70FFB98F80010774B01F0040200
:1071A800D2B27AB941F004016F4883F800A088F898
:1071B800001090F836104FF4860300932C3001F03D
:1071C8000F01EEE293F800A0BAF1000F40F06C86D0
:1071D80065486FF07F45417D01220B3001F00F01BA
:1071E800FF230095FFF708FB64480122817AFF23FB
:1071F80001F00F010095FFF7FFFA98F8003005221B
:107208006AF3820388F800303378484662F3030350
:10721800337009F1A001FFF7CDFA554600F044BEDE
:10722800DFF84481FF2398F8201000226FF07F498F
:1072380008F1160001F00F01CDF80090FFF7DCFA15
:107248002BB2072B18D1337808F121006FF3030311
:107258003370237801220133237098F82B100E2302
:1072680001F00F01CDF80090FFF7C6FA44488021DD
:1072780000221BF0A4FF0025424E96F86B3013F055
:10728800040F00F0118698F857106FF07F43002222
:1072980000933D48FF2301F00F01FFF7ADFA96F880
:1072A8006B303A4A03F00F03012B137003D1002D02
:1072B80008BF01250CE0022B04D12BB2012B08BF1B
:1072C800032505E0032B03D12BB2032B08BF0725A9
:1072D800ABB213F0010F02D02D4A3121517713F0D0
:1072E800020F02D02A4A3221917713F0040F00F0DE
:1072F800DB853322264BDA7700F0D6BD1948254EB8
:1073080000F1C001FFF756FA96F80090DFF85C80AC
:1073180019F00F090CD115F0A5FE98F8003069F3A3
:10732800000388F8003033785A1C62F30303337083
:1073380015F02AFF98F8003013F0010F00F0B4851B
:107348000022154880211BF03AFF0A4B00225A7090
:10735800337862F30303337023780133237000F02A
:10736800A3BD00BF1A400208900C00205E34002024
:10737800A0310020D6330020574200200100002011
:10738800001001404C390020DD0C00209A3100200B
:10739800F40100209117002000180140D04000207F
:1073A8008648874E00F1E001FFF704FA0FA8F9F7C5
:1073B80041FA0FA902468348F9F7C2FA0021824828
:1073C800B18090F8C5106FF07F4300220093BB3066
:1073D800FF2301F00F01FFF70FFA7C4A92F86B10B8
:1073E80092F86C30327843EA012312F0010FB3802F
:1073F80010D0A3F1EB0292B20A2A04D9A3F5E673DE
:107408009BB2282B02D8F3880133F38033786FF3CB
:10741800000333707378002B40F04685684AD288A1
:107428007AB16B4A1BA8117863F3030111702278B3
:107438008DF86F300132227028228DF86C201BF0F5
:10744800DDFE0022F28000F02FBD624EDFF8ACA115
:10745800337803F004085FFA88F8B8F1000F15D103
:1074680009A841461522F8F795FF5B4BCAF800803A
:107478001B684546CDF827303368474643F0040378
:107488003360564BA3F8368300F00EBD03F080033B
:10749800DBB2002B67D1DAF80010002940F0048530
:1074A8004F48FFF787F94F484FF480511BF07DFE96
:1074B800012806D04A4800F1A001FFF77BF900F047
:1074C800F3BC4649B1F83623002A43D0093146486F
:1074D800013AF9F735FA444B03F1100113F8012B7F
:1074E8000D2A01D00A2A02D1202203F8012C8B424E
:1074F800F4D13E4B4FF03C0808FB073808F11E0852
:107508004046F9F797F9414602463948F9F7C2F972
:10751800D8B9022F03D1336843F0100304E0032FD6
:1075280003D1336843F040033360327853005BB2D1
:1075380003EAC263DB173268DBB263F3C712326057
:107548001BB1FFF7CBF900F0AFBC0137FFB2042F36
:1075580008BF0227254B3C2606FB07363046F9F7BD
:1075680069F9314626E0DAF80080B8F1000F40F0FA
:107578009B84737803F02002D2B2002A40D11D4BBD
:1075880009A81A889B781C498DF82630ADF8242064
:10759800F8F75AFF114B5B7A302B07D1FFF79EF9AA
:1075A800336843F40053336000F07EBC09A8F9F750
:1075B80041F909A9FFF772F900F076BC1A400208F0
:1075C800D633002008020020900C00204C390020FF
:1075D8009117002028210020332B0308AC3A002003
:1075E8001A41020800080140040200200C00002093
:1075F800B53A0020382B03083C2B0308242100202F
:1076080003F04003DBB2002B40F08980B14800F161
:107618006001FFF7CFF8B048F9F70CF98046AE499A
:10762800AE484246F9F736F9002873D1AC4B4344CB
:107638005B7A302B6ED1FFF751F93368DFF8D092BF
:1076480043F48043336099F82B106FF07F43009325
:1076580009F12100082301F00F010122FFF7CCF8FE
:107668006423CAF800307F201CF08EFADAF8003064
:10767800002BF8D1984699F88E10D633994E89F890
:1076880086304B3B6FF07F4A89F88730964801F087
:107698000F0142467433CDF800A0FFF7ADF896F815
:1076A800B91106F5D670033001F00F014246FF23E9
:1076B800CDF800A0FFF7A0F896F8C41106F5DD7024
:1076C80001F00F014246FF23CDF800A0FFF794F820
:1076D80096F8CF1106F5E270013001F00F0142462D
:1076E800FF23CDF800A0FFF787F896F8DA1106F522
:1076F800E87001F00F014246FF23CDF800A0FFF724
:107708007BF899F899107948CDF800A001F00F019D
:10771800424646E07648F9F78DF875494AE796F803
:1077280002B0DFF8EC910BF0020B5FFA8BFBBBF1B8
:10773800000F3AD199F82010FF236FF07F4809F124
:10774800160001F00F015A46CDF80080FFF754F8F3
:10775800684B93F86B3003F00803DBB2002B00F0A2
:10776800A38399F82B10012209F1210001F00F01E0
:107778000323CDF80080FFF73FF83368554843F4FA
:10778800003300F180013360FFF714F855485A467A
:1077980090F8E51100F5EC70CDF80080033001F0A9
:1077A8000F01FF23FFF728F87EE3CAF8008099F855
:1077B80020106FF07F4300934246FF2309F1160023
:1077C80001F00F01FFF718F82AB241F211139A429B
:1077D8001DD1434B5B7A302B13D1FFF77FF8336809
:1077E800454668F3514368F38E3368F34D3333608D
:1077F800414B1A7868F303021A7023780133237017
:1078080052E33E48F9F716F83C49FFF747F8394E76
:1078180096F86B3013F0040F00F0468325B938480A
:1078280020211022F8F7B6FD7F201CF0ADF999F859
:1078380057106FF07F43002200933248FF2301F076
:107848000F01FEF7D9FF96F86B202F4B02F00F02BD
:107858000D2A1A7005D125B92C4A412191754FF48A
:1078680080551A78062A08D12AB2B2F5805F04D169
:10787800264A3621D1754FF488551A78082A08D136
:107888002AB2B2F5885F04D1204A3821117641F234
:1078980010151B780B2B09D12AB241F210139A420A
:1078A80004D11A4B2A225A7641F211150D486FF06D
:1078B8007F4390F8F0110022009300F5F370FF2346
:1078C80001F00F01FEF798FF96F86B3013F0010FE7
:1078D800AAD0E9E21A4102081A010020B53A0020AC
:1078E800AC3A002001000020140D00201F0D0020DC
:1078F800FC0000204C39002091170020380100209E
:1079080004020020DD0C00209A310020F401002040
:10791800900C0020A34B1A7842B300221A700F2053
:10792800FAF792FB06460A20FAF78EFB9E4B9F4910
:1079380058824A7812F0010F18D06436301A5883EA
:107948009B4B1A78642A01D19B321A701B78984E87
:10795800FF2B0BD00A21B3FBF1F1964B193119809B
:1079680095481BF0F9FF337801333370DFF86482F0
:1079780098F8003013F00F0612D18E4B19228B485D
:107988001A804378192143F0010343708A481BF099
:10799800E3FF8A4800F12001FEF70CFF04967CE221
:1079A800012E68D1804B5A8BA2F1690189B2112945
:1079B80008D8049911F0010F04D141F00101C9B2AE
:1079C80004910592049A12F0020F0DD15B8A7C4A49
:1079D8001380A3F5C263023B9BB2D72B04D804984B
:1079E80040F00203DBB204931B20FEF785FF0599E4
:1079F800744B0AB2632A05DD642192FBF1F230323E
:107A08001A7401E0092A0CDD059A11B2642291FB6F
:107A1800F2F002FB10120A2012B292FBF0F230329E
:107A28005A74059802B2642092FBF0F100FB112110
:107A38000A2209B291FBF2F002FB101230329A745A
:107A48005B4B1B78FF2B08D158495B484B786FF389
:107A580000034B7000211BF07FFF049A032A40F0BB
:107A680023825248002143786FF300034370524841
:107A78001BF072FF11E2022E03D1534BC8221A6089
:107A88000BE2032E16D1504B1B68002B40F00C82E2
:107A98004A4800F14001FEF78DFE1B20FEF72CFF3F
:107AA800414B5B8AA3F51E630F3B9BB2542B00F23C
:107AB800FB81F2E1042E0CD13B4B988A0EF0F4FDC9
:107AC800002840F0F1813D4800F16001FEF772FEA8
:107AD800E3E1052E07D1344B988A0EF0E5FD032823
:107AE80040F0E281D9E1062E40F0D78122786FF389
:107AF800030301322270D5E1344800F12001FEF77A
:107B080059FE334B1B78002B00F0CE8123780133CC
:107B18002370304B1A786FF30302FFF794B82D4E99
:107B2800DFF8A480337813F00F021AD12A4800F145
:107B38002001FEF73FFE2948F8F77CFE2749024658
:107B48002748F8F77FFB2548F8F774FE254BA3F87C
:107B5800160233785A1C62F30303337019F040FDA0
:107B680091E0012A16D1D8F80030002B40F09C8112
:107B780019F062FD012840F097811B48F8F75AFE7A
:107B8800194902461948F8F785FE002840F08C810B
:107B980011486FE0D8F80020002A40F085810B21B9
:107BA8007BE000BF660E0020F0280020122900208C
:107BB800A01700208C0C0020002C0140DA4102089C
:107BC80094170020F4010020242100205A420208C2
:107BD80090170020911700209A4202087401002093
:107BE800882F0020503E002092010020513E0020A6
:107BF800874E337813F00F080CD186484146FEF7BC
:107C0800D9FD33785A1C62F303033370824BA3F80F
:107C1800028049E1B8F1010F18D1804804211BF016
:107C2800C4FA002800F040817A4800F12001FEF7EC
:107C3800C1FD33784FF0FF315A1C62F303033370F0
:107C4800774B64221A60744B59802DE1B8F1020F0A
:107C5800DFF8CC811BD1D8F80030002B40F024810C
:107C68006E4804211BF0A1FA002840F01D816A4BE0
:107C78005880684800F14001FEF79CFD33785A1C93
:107C880062F3030333706423C8F800300CE1D8F8BA
:107C98000020002A40F008810C21217062F30303C0
:107CA800A9E0604910234FF40052CB700D3B8B7054
:107CB8000A805D481BF02AFA0A2200215B48F8F77F
:107CC80069FB80201BF086F9237801332370504B21
:107CD8001A786FF303021A70514BC8221A60E3E056
:107CE8005348DFF848A100F12001FEF763FD9AF838
:107CF8000030002B00F0D8804E48DAF80020444EBF
:107D08000260BAF8042082809AF8062082713178DD
:107D180011F00F0159D1DFF80881D8F800100029B7
:107D280040F0C2809AF80410A2F5A6524FF0640BF6
:107D3800103A0BFB01229AF805004FF00A0909FBDB
:107D480000200393F9F7ECFE3B49F9F7F5FF0246EB
:107D58009AF80200039BA0F5A65010380BFB030B02
:107D68009AF80100354B09FB00B018600392F9F747
:107D7800D7FE039A01461046F9F722FE304B1860E9
:107D8800F9F7DAFA1EA3D3E9002382468B46F9F7FE
:107D9800ADFD002800F08880504659461AA3D3E963
:107DA8000023F9F799FD00287ED0FEF7DDFD337832
:107DB80048465A1C62F303033370C823C8F80030DE
:107DC80008F02AFFC0B207906EE001296CD10D308F
:107DD8000799832200F044FD114BD3F80080B8F1D5
:107DE800000F61D140461BF0F5F82378013323706A
:107DF800337868F30303337056E000BFAFF30080B5
:107E0800736891ED7CFF7F400AD7A3703D008040E6
:107E180091170020FA420208FA320020000C0140B3
:107E2800242100200E29002000100140A81700205E
:107E38005A4302080402002000007A44A4170020D4
:107E48008C1700208448854E00F12001FEF7B2FC13
:107E5800F37913F0010F27D0DFF8488298F80090E3
:107E680019F00F0920D17E4B0A2259781878103959
:107E780002FB0011B1701979D878103902FB001192
:107E88007170D9799B79103902FB0312327016F0A0
:107E980009FDF37969F30003F37198F800305A1C6F
:107EA80062F3030388F80030DFF8FC9199F800606A
:107EB80016F001063EF43BAE6A4B01221A7018F028
:107EC80043FB2378092B01D00D2B28D101206649CB
:107ED80011F086FB654B664A5B7803F01F03D35CA1
:107EE800644A522B137002D1634B01221A70634B00
:107EF800634A03F1200153F8040B8B4242F8040B48
:107F0800F9D1002117A811F095FB17A80D2119F038
:107F180003FB5C4B1A78013202F003021A7099F8DD
:107F2800006006F00206F6B2002E00F08B800EF01C
:107F380069FE12F053FE06980322431C93FBF2F2EB
:107F480002EB42029B1ADBB20693002B79D1DFF8D1
:107F5800488198F84960C246002E4DD0022E03D1C0
:107F680098F80130312B49D023780E2B13D146488D
:107F780046490522F8F78EFC8246002840D1B21FF8
:107F880037484349F8F7DCFC344B5646DA7942F077
:107F98000102DA7135E00D2B03D13E483A49072238
:107FA80027E0032B22D13C4B002713F8012F2C2A62
:107FB80003D00137FFB2B742F7D113A832493A4686
:107FC800F8F7BEFC7B1C07E00AEB03025278303A54
:107FD800D2B2092A03D80133DBB2B342F4D30AEB95
:107FE8000701FA430FA80231D21802E0264909A86E
:107FF800721EF8F7A5FC03E0069E02E0012600E0E9
:1080080000261E4B204A03F1100153F8040B8B4243
:1080180042F8040BF9D1214B214A03F1100153F81E
:10802800040B8B4242F8040BF9D1402388F8113035
:108038001C3B88F82230023B88F84B3018F0F4FFDC
:1080480000E0002699F8003003F0F5036FF3000311
:1080580089F80030FEF76BBD9A430208BC37002050
:1080680096170020660E0020ED3D0020EC3D002014
:10807800207902081332002090170020F401002014
:1080880056320020B63100205B3A00203F2B03080F
:10809800603A0020A81700205A3A00200402002065
:1080A8006C3A002091170020343A0020AFF300808A
:1080B80010B5044640181146F8F75EFB2046F8F75D
:1080C800B9FBC0B210BD42540131C8B270470000BC
:1080D80010B50C4B0C4A1B780C460E2101FB0323F0
:1080E800997A31B101390523594301F56F5189B2A4
:1080F80001E04FF46F510019042208F09EFD201D85
:10810800C0B210BD71400020A012002010B5054B70
:108118000C46197800190131042200F0A1FB201D3A
:10812800C0B210BD7140002000F5224000F5CF70AC
:1081380008B5013008F070FD10F0FF0F14BF0020E3
:10814800012008BD10B50A4600210446FFF7B0FF1C
:1081580001462046FFF7DAFF114A01462046FFF79D
:10816800A7FF232201462046FFF7ADFF0146204620
:10817800FFF7AEFF5B2201462046FFF7A4FF23224C
:1081880001462046FFF79FFF01462046FFF7A0FF64
:108198007C2201462046BDE81040FFF794BF00BF8F
:1081A800452B030810B55D220446FFF78CFF0D220E
:1081B80001462046FFF787FF0023235410BD38B53A
:1081C8001D460C4640182C1911461A4600F048FB6B
:1081D800E0B238BD2DE9F04118490446FFF7B2FF77
:1081E800174F0E263B78174D73430146EA5A20462F
:1081F8000423FFF7E4FF202201462046FFF763FF30
:108208003B78014606FB035320469A7A0223FFF780
:10821800D6FF202201462046FFF755FF3B7801464E
:1082280006FB035520466A7A0323FFF7C8FF014679
:108238002046BDE8F041FFF7B5BF00BF482B030853
:1082480071400020A01200202DE9F047264E0E2292
:108258003378264F534337F90380FA1824494FF4EB
:108268007A73044698FBF3F8157AFFF76BFF4E22F2
:1082780001462046FFF727FF1E4B1C2202FB05354F
:108288005FFA88F8B8F1030F01460CBF05F1120236
:1082980005F108022046FFF70BFFA146804600259E
:1082A80019E019F8013BA32B07D133780E2202FB02
:1082B8000373204629465A7A08E0242B09D13378DB
:1082C8000E2202FB03739A7A204629460223FFF7FF
:1082D80076FF0135EDB24545E3D120462946BDE894
:1082E800F047FFF75FBF00BF71400020A0120020D9
:1082F800522B030840790208074B187800F0040055
:10830800C0B240B11A686FF382021A60034B0022B0
:108318001A70034B18787047B0310020CC17002032
:10832800B4170020054B00211970054B05481A6841
:1083380061F382021A601222F8F72CB8CC170020D9
:10834800B0310020B417002038B5084C084922780D
:108358000546F7F777FF23780021E954054B1A689B
:1083680061F382021A60207838BD00BFCC17002064
:10837800B4170020B0310020064A07491378112BA2
:10838800C85401D801331370044A136843F0040336
:1083980013607047CC170020B4170020B0310020BC
:1083A800054B1B7813F0010F05D1044B181810F872
:1083B800010CFFF7E1BF7047CD170020DA43020830
:1083C8002DE9F041334C002314F8101094F82A20BA
:1083D80001F00F0161F3030284F82A2004EB400046
:1083E80084F8293084F828304378DFF8B88063F3BC
:1083F8000712638C4FF4D277E38498F800302A266A
:108408007B4306FB0133244D2448E95A84F82A208B
:108418001BF0A0FA98F8003094F82A207B4302F069
:108428000F0206FB0233EB1859881C48013989B240
:108438001BF094FA01210A4618481BF05BFA012147
:1084480016481BF048FA98F8003094F82A207B4325
:10845800120906FB02331248E95A1BF07BFA98F816
:10846800002094F82A3057431B0906FB0376AD1900
:1084780069880B48013989B21BF06EFA01210A4656
:1084880007481BF037FA06480121BDE8F0411BF008
:1084980022BA00BFCE170020E643020800080040B9
:1084A80000340140FA17002030B5164C94F82B50D0
:1084B800A38445F00105002384F82B50628484F8D6
:1084C800211084F8203019E0C55CA5F13002D2B241
:1084D800092A08D9A5F14102D2B2052A9ABFA5F105
:1084E8003702D2B22A46084D013305EB420292F810
:1084F800495392F84823257062700234DAB28A42EE
:10850800E2D330BDCE170020E6430208124B10B567
:108518009A8C0024DA8483F8294083F8284022467C
:1085280001210E481BF0E6F964210C481BF012FAF1
:1085380032210A481BF012FA0121224608481BF092
:10854800D9F9642106481BF005FA05483221BDE82F
:1085580010401BF001BA00BFCE17002000080040F1
:108568000034014010B500212C220348F7F712FF10
:10857800BDE81040FFF7CABFCE17002070B5214CE8
:108588002378042B39D8DFE803F0030D152A3000CF
:108598001D4B012093F82B3013F0010F30D02070C1
:1085A800013870BD184B93F82000FFF709FF02232C
:1085B800237022E0144DEE8CFEB9FFF7A7FF95F863
:1085C800203095F821200133DBB29A4285F820301B
:1085D80001D8042300E003232370304670BD0A4B02
:1085E800D88C50B90123237070BD074BDD8C35B989
:1085F800FFF7B8FF2570012070BD002070BD002076
:1086080070BD00BFFB170020CE170020044B0022CE
:108618005A701A709A7842F001029A70704700BF37
:1086280010190020202102480A46F7F7B3BE00BF00
:10863800F401002038B5044608460D46F8F7FAF864
:1086480098B10319202B094BC8BFC4F120001C198D
:10865800002308E014F8012BE02A14BFEA5C20226A
:1086680004F8012C01338342F4DB38BDF401002007
:108678000D4B46F635321B689B6893420FD043F684
:10868800F82293420BD0122B09D0B3F5E97F08D01A
:1086980046F6D9301B1A584240EB030070470120B8
:1086A80070470120704700BF34180020F0B51F46FE
:1086B80087B006460C46084600211546F7F76AFEBD
:1086C800244B07B19F80B3F9041005A801EB86017C
:1086D800042208F0B2FA002605AB9B5D013BDBB231
:1086E800B92B34D81D2B4FEA031208D8D31803F539
:1086F800164168465231112208F09FFA0BE01649DC
:10870800D3185B186A4603F11007186859680833CC
:10871800BB4203C2F9D12046F8F78CF8C7B26846C5
:10872800F8F788F83818A84203D8E0196946F8F726
:1087380023F86846F8F77EF87B1C1B18AB4203D277
:10874800E0190649F7F780FE0136042EC4D107B0B8
:10875800F0BD00BF10190020710D03086A2B030833
:1087680010B500216C220446F7F714FE0123A3700C
:1087780010BD002343700370837843F001038370B6
:10878800704700002DE9F0419378804613F0010FFF
:108798000D4614463AD06FF30003937018F01CFC92
:1087A8006378002B32D123780BB90A336370A3782E
:1087B800174F6FF30003A37018F00EFC217807EB36
:1087C80008066118073130462A46F8F7B9F83046E6
:1087D800F8F730F8C6B2AE420DD80AD2002323709B
:1087E80006EB08000A33637038182021AA1BF7F734
:1087F800D1FDAE420AD12278A3181B7A1BB10132EF
:108808002270BDE8F08123700A236370BDE8F0810F
:10881800F4010020054B1A780AB100221A701B785F
:1088280046F69B2202FB0311FFF704BF171800202E
:10883800F8B505460C460818002108F0E3F9013C94
:10884800E4B26719384608F0E7F9C6B2202E03D813
:108858003846002108F0D6F90CB1202EEFD9F8BD22
:1088680002F00F03032B22F07F0230B5D2B20CD9ED
:108878004FF47A7491FBF4F42025E4B2057002B148
:1088880014B13034047000220130B1F57A7F05DB71
:108898004FF47A7491FBF4F504FB1511022B0BD9F4
:1088A800642491FBF4F42025E4B2057002B114B1FC
:1088B8003034047000220130632904DD642491FB04
:1088C800F4F504FB1511012B0AD90A2391FBF3F3E4
:1088D8002024DBB2047002B10BB1303303700130D5
:1088E800092904DD0A2391FBF3F203FB121130314D
:1088F800017030BD13B5104B01461B689A899C7BEB
:1089080012F0100214BF0220012034B10B4C9B7CE2
:108918002478634303FB001109B23AB10DF1060054
:10892800022208F08AF9BDF8060002E0084608F0BD
:1089380073F900B21CBD00BF34180020C118002014
:1089480010B50F4B1B689A899C7B12F0100214BF5C
:108958000221012134B10B4C9B7C2478634303FB37
:10896800010000B22AB108490222BDE8104008F00F
:108978005EB9054B1968BDE8104008F043B900BF5F
:1089880034180020C1180020D81800203038C0B290
:10899800092894BFFF20002070470000024B1A7876
:1089A8006FF300021A7070470119002070B58F4CE0
:1089B800FFF7F4FF2678254606F0F006202E72D140
:1089C80008F09EFC00286ED1894B1B7833B92378B8
:1089D800C3F30312013262F307135EE0854B1B7881
:1089E80003F08003DBB2002B59D08348F7F722FF4E
:1089F800C5B2824CBDB1204681493246F7F7A0FF87
:108A08000A2D0BD82A4620467B49F7F799FF6019AB
:108A18003146C5F10A02F7F7BDFC04E02046764965
:108A28000A22F7F78DFF774B1B7813F0010F01D05F
:108A3800472300E02023E372704C042204F10C0069
:108A4800A521F7F7A7FC704B1A7852B1FF23012A2A
:108A5800237306D9022A637303D0032AA37318BFAA
:108A6800E3736A4C257815F0600502D194F8A330B9
:108A780013B96748674902E0654804F1A301062273
:108A8800F7F75EFF644B1B78452B40F09D81002D66
:108A980040F09A81237843F08003237070BD5748D3
:108AA8005E49324685E12C7804F0F004102C3FD161
:108AB80008F026FC00283BD1202259494F48F7F7F7
:108AC8003FFF4E4856492246F7F73AFF554B1B7869
:108AD80013F0010F06D05448F7F7ACFE524902468E
:108AE800524805E05248F7F7A5FE514902464F485B
:108AF800F7F726FF3E4B1B781BB94E484E4910220C
:108B080057E14C484D491022F7F71AFF394B1B78AB
:108B180003F08003DBB22BB14348F7F78BFE024624
:108B280047484FE04248F7F785FE0246444842E08E
:108B38002B7803F0F003302B46D108F0E1FB002836
:108B480042D12E4C20223F492046F7F7F9FEA521B5
:108B5800052204F10B00F7F71DFC3B4B1B78042B97
:108B680002D9FF23E37300E002D1FF23A37301E0DE
:108B7800032B02D1FF23637301E0022B02D1FF23F1
:108B8800237300E00BB1FF23E372304B5B7813F0E3
:108B9800600F05D03F23E37223736373A373E373FA
:108BA8002B4B1B7803F02003DBB233B12048F7F7D7
:108BB80041FE024627481E49FBE01B48F7F73AFEEC
:108BC800024624481849F4E02B7813F0F00347D103
:108BD800202221490948F7F7B3FE204B0748198896
:108BE8008322BDE87040FFF73BBE00BF011900209B
:108BF80054210020282100202C210020F4010020ED
:108C08007ED3020868400020212200205C21002039
:108C18000E02002067AB0208FC1700203CD30208B4
:108C2800600903085E340020AA0A03080102002034
:108C3800CB0A0308040200202D0F0308810903084A
:108C4800110200200CAC0208DF23002018290020A4
:108C5800B03100200F020020A9AB02081218002032
:108C6800602B1ED108F04CFBD8B95849202258482F
:108C7800F7F766FE5748F7F7DDFD564902465648AE
:108C8800F7F75EFE5548F7F7D5FD544902465448B4
:108C9800F7F756FE5348F7F7CDFD524902465248BA
:108CA80087E02B7803F0F003102B06D108F028FB9F
:108CB80018B147484D4920227BE02B7803F0F00497
:108CC800402C02D0502C78D108E041484849202255
:108CD800F7F736FE474B1B784BB94CE03C48464902
:108CE8002022F7F72DFE454B1B783BB943E0444B58
:108CF8005A7882B11B78022B14D105E0414B1B78BE
:108D080013F0010F07D00DE03F48F7F793FD3E49F8
:108D180002463E4835E03E48F7F78CFD3C4902469E
:108D28003A482EE03B48F7F785FD3A49024637486E
:108D3800F7F706FE402C0BBF314B374B5B78DB78DF
:108D4800022B0AD0042B0FD0012B1CD13348F7F784
:108D580071FD3249024632481BE03248F7F76AFD96
:108D6800304902462E4814E02F48F7F763FD2E4994
:108D780002462B480DE02D48F7F75CFD2B490246CB
:108D88002248F7F7DDFD2A48F7F754FD284902463F
:108D98002348F7F7D5FD274B1B78ABB920210722CD
:108DA8001F48F7F7F7FA2148F7F744FD1F4902462D
:108DB8001B48BDE87040F7F7C3BD1F4A6FF30713A0
:108DC80013701E4B00221A6070BD00BF88AB0208EA
:108DD800F401002088A40208F801002092A40208E7
:108DE800080200208DA402080F020020EBAB020845
:108DF800A209030898310020C30903085421002060
:108E0800AA2D002068400020680A0308FD01002000
:108E18000D0B0308AA0A0308FC200020E409030834
:108E28000D020020050A0308260A0308EC0A0308B5
:108E3800470A0308902B002001190020341800204D
:108E4800204B70B5F022204D1A702B7813F0010FCB
:108E58000BD01E4C207810F0010006D11C49FFF7FA
:108E6800D9FC237843F0010323701A4E3378532B2F
:108E78000ED1164C237813F0010F07D000201649A5
:108E8800FFF7C8FC23786FF300032370FFF786FD14
:108E98003378232B14D10D4B1B7813F0010F0FD10E
:108EA800FFF77CFD2B780D4A43F006032B701378EF
:108EB800013BDBB213700A4A52F82320094B1A60AF
:108EC80070BD00BF0D1900200119002039180020BD
:108ED80031FF0208FC17002010FF0208EF180020DD
:108EE800F0180020341800202DE9F0415C4BF022E6
:108EF8005C4D1A702A7802F01003DBB2002B2DD1DA
:108F0800594963F347120B601C462A70574A9A5C0A
:108F18002D2A01D00134E4B20133082BF6D1544E86
:108F28003A213046F7F7B4FA38B1801BC0B20130A5
:108F3800301821460222FFF793FC4E4B1B78452B35
:108F480040F08B8000242046013411F09FFE082C4D
:108F5800F9D12B7843F010032B7038E0464C237876
:108F680013F0010F17D1404E4448FFF7F9FB404F6B
:108F78003168384601310222FFF772FC2D23BB709D
:108F8800307846F661533E496522FFF78FFB237818
:108F980043F00103237003200D21384AFFF7F2FB49
:108FA8002D78304E15F0E00541D110203549FFF7F6
:108FB80031FC304B1B78442B0DD12B4A13680133FD
:108FC8002A4903F00703C95C2D29F8D01360BDE8CE
:108FD800F041FFF7E3BC532B0DD132784E3B63F3DE
:108FE80047123270204A28491268062000FB0212F4
:108FF8005380BDE8F081232B2FD11B4B1D603378A4
:1090080003F0EF0365F347133370FFF7C7FC2378CA
:109018001E4A43F0060323701378013BDBB213703A
:109028001B4A52F823201B4B1A60BDE8F081104CF4
:1090380010201949FFF7EEFB04F110002821F7F77B
:1090480027FA50B1001B3178C0B201302018490905
:109058008022BDE8F041FFF703BCBDE8F08100BF06
:109068000D19002039180020D8180020DD32002002
:10907800F4010020FC17002001190020101900201D
:1090880017190020ADFE0208FA320020EF18002060
:10909800F018002034180020CEFE0208454B2DE9B8
:1090A800F041F022444E1A703378444D43F00103E6
:1090B80033702B68424C9B7C022B06D1414B1B78AA
:1090C80003F04003DBB23BB10FE0012B0DD13E4B67
:1090D8001B7813F0010F08D108F084FA23680020E8
:1090E8006FF355532360394944E0A378344F03F0B4
:1090F8002003DBB2C3B908F075FAF87800F0200055
:10910800C0B288B92968324B897C1A7861F30102A8
:109118001A703B682D4943F400133B60FFF77AFB54
:109128002C4B802283F843200CF06EFE804678B1E9
:109138002B689B7C012B08D1234B5B7803F0100331
:10914800DBB213B10020244914E00020234911E0C8
:109158000CF08AFE074610B1404621490AE00CF09F
:10916800CBFE10B138461F4904E01A4B93F8433040
:1091780013B91D49FFF74EFB1C4B1B78232B16D147
:10918800FFF70CFC337843F00603337008F02AFA33
:1091980023686FF3555323600BF0A2FD144A13782C
:1091A800013BDBB21370134A52F823302B60BDE841
:1091B800F08100BF0D19002001190020341800208B
:1091C800B0310020282100205E34002052FF020820
:1091D80063340020A91C002094FF020873FF0208D2
:1091E800D6FF0208B5FF0208F7FF0208FC170020A7
:1091F800EF180020F01800202DE9F3416E4B6F4D59
:10920800F0221A702B686E4C9B7C1BB9637843F074
:10921800100302E0637843F008036A4E6370337802
:1092280043F001033370238823F47E6323F01E0385
:10923800DB04DB0CB3F5805F08D0634B1B7883B18C
:109248005F4B5B7803F00803DBB253B1637800200F
:109258006FF341035D496370FFF7DCFAF8F730FFFD
:1092680084E06378564F03F00203DBB2FBB9BB78A6
:10927800EBB9574B93F8008018F0010817D1F8F7AD
:109288001FFF7B7843F002037B702B68B3F9103023
:10929800022B7B780CBF43F0040368F382030021A0
:1092A8007B70082001220B460091F9F725FAA37874
:1092B800434A032B28D003D8012B0BD00DD806E046
:1092C800052B2DD0517825D3FF2B32D12BE0002050
:1092D8003E4949E000203F4946E03F48F7F7AAFAEF
:1092E800DFF82C81C7B23C4908F110003A46F7F77D
:1092F80027FB0F2F3AD807F1100040442021C7F16F
:109308001002F7F747F831E0344B187800282DD1D0
:10931800334929E06FF3410151700020314923E0BE
:109328000020314920E06FF34101517000202F499E
:109338001AE0053BDBB26FF34101022B517002D1F9
:1093480000202B4910E0012B02D1002029490BE015
:10935800032B02D10020284906E0052B02D100206A
:10936800264901E026490020FFF754FA637803F004
:109378000203DBB20BB9F8F7A3FE224B1B78232BB1
:1093880018D1FFF70BFB3378002243F00603337044
:109398006378A27003F0E50362F382036370F8F761
:1093A8008FFE194A1378013BDBB21370174A52F843
:1093B80023302B60BDE8FC810D19002034180020F3
:1093C8006840002001190020AA2D002052FF020841
:1093D8006E40002095FB0208774000206C4000207A
:1093E800B6FB02085A0003083AFC02089DFC020872
:1093F800D7FB0208F8FB020819FC02085BFC02080C
:109408007CFC0208FC170020EF180020F018002050
:10941800F40100207B4B2DE9F341F0227A4E1A70BB
:1094280033787A4D43F0010333702B68784C9B7C7A
:10943800022B11D1774B1B7803F04003DBB293B1B9
:10944800754B1B7803F02003DBB2BBB1A37803F0A4
:109458004003DBB23BB111E0012B0FD16F4B1B78FE
:1094680013F0010F0AD1F8F72BFE2368002023F42C
:1094780080036FF3D753236069498FE0A778DFF83B
:10948800908107F04003DFB2002F34D1F8F718FEBF
:109498002968644B897C1A78384661F301021A708E
:1094A800D8F800305E4943F4800367F3D753C8F80F
:1094B8000030FFF7AFF92B68198A21B9009108200D
:1094C80001220B4615E00BB2022B0CD101223B46C0
:1094D800082039460097F9F70FF9534B1A7842F0EC
:1094E80008021A7007E0012B05D100970E203946B3
:1094F8003A46F9F701F90CF087FC074678B12B6872
:109508009B7C012B08D1454B5B7803F01003DBB241
:1095180013B10020454941E0002045493EE0414B58
:109528003946187800F00300F8F702FFFF280FD13A
:109538003D4B1B7803F01803182B31D0A07800F0AE
:109548008000C0B210B138463A4927E03A4925E0D0
:109558000CF08AFC8046E0B1334B187800F008081C
:109568005FFA88F8B8F1000F0AD1F9F735F8C0B2F8
:10957800022801D840460AE0062811D8404604E0EF
:1095880000F01000C0B210B138462C4906E02C4952
:1095980004E00CF0B1FC18B12A494046FFF73AF94B
:1095A800294B1B78232B29D1FFF7F8F9337843F09F
:1095B80006033370F8F784FD236823F480036FF300
:1095C800D7532360184B1A786FF3C3021A701F4AD7
:1095D8001378013BDBB213701D4A52F823302B601D
:1095E800104B1B7803F00303022B02D10CF0E2FBB3
:1095F80020B102B0BDE8F0410BF072BB02B0BDE88B
:10960800F08100BF0D190020011900203418002036
:10961800B0310020282100205C2100205E34002089
:1096280052FF020863340020381A002094FF020811
:1096380073FF02085A0003087B0003083900030877
:1096480018000308B5FF0208FC170020EF180020D7
:10965800F018002010B5FFF7A1F9124B2522DA7790
:10966800114B124C1B6818219A7C01FB024251785D
:1096780001F00F000F2814D00A2803DD0A2060F338
:10968800030151709B7C182202FB034463780A2172
:1096980003F00F03594306486B32BDE81040FFF74B
:1096A800DFB810BDF401002034180020BC310020C0
:1096B800100200202DE9F74F984BDFF8B0A2F022F6
:1096C8001A70DAF80030D0469C6847F2DB13E11ACA
:1096D8004C4244EB0104D83A6243914B9D5C9F187D
:1096E800C5F30005EEB29946002E29D130468D49C2
:1096F800FFF790F88C4B1B78232B40F038857B784C
:1097080066F304137B70FFF749F9884B1A7842F027
:1097180006021A70864A1378013BDBB21370854A39
:1097280052F82330CAF80030834B1D70834B1D70EC
:10973800834B1D70834B1E60834B1D7000F017BD5B
:10974800824E814D337893B1814A4FF4A0711378DA
:1097580003F01F005B0959430A2303FB00137D49EB
:10976800CB18DB78002B40F06682137084E06E4BD8
:109778001B78532B40F0FC8095F80080B8F1000F5F
:109788002ED14046214614F06CFC5FFA80FABAF1FB
:10979800000F25D07B7868F304137B706E4F3A78FE
:1097A8001AB9204614F074FB13E0531E6B49002BC2
:1097B800184603EA0101B8BF02F11E004011002952
:1097C80003DA013961F01F01013114F0ADFB002308
:1097D8003B7014F0D9FC85F800A00022594BE2E058
:1097E8002B78002B00F0278256490A680F460B2A6F
:1097F80001D10C2316E00C2A11D1013B6101544A16
:1098080059181170554903EA0101002903DA013991
:1098180061F01F010131204614F086FB1CE0092A83
:1098280002D10A230B60D0E10A2A27D14B49013B18
:1098380003EA0101002903DA013961F01F0101314E
:10984800204614F0B3FB2B786201D318DBB2404AF0
:10985800591E1170404A13704FF00008C7F8008075
:10986800FFF79CF8182303FB04935A7842F0100280
:109878005A7085F8008014233370DCE1043A042A16
:109888003FD83749D2B20878364F60B30020087005
:10989800397841B13448401810F8010C032802D037
:1098A800002840F0C881013B0A2058434FF4A07EAD
:1098B8000EFB0400DFF89CE07044801841716001E1
:1098C8001B18D8B200EB800000F5EC405F30801820
:1098D80007F098F9387818B1013814F0BDFCAAE1FE
:1098E8000DF03CFAA7E101200870013B0A214B4327
:1098F8004FF4A07101FB04331649CB189A18537919
:109908000AE00F4F3B7823B901223A700A4A1370D4
:1099180091E1FFF743F800233B708CE10D1900201B
:10992800BC310020D7B90208FC170020011900201B
:10993800EF180020F0180020191800204218002005
:10994800C1180020D8180020CB18002011180020BA
:10995800C2180020353500207D1900201F00008026
:10996800D71800207C190020E0230020341800209C
:10997800432B1AD1964A1278002A40F043812B785B
:10998800002B00F05881934B1A78002A40F053813D
:10999800914B19680C2903D00A2903D02A7014E1C5
:1099A8000B2200E009221A600FE1232B7ED1884A9E
:1099B8001278002A40F026812978DFF818A20029B9
:1099C80035D09AF8003053B184490F2B0A70844976
:1099D8000A7000F2308101338AF800302BE17E4AA8
:1099E8001368082B1ED84FF4A077674301394FF04E
:1099F8000A0E0EFB01717B4F181F7918C9780627CC
:109A0800013907FB0101784800EB810151F8040F87
:109A18000133002840F0D880032B40F2D580082B72
:109A2800F4D9D1E0092B40F006810233CCE07B78F1
:109A38006E4E61F304137B7032781AB9204614F025
:109A480027FA13E0531E6A49002B184603EA01015E
:109A5800B8BF02F11E004011002903DA013961F094
:109A68001F01013114F060FA0023337014F08CFBED
:109A78000DF074F9FEF792FF5E4B1A7842F0060279
:109A88001A705D4A1378013BDBB213705B4A52F8D7
:109A98002330524AC8F8003000231370504A8AF81D
:109AA800003013704C4A2B70136060E32A2B3CD1B2
:109AB800474A1278002A40F0A58046490B784BB1F6
:109AC8004648012B02704648027040F2B480013BC0
:109AD8000B70B0E02878002800F0AD803E4A13688B
:109AE800002B00F0A880092B1AD84FF4A07161430D
:109AF80001384FF00A0E0EFB00103A491F1F0818D4
:109B0800C1780620013900FB0171374800EB81015B
:109B180051F8040D013B002856D1032BF8D853E027
:109B28000B2B40F08880023B4EE0442B1AD1284A88
:109B38001278002A66D1274B1B78002B7BD1287816
:109B4800431EDBB21E2B76D8214614F08AFAC0B227
:109B5800002870D0204A13680C2B6CD00A2B6AD0CE
:109B680028701BE0552B4DD1194A1278002A49D18B
:109B7800184B1B78002B5ED1287801285BD9023856
:109B8800214614F07FFAC0B2002854D0124A136854
:109B98000C2B50D00A2B4ED019490870043B042BCB
:109BA80013D84FF4A071614301380A2707FB00104E
:109BB8000C490818C1780620013900FB01330A490D
:109BC80051F823300BB904331360FEF7E7FE32E097
:109BD800D7180020C1180020D81800201918002014
:109BE8004218002035350020840D00207D19002002
:109BF8001F00008001190020EF180020F018002035
:109C0800CB180020303BDBB2092B14D89C4A1268D1
:109C1800043A042A0FD89B4A117861B99A4A1278F3
:109C28004AB19A4A0A27107807FB0033DBB2402B67
:109C3800137088BF11702F78DFF8B482002F5FD1BE
:109C480098F8000010F0010012D114B9204690498C
:109C580000E09049FEF7DEFD98F8003043F6DF207B
:109C680043F0010388F8003006F0D6FF8A4B1870DD
:109C7800337813B989488A4901E0884889490A2212
:109C8800F6F75EFE204614F0DBF9874D0146022206
:109C980005F11900FEF7E4FD844B1B7803F08003FF
:109CA800DBB22BB3824B1B88EB81337803BB814B30
:109CB80018781A4618B9204614F0B6F818E07E4B02
:109CC800411E01EA0303002B03DA013B63F01F0383
:109CD80001334FF4A07161430A2505FB031377494B
:109CE800CB18DB7813B914F07DF901E00023137069
:109CF800182303FB0494637843F01003637036E27F
:109D08004FF4A0736343013F0A2202FB07336B4EF3
:109D1800F31893F803B06301FF1898F80030FFB206
:109D280013F0010F46D16648FEF71AFD07EB07113D
:109D380001F5E241DF311022624806F07EFF604BF8
:109D4800594811229A7144230370173BC370791C38
:109D580001300F3AFEF784FD494B1B6813B91020F8
:109D680059491FE0012B02D1102058491AE0022B53
:109D780002D11020564915E0092B02D1102055496F
:109D880010E00A2B02D1102053490BE00B2B02D113
:109D98001020524906E00C2B02D11020504901E056
:109DA80050491620FEF736FD98F8003043F00103BD
:109DB80088F80030334B1A789846002A00F0EB8078
:109DC80007EB071707F5E247DF3710223648394611
:109DD80006F033FF00229146334B995C9A4641B115
:109DE80009F101095FFA89F90132B9F1100FF3D1CC
:109DF80006E003EB09002021C2F11002F6F7CAFAC7
:109E080098F8000048450BD90138C01906F004FF3E
:109E180030B91C4B202118780138C01906F0F2FE21
:109E2800DFF8D09099F8003018460193FEF7AEFDA0
:109E38004A46019BDFF8C09018B9432B40F0858053
:109E480001E0432B04D1002389F80030202173E07E
:109E5800DFF8A8E024499EF800C024489C454FD16B
:109E68000B78ACF1300C0133DBB24FF00A0E0B70FB
:109E78000EFB0C33C35C002B54D10B7052E000BFB7
:109E8800D8180020C1180020D71800207C190020FD
:109E98007CBA020800BB020843320020FA01002005
:109EA80042BB020863BB0208F4010020B031002065
:109EB800692B03087D1900201F000080353500201C
:109EC80010190020171900206BBC02084ABC0208B0
:109ED8008CBC0208F7BD020818BE020839BE020889
:109EE8005ABE02087BBE02084218002054470208E6
:109EF80001190020FC17002019180020161800204E
:109F08008EF8003099F800304FF0000C81F800C04E
:109F180043B198F800300F2B04D803F1010E954B8C
:109F280083F800E0402389F8003013780978303B43
:109F38000A2202FB0313C15C98F8000001380AF8F2
:109F48000010381806F05EFE0EE08B4B1B7803F00D
:109F58008003DBB243B199F800302BB998F8003090
:109F6800FF22534403F8012C99F8003013B1834AB7
:109F7800013B137099F80030012B11D198F800308B
:109F88000F2B02D87B4A013313707D4A002389F8CE
:109F98000030137004E004200C217A4AFEF7F2FB2B
:109FA800794B1F681FBB4FF4A07254432B780A22C9
:109FB800013B02FB0344361975782D090F2D00F07B
:109FC800D680724CA52104F11C00063AF6F7E2F996
:109FD800FF232377002D00F0CA80012D637700F05E
:109FE800C680022DA37700F0C280E377BFE0012F7F
:109FF80018D14FF4A07254432B780A21013B01FB7E
:10A0080003443619737803F00F030F2B00F0AF8069
:10A01800092B04DC01335E485943BD3AA2E05C4891
:10A0280059436AE0022F38D10BF1FF3B5FFA8BFBF3
:10A03800BBF1070F98BF574BDFF850819CBF5B44BB
:10A0480093F8647008F11B0088BF002720210522BF
:10A05800F6F7A0F92878C7EB08080138002318E0BC
:10A068004FF4A07262430A2101FB0022B25C08EBA4
:10A0780007011A4112F0010FC7F1000202D08A1835
:10A08800DB2101E08A18A52182F82010013308F1AC
:10A098000108DAB2BA42E3D369E0032F2FD14FF4B3
:10A0A800A07254432B780A25013B05FB0343F218A1
:10A0B800F35C13F0400F02D01020374906E0937884
:10A0C8005A1ED2B2FD2A06D93449102003B0BDE881
:10A0D800F04FFEF79FBBFE2B02D110203049F5E769
:10A0E80010203049FEF796FB2F4B30481B78013B78
:10A0F80005FB03442E4D2C19A178832232E0043F3E
:10A10800042F34D80622FFB20BF1FF3B02FB0B7B76
:10A11800284B294853F82B100A31F6F711FC274B26
:10A128001B7893B1144B1B7803F08003DBB23BB16F
:10A1380023482021022203B0BDE8F04FF6F72AB9E0
:10A14800204B1F48197882220CE02B780A22013B09
:10A1580053434FF4A07202FB04343619F719184818
:10A168007979BE3A03B0BDE8F04FFEF779BB03B08A
:10A17800BDE8F08FC1180020B03100201918002068
:10A188004218002010190020D8180020F4010020DF
:10A198000F02002054470208B5BD0208ADBC0208F2
:10A1A800CEBC0208D6BD0208CB1800201102002040
:10A1B80035350020840D002004020020D718002027
:10A1C800120200207C1900202DE9F0474C4C4D4F1D
:10A1D8002378F02243F0010323704B4BDFF85C91A6
:10A1E8001A703B68494A9E6847F2DB13F01A4642E8
:10A1F80046EB000618217143555C5318C5F300055A
:10A208005FFA85F89246B8F1000F23D140464049DD
:10A21800FEF700FB99F80030232B6FD1FEF7BEFB49
:10A2280023783C4A43F0060323701378013BDBB2E2
:10A238001370394A52F823303B60384B1D70384B45
:10A248001D70384B1D70384BC3F80080374B1D709C
:10A25800BDE8F08799F80020232A23D15A786FF3B4
:10A2680004125A7013F090FF0CF078FDFEF796FB7D
:10A278002378284A43F0060323701378013BDBB2A6
:10A288001370254A52F82330244A3B600023137088
:10A29800234A1370234A1370234A1360234A137006
:10A2A800BDE8F087532A0DD15A78C2F300144CB98F
:10A2B80042F010025A7021463046013413F034FE41
:10A2C800202CF8D1304613F0BBFE182303FB06A65A
:10A2D8007378C1B213F0100F0AD0202902D10020E0
:10A2E800134901E013490020BDE8F047FEF792BA90
:10A2F80011480222BDE8F047FEF7B2BABDE8F08780
:10A3080001190020341800200D190020BC3100204C
:10A31800D7B90208EF180020F018002019180020FB
:10A3280042180020C1180020D8180020CB1800209F
:10A338006A0203088B0203080D020020FC170020A4
:10A348002DE9F0412D4E2E4F307800F5E240BD301A
:10A3580006F062FC3B78C4B213F0010F26D0294DF9
:10A368002B78552B0AD1EC2C01D0013CE4B2307883
:10A37800214600F5E240BD3006F044FC2B78442B22
:10A388000DD1A4F11403DBB2D72B01D90134E4B207
:10A398003078214600F5E240BD3006F033FC2B78DA
:10A3A800532B03D1FEF7FAFA0CF0D8FC164B1B78A6
:10A3B80003F08003DBB253B13B7813F0010F06D0F2
:10A3C800124820210422BDE8F041F5F7E3BF14F05C
:10A3D800800F0F4805D12B230A21037461431130E4
:10A3E80006E02D230374373B5C43113004F52061EC
:10A3F8000322BDE8F041FEF733BA00BFC1180020C0
:10A4080001190020FC170020B031002004020020B0
:10A41800F40100201FB5204B20491A781AB108789A
:10A4280040F00100087009781C4C11F0010F31D080
:10A438001B490978532901D00AB103E082B90122E6
:10A448001A700DE023290BD1002018701549FEF76A
:10A45800E1F9FEF7A3FA237843F00603237019E025
:10A468001B78012B16D120210A460F48F5F792FFD9
:10A478000E4B68461B681022996806F0DEFB002424
:10A4880009491DF8040001EB4401013417F0BCFE32
:10A49800102CF5D11FBD00BFC118002001190020E4
:10A4A800FC170020A3050308F4010020341800203D
:10A4B800034B1B78532B01D1FEF770BA704700BFCE
:10A4C800FC170020084BFF281A68936807D1917B76
:10A4D80041B10649927C097801FB023302E0927C83
:10A4E80002FB00331846704734180020C1180020BA
:10A4F8004328F8B504460D46174608D1114B0A26DD
:10A508001A7891FBF6F66FF3C3021A7000E00E4654
:10A518002046FEF73BFA90B10A4B303C1A780A26DF
:10A5280002F00801C9B2002918BF002506FB05463C
:10A538006FF3C30236B21A70BE42A8BF3E4630B2AD
:10A54800F8BD00BF01190020634B2DE9F3411A68DB
:10A558009846157C977C614C2DB161482178022280
:10A56800FEF77EF900E02570FF01237807F50C4718
:10A578003C3707EB43075B4E0BB90DB10FE015B93C
:10A5880001A8394601E001A8B91E022206F055FBD0
:10A598009DF80430F3759DF80530337605E006F133
:10A5A80017003F210222F5F7F5FE5B23B37502334E
:10A5B80073764D4B1B7813F0010F61D04B4B1B7812
:10A5C800A3F13002D2B2092A35D822780AB9002D6F
:10A5D80040D1474A117814469942464A01D0002191
:10A5E8001170DFF814E10DF1080C9EF800E0A3F1FA
:10A5F8003000E644DFF80CC1117800EB80006044BD
:10A6080000EB010C0131C9B240189CF86CC090F8FD
:10A618006C000EF804CC117008B1032901D900218F
:10A62800117023700DB9384600E0B81E01A9022246
:10A6380006F0FDFA17E0232B04D12F4B1A7892B9B4
:10A64800013205E02A2B05D12B4B1A785AB1013A71
:10A658001A7008E0532B06D1284A533B1370264A38
:10A668001370FFF725FF264B1B7803F08003DBB23E
:10A67800002B2FD0204B1B78F6182023F37529E0E8
:10A6880045B31A4B1878A0F13003DBB2092B10D868
:10A698001A4A137803B92370013303F001031370C6
:10A6A800D8F800302178B3F91020FFF721FF207087
:10A6B80005E0432803D1114B1B7803B92370104BD5
:10A6C8001B7803F08003DBB223B105482021022266
:10A6D800F5F760FEBDE8FC8134180020431800201F
:10A6E80002020020F401002001190020FC170020BC
:10A6F800161800204218002014180020CB1800203B
:10A70800B031002054470208F7B5394E394D337837
:10A71800394C6FF34103337016F050FAFFF7C8FE57
:10A7280002238DF807302B788BB1344AD17941F068
:10A738000101D171324A207802EBC303D3F8A0702B
:10A7480093F8A5203978FFF7D3FE38700DE03378F9
:10A7580013F0010F06D02378303BDBB2062B9CBFE9
:10A76800264AD37003238DF80730337813F0010F8E
:10A7780012D0244B1B7803F08003DBB263B1297835
:10A788001F4B214803EBC10393F8A4309DF8072021
:10A79800C0182021F5F7FEFD2378232B09D11B4A89
:10A7A8002B781268927C013A934202DA114A0133FB
:10A7B800137023782A2B04D12B7813B10D4A013B4F
:10A7C80013702378532B0FD114F06CF80B4B002126
:10A7D8002970DA7961F30002DA71FFF769FE0C4B30
:10A7E8009A7942F004029A7100232370FEBD00BFDB
:10A7F80001190020CB180020FC170020BC370020CE
:10A8080054470208B0310020F40100203418002019
:10A818002C1A00202DE9F74F864E874C3378874D48
:10A82800232B874F25D12368986843F6F123984254
:10A8380017D1DFF83482296898F8000000F56A50CB
:10A84800713006F0DFF998F80000013000F00100DF
:10A8580088F8000000F56A50713006F0DDF92860CC
:10A8680007E000B2FEF746F828603B7843F008039B
:10A878003B703378532B40F06E81236848F6E932F9
:10A888009B68934202D12A686E4B15E04AF28A32DD
:10A89800934202D12A686C4B0EE04AF20732934287
:10A8A80002D12A68694B07E048F63A42934204D13C
:10A8B8002A68674B02B101221A7023689A6843F626
:10A8C800DD239A420AD1634B29681A7861F30002A2
:10A8D8001A7006F015FD08B106F030FD236843F63E
:10A8E800E0229B68934206D15A4B29681A7861F393
:10A8F800C7121A7019E043F6EA22934206D1554B63
:10A9080029685A7861F300025A700EE043F6E7228C
:10A9180093420AD12968504B19B11A6842F0005283
:10A9280002E01A6861F35D721A6023689A684AF255
:10A9380020439A420AD12968484B19B11A7842F043
:10A94800200202E01A7861F345121A7023689A68A7
:10A958004AF2AD439A4202D1287816F097FE23684E
:10A9680043F6DA229B68934202D12A683C4B05E001
:10A9780043F6E822934203D12A683A4B1A7008E05A
:10A9880048F6F232934204D12B6813B92B4B0122BB
:10A998001A6023689A684AF2AE439A420BD1324A47
:10A9A8002B6812783149032B8B5404D1304B5A79D8
:10A9B80042F010025A71236848F632429B6893426B
:10A9C80002D129682B4A05E048F63542934203D163
:10A9D8002968294A117016E048F63642934203D195
:10A9E8002968264A117015E048F63842934203D187
:10A9F8002968234A11704DE048F63942934202D142
:10AA08002A68204B13E043F60452934202D12A6885
:10AA18001D4B0CE049F24062934202D12A681B4B5D
:10AA280005E04AF29E32934234D12A68184B1A70D4
:10AA38003BE000BFFC17002034180020D818002085
:10AA4800011900205421002098310020902B00206B
:10AA5800FA1700207E190020B0310020684000203D
:10AA68004A3A0020F9310020C1180020981200202D
:10AA7800FC200020303500202E35002061340020D5
:10AA8800D5330020AC1A0020D61000203117002042
:10AA9800B217002048F6EA32934206D12A68A14B41
:10AAA80001201A7001460CF03DFF2368986843F6B0
:10AAB800F12398420DD1DFF87882296898F80000D0
:10AAC80000F56A50713006F09DF8002388F80030D0
:10AAD80002E000B2FDF734FF23689A6843F6981342
:10AAE8009A4236D12968DFF844B2DFF84CA20BEB62
:10AAF800C1031B79DFF83882C3F34113012BDFF858
:10AB08003C9221DD98F8000000F56650203006F0F0
:10AB180079F898F80030DAF8001009EB030211729E
:10AB28000BEBC1021279C2F34112032A0CD17E4AFF
:10AB3800126890681030C01806F064F898F8003071
:10AB4800DAF800204B441A7498F800302A6809F89B
:10AB58000320FFF7ADFC3B78DFF8E48113F0010F29
:10AB680000F0F080216843F698128B68934240F019
:10AB780081806E4A2B68914602EBC3010979C1F3C3
:10AB88004111012906DD6A4A1278072A02D9FDF720
:10AB980005FFE3E03278442A36D15FFA83F82DE0E6
:10ABA80008F10108614B5FFA88F803EBC8031B79C9
:10ABB800C3F34113012B06DD5E4B1B7823BB5C4BB3
:10ABC8001B78072B20D8DFF868A19AF800301F2BD4
:10ABD80008D806F095FB70B109EBC8031B7913F090
:10ABE800100F08D19AF800301F2B07D909EBC803BA
:10ABF8001B79DB0902D0C5F8008005E009EBC80322
:10AC08001B7913F0080FCBD03378552B40F0A68072
:10AC18002E782CE0013EF6B209EBC6031B79C3F38C
:10AC28004113012B09DD434B1B78002B40F0968024
:10AC38003F4B1B78082B00F29180DFF8F48098F8DE
:10AC480000301F2B08D806F05BFB70B109EBC60378
:10AC58001B7913F0100F08D198F800301F2B06D974
:10AC680009EBC6031B79DB0901D02E6076E0002EC4
:10AC7800D0D173E04AF2AE4293420BD006DCA3F582
:10AC88002242A2F5CF72012A0ED803E04AF20B52F3
:10AC9800934209D133782F2B60D9B1F91020303283
:10ACA80093425BDC303B30E043F6F122934207D11C
:10ACB8001F4B1B7823B13078B5F900103B222CE0EC
:10ACC80006F01EFB18B3236843F6C4219A688A422B
:10ACD80003D047F2CD018A4204D13078B5F900108B
:10ACE8002D221AE0A2F56A516139052903D943F6E4
:10ACF800E9218A4201D1012307E043F6E0218A4293
:10AD080002D00A318A4203D100232B6026E023684F
:10AD18003078B5F90010B3F91020FFF7E9FB286087
:10AD28001CE000BF4E33002034180020140400201B
:10AD3800C1180020820D0020D8180020E023002030
:10AD4800011900202368B3F90800FDF7D3FD286036
:10AD580098F8003043F0080388F80030FFF7A8FBA4
:10AD6800236843F6D222986890420BD12B6813B916
:10AD78009C489D4901E09B489C490222F5F7E0FD6B
:10AD88000226B0E14AF20B5290420AD12B6813B95D
:10AD98009748984913E0012B95480CBF9649974965
:10ADA8000DE04AF2AE42904218D12B68012B02D135
:10ADB8008F48934903E0022B05D18D489149102211
:10ADC800F5F7BEFD8EE1032B02D189488E49F6E7DF
:10ADD800042B87480CBF8D498D49F0E74AF29E3213
:10ADE80090420AD12B6813B981488A49E7E7022BB8
:10ADF8007F480CBF88498949E1E74AF29F3290426F
:10AE08000AD12B6813B97A488549D8E7012B40F055
:10AE1800698177488349D2E748F63742904203D0A0
:10AE280043F6EE2290420ED128680A21B0FBF1F2D7
:10AE380001FB12017C4B3031D97730322E219977C2
:10AE48005A7703264FE143F6F12290423ED1774BE1
:10AE58001B78E3B9022229687548FDF701FD43F61E
:10AE6800F220FDF747FD022201465E48FDF7F8FC97
:10AE78003B7813F0010F00F086816E4B1B7803F0CE
:10AE88008003DBB2002B00F07E81694819E0FDF7F2
:10AE980031FD022201466648FDF7E2FC02225148D4
:10AEA8002968FDF7DDFC3B7813F0010F00F06B819A
:10AEB800604B1B7803F08003DBB2002B00F063814A
:10AEC800484820210222F5F765FA5CE143F698121A
:10AED800904240F0F5802B68574EDFF8508156F8C5
:10AEE800331010224248F5F72BFD0DF1060298F8B1
:10AEF80000000DF107010EF0F7FC4246334620B37F
:10AF080016784E49895D03291FD0296803EBC101D2
:10AF18000979C1F34111012917D1072E15D94849DB
:10AF28000B224848F5F70CFD4748711C0222FDF733
:10AF380097FC9DF80710454801310222FDF790FC67
:10AF48009DF806104248013118E02E68157803EB89
:10AF5800C601097903EBC6063679C1F34111012907
:10AF680006F00706C8BF05F00705012E0ADC3949B7
:10AF780034480B22F5F7E4FC3348691C0222FDF73C
:10AF88006FFCAFE0022E0BD133490B222D48F5F7A9
:10AF9800D7FC32462C48691CFDF762FC0E36A2E04D
:10AFA800032E0BD12D490B222648F5F7C9FC26485C
:10AFB800691C0222FDF754FC0D3694E0042E51D191
:10AFC80027490B221F48F5F7BBFC1F48691C0222C2
:10AFD800FDF746FC1D4805F109010222FDF740FC7A
:10AFE8000C3680E012020020244802082648020895
:10AFF8000402002087F10208C9F10208A8F102083A
:10B008005EF002087FF00208A0F00208C1F0020812
:10B018003DF002082CF202086EF202084DF2020816
:10B02800B0F20208D1F20208F4010020C118002091
:10B038000F020020B031002014040020E02300207B
:10B04800150C0308F9010020FA010020FE01002078
:10B0580001020020D30B03082E0B0308B20B0308D0
:10B06800700B0308052E11D148490B224848F5F703
:10B0780067FC4848691C0222FDF7F2FB464805F1C7
:10B0880009010222FDF7ECFB0B362CE0062E29D134
:10B0980042490B223E48F5F753FC3E48691C022200
:10B0A800FDF7DEFB3C4805F109010222FDF7D8FB5C
:10B0B8003B4805F111010222FDF7D2FB0A3612E0E6
:10B0C800B3F91060092E04DD632ECCBF03260226D7
:10B0D80000E0012633482968801B46F08002FDF70E
:10B0E800BFFB00E010263B7813F0010F0BD02E4B6E
:10B0F8001B7803F08003DBB22BB12A482021801B88
:10B108003246F5F747F9294EB37803F00203DBB26C
:10B11800002B38D0FDF7ACFA254D034628B928781E
:10B12800F11D6522FDF7C2FA08E0B2792978B388E3
:10B13800F01D01FB023109B205F07FFD236847F2DB
:10B14800CD029B68934213D006DC43F6C422934297
:10B158000ED043F69A5209E047F24D12934207D0B7
:10B1680048F6F232934203D047F20D1293420AD1C5
:10B1780005200B210D4AFDF705FB29780D48013103
:10B188000222FDF76DFBBDE8FE8F00BF4F0B0308E1
:10B19800F9010020FA010020FE010020910B0308AC
:10B1A8000202002014020020B031002010190020F3
:10B1B800C1180020F5010020F0B5114B1F78114B84
:10B1C800303F1E680DE0D6F814C01CF803C00133E8
:10B1D800644501D112E00023DAB28242F3D301358B
:10B1E8000D70094B0622094902FB07330D785B19DC
:10B1F80093F8D440002CEED10C70F9321046F0BD13
:10B20800FC17002034180020544702084218002078
:10B218002DE9F74F974C984E23689A6843F60553E3
:10B228009A4203D133780BB9013333702368934FB3
:10B238009968B3F910303A78B3F1010848BF03F1BF
:10B2480006084FEAE808337808F1010812F0010F00
:10B2580003FB08188A4D00F0AD808A4B1A7899468E
:10B26800432A4DD128780FFA88FA0AEBD00005F066
:10B27800D3FC2268844B916846F2C46291421860FC
:10B2880001D12A783AB12A78012102F0070211FA8D
:10B2980002F250401860287819780AEBD00005F0BF
:10B2A800B1FC236847F2AD129B68934209D1744BF5
:10B2B8001A78764B03EBD203734A126883F8A021FD
:10B2C8001EE046F67532934205D1317800200131EF
:10B2D8000CF048FE14E046F28B7A4FF0000B23681E
:10B2E8009B68534504D101200BEB00010CF03AFE9A
:10B2F8000AF1080A46F2AB739A450BF1010BEED13D
:10B3080099F80030232B10D122682B78927C013ACF
:10B3180093420ADA5A4A013313705D4B9B7803F063
:10B328000203DBB20BB1FDF771F999F800302A2B53
:10B338000CD12B7853B1524A013B1370544B9B7874
:10B3480003F00203DBB20BB1FDF760F999F80030A6
:10B35800552B14D12368997C0F2910D92A780839DC
:10B368008A42474B01DA083200E000221A70484B43
:10B378009B7803F00203DBB20BB1FDF747F999F8AC
:10B388000030442B42D123689A7C0F2A3ED9297871
:10B398003B4B072902D90839197001E0083A1A709D
:10B3A8003B4B9B7803F00203DBB2002B2ED0FDF75A
:10B3B8002DF92BE048F6A93399420ED1314B1B7871
:10B3C800A3F13101C9B2032907D842F006023A7045
:10B3D80007225343284A573B137023689A6843F659
:10B3E80005539A4212D133781B2B08D9284B46F6BD
:10B3F80061429A809A7842F002029A7006E05901F6
:10B40800C918244B0020C918FDF704FAFFF750F8B3
:10B41800214A2B7811789346994288BF1370127885
:10B428000F32934202DD1C4A0F3B137023684FF022
:10B43800000A93F81290B9F10F0F9ABFC9F12009C9
:10B448005FFA89F94FF010099BF800004FFA8AF368
:10B4580018180FFA88F202EBE000019305F0DCFB04
:10B468009BF80020019B5FFA80FC9B1803F0070300
:10B478002BE000BF34180020C1180020011900205B
:10B48800CB180020FC170020D8180020E02300204B
:10B4980010190020E1F40208C31800204CFA03F048
:10B4A8006549013300F0010000280CBFA520DB200E
:10B4B800DBB201F809000AF1010A09F10109082BB8
:10B4C8005FFA8AFA5FFA89F903D0B9F1200FE5D15A
:10B4D80009E0B9F1200F06D023684FFA8AF19B7C66
:10B4E80089189942B0DB3B7813F0010F15D0236817
:10B4F80052499B7C09780F2B01F0800198BFC3F15A
:10B508001003C9B294BFDBB2002331B129781031DE
:10B518008A1A4949CB185F219954DFF8288198F88D
:10B528000230474603F00203DBB2002B64D0FDF77C
:10B538009FF8034600BB226846F6753192688A4236
:10B5480006D024318A4203D043F6E5118A4204D159
:10B5580030783B496522002309E043F605518A42C9
:10B5680008D130781C38C0B208F107016522FDF710
:10B578009DF818E02878F7E7236846F635329B6887
:10B58800934203D043F6F822934202D1BA79317834
:10B5980001E0BA792978BB88294801FB0231BA79D8
:10B5A80009B205F04AFB23689A7C102A02D90520C3
:10B5B8000B211EE09B6846F6353293420ED006DC1E
:10B5C80043F6E512934209D043F6F82204E046F622
:10B5D8007532934202D02432934201D1102007E001
:10B5E80043F60552934202D10020102101E00020C9
:10B5F8000721144AFDF7C6F8226846F6D931936840
:10B608008B4216D046F693218B4212D043F6ED2199
:10B618008B4202D1084BDB219977937C102B08D9F8
:10B62800297809480131022203B0BDE8F04FFDF73F
:10B6380017B903B0BDE8F08FF4010020B031002045
:10B648001719002010190020F5010020114B0022C5
:10B6580070B50D461A7118B11B7803B920234370D1
:10B66800BDB10D48F5F7E6F80446681C5CB10A4917
:10B678002246F4F7E7FD022C0BDC601C2818202179
:10B68800C4F1030201E020210322BDE87040F4F771
:10B6980081BE70BDB0180020B118002038B505462D
:10B6A800002408E0601905F0B7FA3038C0B209285C
:10B6B80008D80134E4B2044B1B78303B9C42F1DBE0
:10B6C800012038BD002038BD1818002008B505F045
:10B6D800A3FA0023C0B2064AD25C824201D12028D4
:10B6E80004D10133082BF6D1002008BD012008BD84
:10B6F8006448020870B506460D4600240DB12D2396
:10B708002B55A0190021013405F07CFA062CF5D13F
:10B7180070BD00002DE9F04F974C984F206839789C
:10B728008368068A9AB201FB06260D4647F6100181
:10B738008B4287B0B6B20BD1914B1A785B7802F086
:10B748000702C3F3420303EBC20306EBC3062BE075
:10B7580047F6D0118B4212D1894B8A481A7859780A
:10B7680002F0070288235A43C1F34201773B03FBE7
:10B77800012320210822F618F4F70CFE14E047F6FE
:10B7880088518B420BD17E4B1A785B7802F0070206
:10B79800C3F3420303EBC2039B01F61804E0B3F5BD
:10B7A800E97F08BF02EB4506774B784D1A78984633
:10B7B80012F0010F53D123689A6846F6D5739A425E
:10B7C80004D046F6D5539A4240F04481704B1B781A
:10B7D8002A2B3BD16F4B93F8009009F1010909F02E
:10B7E800010983F80090B9F1000F1AD046F6D55335
:10B7F8009A4208D1684B46F661429A809A7842F09C
:10B8080002029A7026E1202110226448F4F7C2FD52
:10B818003B7863495A01D3180020C918FCF7FAFF8E
:10B8280018E15D48FCF79CFF236848469A6846F68D
:10B83800D5539A420CBF5B495B49FCF7EBFF39785B
:10B848005A4801310222FDF70BF803E1552B02D0CB
:10B85800442B40F0FF804F4B00221A70FAE0236817
:10B868005869F4F7E7FF4A4B834693F800A09946D6
:10B87800BAF1450F02D14E4B00221A705046FDF71F
:10B8880085F800284DD04B4B5FFA8BFB1A78524550
:10B898000ED15846FFF790FCFF2804D15846FFF711
:10B8A8008BFCFF283DD0444B1A7801321A7015E002
:10B8B800DFF804A100228AF8002058460593FFF714
:10B8C8007BFCFF28059B04D09AF8002001328AF8F7
:10B8D800002099F80020FF281A7022D02168374AE2
:10B8E8004B6910601B5C886846F6D5718842136006
:10B8F80092460FD1562B01D0542B0BD13B78123BDB
:10B90800DBB2022B06D82B7830B2C01805F084F9C8
:10B91800CAF800002B7830B2C018DAF8001005F029
:10B9280071F999F80030552B17D12368997C0F29A4
:10B9380013D92A7808398A42144B01DA083200E010
:10B9480000221A70144B9B7803F00203DBB20BB190
:10B95800FCF75CFE184B00221A7099F80030442B53
:10B968003BD123689A7C0F2A37D92978074B0729B6
:10B9780026D90839197025E034180020C11800208C
:10B98800C61800200402002001190020CB1800204E
:10B99800FC1700200C19002010190020F4010020C9
:10B9A80004ED020815EB020857EB0208F501002028
:10B9B800141800201618002042180020D81800205B
:10B9C800083A1A70964B9B7803F00203DBB20BB16E
:10B9D800FCF71CFE934B00221A7099F80030432B99
:10B9E8000CD1236830B25B6919788F4B19602B78BA
:10B9F800C01805F007F98B4B00221A7099F800302F
:10BA0800232B13D122682B78927C013A93420DDACA
:10BA1800864A01331370834B00221A70804B9B783F
:10BA280003F00203DBB20BB1FCF7F0FD99F800302C
:10BA38002A2B0FD12B786BB17C4A013B1370794BC1
:10BA480000221A70764B9B7803F00203DBB20BB12D
:10BA5800FCF7DCFDFEF72CFD754A2B781178924631
:10BA6800994288BF137012780F32934202DD704AF0
:10BA78000F3B137023684FF0000B93F81290B9F145
:10BA88000F0F9ABFC9F120095FFA89F94FF0100921
:10BA98009AF8000033B218185844059305F0BCF81A
:10BAA800644A02F8090009F101095FFA89F9B9F154
:10BAB8001F0F059B05D821680BF1010B897C8B456D
:10BAC800E6DB98F8001011F0010F16D021685A48EB
:10BAD800897C00780F2900F0800098BFC1F110011F
:10BAE800C0B294BFC9B2002138B128789AF8006072
:10BAF80010305218801B5F2111542268906849F257
:10BB08003E6290420AD14D4B1B78532B2FD105F042
:10BB180083F84B4B187005F079F928E0B0F5E97F08
:10BB280025D1464A1278532A21D11846FFF7CEFD6F
:10BB38000646E0B93B78DA00D31A03F11200FFF7A2
:10BB4800ADFD60B1FF2300933E4B01961B78792031
:10BB58000133029331460422334605F0DBF83B7883
:10BB68000021DA00D31A03F11200FFF7C3FD2C4EAF
:10BB7800B37803F00203DBB2002B6ED0FCF778FD3C
:10BB8800034680B9226847F6885192688A420AD0EB
:10BB980046F6D5518A4214BF28783878F11D6522B7
:10BBA800FCF784FD0FE02368B2799B682648B3F55B
:10BBB800E97F0CBF39782978B38801FB0231B27963
:10BBC80009B205F03AF823689A7C032A08D99A68DA
:10BBD80047F610018A4203D046F6D5518A4214D15D
:10BBE8009B6847F6100293420CD198F8003013F086
:10BBF800010F01D010202CE0202107221348F4F770
:10BC0800C9FB2AE0B3F5E97F02D105200B2121E029
:10BC180046F6D55293421BD1002010211AE000BFEE
:10BC28001019002042180020D8180020CB18002036
:10BC3800C3180020F4010020B0310020FC170020B8
:10BC480018180020C118002017190020040200202D
:10BC580000200721104AFCF795FD23689A7C032AE7
:10BC680016D9B27802F00202D2B28AB19B6847F6BE
:10BC7800100293420CD046F6D552934208D0297848
:10BC880006480131022207B0BDE8F04FFCF7E8BDD5
:10BC980007B0BDE8F08F00BF10190020F5010020A3
:10BCA8002DE9F04F7A4E8BB033689D6893F8129067
:10BCB800122D01D00B2D09D1764A122D92F8009041
:10BCC800A9F130095FFA89F915D01DE04AF2BB43A2
:10BCD8009D4203D028339D4240F055836E48282169
:10BCE800F4F7D6FB8046002800F050830130282165
:10BCF800F4F7CEFB4AE39F7B37B9684BB846D8794F
:10BD0800FEF7E0FB044615E00027B846FF20FEF7E3
:10BD1800D9FB4AF2AC239D4204460BD14AF28B3040
:10BD280004F07AFFC0B2089020B15C4B9B790BB14C
:10BD3800FCF734FE33685A4D9A68122A1AD19B7B55
:10BD4800C3B12B7813F0010F08D12046FFF7A6FCEA
:10BD5800544B10B101221A7000E018704F4B9B79B8
:10BD680043B12046FFF79AFC20B14E4B1B780BB12C
:10BD7800FCF714FE2978DFF848A111F0010100F062
:10BD880089819AF80030DFF83CB118460793FCF730
:10BD9800FDFD079B002800F0B7804349002008708C
:10BDA8004248434A90F800C013609C45414940F01E
:10BDB8008B8033689B8903F00F03032B21D1ACF1EF
:10BDC800300C0A2000FB0CF03B4BDFF8F0C093F876
:10BDD80000E00590704409900EF1010E1CF8000077
:10BDE800DDF814C05FFA8EFE106083F800E00CEBFB
:10BDF8000E00DFF8C8E01EF80000002871D11870A6
:10BE08006FE0082B2BD12C48ACF1300C03780CEBED
:10BE18008C0E0993294B9E44099B734493F86CE05C
:10BE28000993264BBEF1000F01D180F800E090F88D
:10BE380000E00CEB8C0C634403EB0E0C0EF1010ECE
:10BE48005FFA8EFE73449CF86CC093F86C30C2F8AD
:10BE580000C080F800E0002B43D1174811E0072B01
:10BE680011D1BCF1300F10D11348037823B14FF032
:10BE78002B0EC2F800E001E0C2F800C0013303F065
:10BE8800010303702DE0062B2BD10B78013327E03B
:10BE9800341800201818002004020020CE180020B2
:10BEA80001190020670E00204F3A002016180020C4
:10BEB800D8180020CB180020421800205447020848
:10BEC800FC17002019180020DFF898E203709BF88F
:10BED80000304FF0010C8EF800C013B10B786344AA
:10BEE8000B7040238BF800300B784B4503D39B4BEA
:10BEF80009F1FF30187008781168201804F082FEE4
:10BF08002B7843F004032B709AF80030232B2FD1A1
:10BF1800924B09F1FF311A788A4229DA72B93268EC
:10BF28004AF2BB4192688A4208D028318A4205D039
:10BF38002046079304F070FE079BC8B118780130BB
:10BF4800C0B21870201804F067FE28B9834B20216E
:10BF58001878201804F056FE814B40221A702B786E
:10BF6800804A43F004032B7000238BF800301370D1
:10BF78009AF800302A2B10D1784B1A786AB1013A16
:10BF88001A70774B40221A702B78764A43F00403D4
:10BF98002B7000238BF8003013709AF80030432B75
:10BFA8001FD16E4B1878484505D2201820210793D9
:10BFB80004F028FE079B9BF800203AB91B7809F18A
:10BFC800FF32934202DA654A013313702B78644AD0
:10BFD80043F004032B7000231370624A8BF800307F
:10BFE80013709BF8003013B15F4A013B13709BF844
:10BFF8000030012B0ED1594B1A784A4501D2013233
:10C008001A70584A002313702A7842F004022A70E2
:10C018008BF800302B7803F00402D2B2002A71D0DA
:10C02800524A6FF382031370002111225048F4F72B
:10C03800B1F9504A494B11781B78994288BF13705F
:10C0480011780F318B4202DD4A490F3B0B70117892
:10C0580047481022611804F0F0FD4548F4F7EAFB60
:10C0680033684AF2BB419B68C2B28B4202D0283186
:10C078008B4205D122B94048F4F7DCFB421CD2B20E
:10C088000F2A3FD83A4820218018C2F11002F4F74D
:10C0980081F937E0DFF8D8B011225846F4F77AF979
:10C0A80033684AF2BB429B68934202D028329342DB
:10C0B80009D1214604222E4804F0BFFD40463946E6
:10C0C800FFF7C4FA1EE021461022584604F0B5FDD9
:10C0D8005846F4F7AFFB02462021C2F1100258443B
:10C0E800F4F758F921464A46244804F0A6FD244AA4
:10C0F8001020937882F8069043F00203937001466B
:10C10800FCF740FB9AF80030532B75D133689A68D6
:10C118004AF2AC239A4208D1204604F07DFD20B1B2
:10C128004AF28B30012104F06DFD3368DFF838A046
:10C138009B68122B40D12046FFF7B0FA83460028AF
:10C1480030D0104BFF2219780F4BF9B900920191AA
:10C158001B78782001330293FB3A1FE0CB180020AC
:10C168004F3A002042180020191800200119002019
:10C17800B0180020C3180020B11800204B18002068
:10C1880044180020670E0020C118002000210092EA
:10C1980001911B787A200133029304220B4604F0A4
:10C1A800B9FD09E08AF800007D492046FFF7A2FAA8
:10C1B8007C4B83F800B0EFE020464946FCF738FB9B
:10C1C800794B0020187033688AF800009B6849F2A0
:10C1D8005262934202D10090013005E04AF2CE2229
:10C1E800934206D1012300930146024603460BF011
:10C1F800E5FE6E48FCF7B4FAFEF75AF92B7813F00F
:10C20800010F17D033684AF2BB429B68934202D0B1
:10C218002832934204D140463946FFF717FA09E01D
:10C228005F4B634A03F1100153F8040B8B4242F849
:10C23800040BF9D133689A68122A1ED19B7BE3B1AB
:10C248002046FFF72BFAC0B12B7813F0010F14D159
:10C25800584B9A7922B9DA79574B1B789A420CD005
:10C26800564B1A780023303A05E055492A20C91858
:10C2780001330874DBB29342F7DB326893680B2B07
:10C2880001D0122B0AD14A4B991D13F8010B202813
:10C2980002D10D3003F8010C8B42F6D192684AF2B4
:10C2A800AC239A4214D1434B9B798BB1089878B14F
:10C2B8004FF0000909EB040004F0AEFC18B1404B44
:10C2C8002A224B441A7409F10109B9F1100FF1D16E
:10C2D8002B7813F0010F25D03A4B1B7803F080031D
:10C2E800DBB2FBB133689A684AF2BB439A422D4BE2
:10C2F80003D04AF2E3418A420CD11B7833B9B8F132
:10C30800000F0FD05F3388F801300BE057B15F2280
:10C31800FA5407E0244A1B78127810339B1A284AEB
:10C328005F21D154284CA37803F00203DBB2002B21
:10C3380032D0FCF79DF92049034628B908786522D0
:10C34800E11DFCF7B3F912E03068B4F90430A279C2
:10C3580084680978122C01FB023105D1807B18B959
:10C368001449C97902FB0131184804F066FC3368A6
:10C378009B68122B10D10820134A01460BB0BDE868
:10C38800F04FFCF7FFB90027B84600E0074609F16F
:10C39800FF395FFA89F9B9E40BB0BDE8F08F00BF47
:10C3A800B0180020CB180020C31800204418002023
:10C3B80004020020CE180020C11800201818002000
:10C3C800F4010020B03100201019002017190020B6
:10C3D80024282DE9F041144626D16B4B43F6383218
:10C3E8001B686A4D9B686A4E934206D12B7813F0FE
:10C3F800010F0ED02438674909E04AF2E34293421C
:10C408000AD12B7813F0010F03D063490020FCF701
:10C4180001FA2978490800E0297830190131022207
:10C42800FCF71EFA0234AAE0E72809D1574B58480E
:10C438001978801801310322FCF712FA03349EE0C0
:10C44800A3282AD1514D2B783F2B15D81046534994
:10C45800FCF7E0F95148F4F7EDF92A2124184C4883
:10C46800E4B2F4F715F8002800F08A80297802224F
:10C478000131FCF7F5F983E05901494DC9186918EC
:10C4880001F57E5110467031FCF7C4F905F590406E
:10C498000F30F4F7CFF9241871E0F22821D13B4F7F
:10C4A8003B4D3978072605EB0208B1FBF6F140460B
:10C4B80001310222FCF7D4F939782D23B1FBF6F6C5
:10C4C80088F80230F3009E1B8B1B364FDBB207EB5C
:10C4D80083031988E21CA9529B78A8188370063434
:10C4E8004DE025280BD1304B46F661429A80452213
:10C4F8009A719A78053842F002029A703CE05E28F8
:10C508000BD1294B46F661529A8045229A719A7846
:10C518003E3842F002029A702EE07C280BD1224B62
:10C5280046F244129A8011229A719A785C3842F045
:10C5380002029A7020E0EC280BD11B4B46F6A5525C
:10C548009A8045229A719A78CC3842F002029A7001
:10C5580012E0A7280BD1144B46F6C5529A80452203
:10C568009A719A78873842F002029A7004E0E028BB
:10C5780001D1541C03E018B1054B18550134E4B23D
:10C588002046BDE8F08100BF34180020C118002003
:10C59800F401002069E5020827E50208E3EC020837
:10C5A800D4A4020845D002081019002038B50A4B57
:10C5B80046F69B251B78002405FB030507E0074B7F
:10C5C80022461978FFF704FF041B2D190446287822
:10C5D80008B11F2CF3D938BD17180020C118002046
:10C5E80070B5002543F61C64204604F015FB06468A
:10C5F80004F1080004F010FB16F0FF0F06D020F03D
:10C608007F0010F0FF0F01D00135ADB246F23B13A9
:10C618009C4201D00934E7E7284670BD38B5B0F927
:10C6280000500B4C05EBC50505F578552435284613
:10C6380004F0F2FAC1B211F0800F07D0238828461F
:10C64800013B01F07F01238004F0DCFA208838BD2B
:10C6580012180020454B2DE9F74F1B88444A044621
:10C6680089461788DFF80C8123B14FF0000A0AE0E9
:10C678009A4608E00529FBD198F8003043F00403F6
:10C6880088F8003070E098F8003013F0030F0BD0F2
:10C6980013F0010F02D0B4F1FF3F05D103F00203FC
:10C6A800DBB21BB1012C01D03F19BFB23BB2B3F1D1
:10C6B800FF3F04D0B3F57A7F08BF002701E040F2BE
:10C6C800E7370FFA87FB0BEBCB0303F5785303F13E
:10C6D8001C00019304F0A0FA10F0FF0F019B16D084
:10C6E800B9F1050F09D103F1240004F095FA20F0FF
:10C6F8007F0010F0FF0FC6D022E0B9F1000F1FD065
:10C7080003F1240004F088FA00F07F0618E00AF12B
:10C71800010AB4F1FF3F1FFA8AFA04D198F80030F1
:10C7280043F0010305E0012C05D198F8003043F0EF
:10C73800020388F80030BAF57A7F0DD03D46A2E7AB
:10C748004E4505D0B9F1000F02D0B9F1050F9AD1C5
:10C75800BAF1000F05D000E03D46054A2DB215603C
:10C7680002E0034BC3F800B0BDE8FE8F12180020AA
:10C77800D8180020DC180020F0B503789BB05A1EAA
:10C78800D2B2792A0F4600F2C8805E01644AF318D3
:10C798009B18644A46F69B261278457806FB0236B3
:10C7A800E7213046F3F774FE0446F0B930467C21A1
:10C7B800F3F76EFE0446C0B930462521F3F768FE4C
:10C7C800044690B930462421F3F762FE044660B966
:10C7D80030464021F3F75CFE044630B93046F92173
:10C7E800F3F756FE0446002876D0A41B0FB14E4836
:10C7F80000E04E4831462246A619F4F7A1F8304623
:10C80800E721F3F745FE30B128466946652246F62A
:10C81800A553FBF74BFF30467C21F3F739FE50B1A7
:10C82800691EC9B201EB011101F5C24168464431E4
:10C83800112204F002FA30462521F3F729FE38B117
:10C84800681EC0B26946652246F66143FBF72EFFB3
:10C858003046F921F3F71CFE38B1681EC0B26946AC
:10C86800652246F66153FBF721FF30464021F3F776
:10C878000FFE50B1691EC9B201EB011101F5E24189
:10C888006846DF31112204F0D8F930462421F3F745
:10C89800FFFD50B10FB1244800E024480019294693
:10C8A8000222FBF7DDFF02340BE00FB11E4800E067
:10C8B8001E4800196946F3F75FFF6846F3F7BAFFA9
:10C8C8000419002F29D01A4A9378141943F0020347
:10C8D80093700023E37116E03046F3F7ABFF05468B
:10C8E8001FB9124831462A4615E0102810DD2A469D
:10C8F8000D483146F4F724F80D4A9378551943F05A
:10C9080002039370EC7110200146FBF73BFF04E033
:10C91800084831461022F4F713F81BB0F0BD00BFE9
:10C92800E9D4020817180020171900202C2A002023
:10C9380010190020040200200C4B1B7813F0010290
:10C9480002D000200A4905E003F00200C0B218B185
:10C9580008491046FBF75EBF03F00403DBB20BB1D6
:10C968000549F7E705480121FFF706BFDC18002055
:10C9780090AC02086FAC0208B1AC020803190020A1
:10C9880070B5124D124C00201249FBF753FE284691
:10C99800A1780222FBF764FFE81CE1780222FBF78A
:10C9A8005FFF05F1080021790222FBF759FF05F125
:10C9B8000B0061790222FBF753FFA17905F10E0004
:10C9C8000222BDE87040FBF74BBF00BFF401002016
:10C9D800031900206D4802082DE9F341504F514CCE
:10C9E8003B689D7C237813F0010F2FD1022243F678
:10C9F8001A610DF1060004F020F94B4EBDF806301F
:10CA08004FF0FF3033602946FFF724FE237843F0C8
:10CA180001032370454B1B7813F0030F14D1B6F9AB
:10CA28000010434801EBC10101F578511C3109227E
:10CA380004F003F93F4B1B881BB13046FFF7EEFDAE
:10CA480010B90020F9F7E0FAFFF79AFF3A4E337869
:10CA5800552B0DD1DFF8D4803848FBF781FE98F8C4
:10CA680000304FF0FF306FF3410388F800300DE0DD
:10CA7800442B2BD1DFF8B4803048FBF771FE98F8CF
:10CA8800003001206FF3000388F800302946FFF7D3
:10CA9800E1FD98F8003013F0030F15D1224D24481A
:10CAA800B5F90010092201EBC10101F578511C31DB
:10CAB80004F0C3F81F4B1B881BB12846FFF7AEFDD7
:10CAC80010B90020F9F7A0FAFFF75AFFFFF734FF73
:10CAD8003378232B22D1154B184E1A7802F0FC021A
:10CAE8006FF382021A70FBF759FFB3786FF34103B3
:10CAF800B370134B1D7835B9FBF788FD3046FBF74B
:10CB08002FFE3D600AE02278013DEDB242F00602B8
:10CB180022701D700B4B53F825303B60BDE8FC813B
:10CB28003418002001190020D8180020DC18002033
:10CB38000319002012180020FC17002010190020EB
:10CB4800EF180020F01800202DE9F0411646104A91
:10CB58000F4653780E21C3F342034B43117803F574
:10CB6800EE43A0330B4D01F00701044603EB4101EE
:10CB7800022204F062F8E81921780222FBF770FE1D
:10CB88006178A8190222BDE8F041FBF769BE00BF31
:10CB9800C6180020F4010020044B02225978044BE7
:10CBA800C1F3420118180131FBF75ABEC61800201C
:10CBB800F401002010B5074B074C1B78074A03F017
:10CBC800070304EB83031C88111814529B788B709D
:10CBD80010BD00BFC618002045D00208F40100208F
:10CBE800084B1B789B0902D0012B06D102E01020CC
:10CBF800054904E01020054901E005491020FBF72C
:10CC080009BE00BFC618002032B9020853B902088D
:10CC180074B902082DE9F041DFF868800F4698F8EA
:10CC28000010174DC1F382010446164605F10800AD
:10CC380001310222FBF714FE98F80010042201F0DB
:10CC48001C0101F50A41204601F5C47103F0F5FF06
:10CC5800E81921780222FBF703FEF81C28186178EE
:10CC68000222FBF7FDFDA819A1780222FBF7F8FDC7
:10CC7800F01CE17828180222BDE8F041FBF7F0BD6E
:10CC8800F401002015180020064B1B7803F08003E0
:10CC9800DBB233B1435C04482021C0180222F3F709
:10CCA80079BB7047B0310020F40100202DE9F7432B
:10CCB800654D664C2B6821789B68022203EB410185
:10CCC8000DF1060003F0B9FF2B68A9469A6843F6F0
:10CCD800F4239A4208D100205D49FBF79BFDBDF87B
:10CCE80006804FF4B46303E0BDF806804FF4616337
:10CCF800B8FBF3F103FB11883C221FFA88F8B8FB54
:10CD0800F2F302FB1388CFB2DEB202225148394651
:10CD1800FBF7A6FD5FFA88F802224F483146FBF779
:10CD28009FFD02224D484146FBF79AFD4C4B1B786C
:10CD380013F0010F6ED04B4B4B4D1878232804D1BC
:10CD48002B78012B62D8013305E02A2805D12B78EE
:10CD5800002B5BD0013B2B7058E0A0F13003DBB215
:10CD6800092B01D943284BD12B7873B9D9F8003056
:10CD780039B29A6843F6F4239A4201D10A2200E0B4
:10CD88001122FDF7B5FBC7B216E0012B0ED1D9F879
:10CD9800003031B29A6843F6F4239A4201D117223F
:10CDA80000E03B22FDF7A4FBC6B205E041463B226A
:10CDB800FDF79EFB5FFA80F8D9F800309A6843F6D1
:10CDC800F4239A4209D13C235E434FF4B46303FB36
:10CDD8000767B844ADF8068006E038463146424653
:10CDE8000EF0ABF8ADF80600D9F8003020789B6853
:10CDF8000DF1060103EB4000022203F018FF05E0E5
:10CE0800532803D100232B70FDF752FB17482978CC
:10CE1800FFF73AFFD9F800309A6843F6F4239A42AC
:10CE280010D02078124965220023FBF73FFC05202B
:10CE38000B21104AFBF7A6FC21780F48013102228A
:10CE4800FBF70EFDBDE8FE8334180020C118002052
:10CE580068E90208040200200A02002012020020E9
:10CE680001190020FC170020CB1800207E4802087A
:10CE78001719002010190020F501002073B59A4BEE
:10CE88009A4D1A7812F0010F05D12A7812F038025B
:10CE980004BF2A706A701A78934E42F001021A7021
:10CEA8002B78924C13F038023ED1914909785529D4
:10CEB80004D113F0070F2FD0DA1D0AE044290CD152
:10CEC80003F0070201323D3992FBF1F1C800411A23
:10CED800521A62F3020323701EE053290AD1C3F3E6
:10CEE800C201013161F3C5032370637862F3430320
:10CEF800637011E023290FD1FBF750FD33787D4A89
:10CF080043F0060333701378013BDBB213707A4A9F
:10CF180052F82320794B1A6000207949FBF77AFCF4
:10CF28001C20FFF747FEDDE0082A2ED175490020B6
:10CF3800FBF770FC0620FFF72FFE0C20FFF73AFEE8
:10CF48001521182201A8FFF7FFFD694B1B78552B07
:10CF580006D1637803F0FE03C3F34202013A07E007
:10CF6800442B0BD1637803F0FE03C3F34202013272
:10CF780002F0030262F343036370B3E0532B28D03B
:10CF8800232B40F0AF802378A6E0102A51D15D49C9
:10CF98000020FBF73FFC0620FFF7FEFD0C20FFF703
:10CFA80009FE1521182201A8FFF7CEFD6178564821
:10CFB80001F00101FFF768FE4D4B1878232801D0D6
:10CFC8002A2804D16378DA4362F30003D4E75328AC
:10CFD80004D12378C3F3C202013280E0A0F1300308
:10CFE800DBB2092B01D943287CD16B7802AA03F064
:10CFF80001033B21D41883F001024B43172606FB9B
:10D00800023214F8041CFDF773FA04F8040C6B7868
:10D018000E22C3F342035343287803F5EE43A033AB
:10D0280000F0070003EB400001A90C3A03F0FFFDF4
:10D0380058E0182A4DD133490020FBF7EBFB0620B6
:10D04800FFF7AAFD0C20FFF7B5FDFFF7C9FD284B38
:10D058001B78552B07D1237813F0C00F42D0C3F3A8
:10D068008112013A06E0442B07D123789A09012A54
:10D0780038DC013262F3871333E0232B04D12378A1
:10D08800C3F3C202023A2AE0532B2BD1FBF786FCEA
:10D0980033781E4A43F006033370164B1648197846
:10D0A80040F82120013119702378C3F3C2010131FE
:10D0B80061F3C503C3F381112370104B11B101292A
:10D0C80004D101E01C3202E0114A00E0114A1A6062
:10D0D80008E0114A00211170C3F3C202013A62F359
:10D0E800C50323707CBD00BF01190020C6180020AD
:10D0F800FC170020EF180020F0180020341800203A
:10D10800F0B8020811B902088148020884480208E8
:10D11800BC480208D8480208CB18002073B5494B10
:10D12800494D1A7812F0010F04D12A7812F003023F
:10D1380008BF2A701A78434E42F001021A702B7801
:10D14800414C13F003022ED1404A1278552A03D1DC
:10D15800C3F38202013A04E0442A06D1C3F38202EF
:10D16800013262F38403237017E0532A03D15A1C57
:10D1780062F30103F7E7232A0FD1FBF70FFC33789B
:10D18800334A43F0060333701378013BDBB2137064
:10D19800304A52F82320304B1A6001A810211B2274
:10D1A800FFF738FD4DE0012A4BD101A810211A32B2
:10D1B800FFF730FD254B1878232804D12378C3F3D3
:10D1C8004112013205E02A2807D12378C3F341121E
:10D1D800013A62F3461323702DE0532804D12378D3
:10D1E800DA1C62F30103F6E7A0F13003DBB2092B86
:10D1F80001D943281FD12B7802AAC3F34113D418AD
:10D208000C215A1C03F001034B4302F001021F26B4
:10D2180014F8041C06FB0232FDF76AF904F8040C42
:10D22800287801A900F01C0000F50A4000F5C47038
:10D23800042203F0FCFC29780848C1F34111FFF7E8
:10D2480023FD7CBD0119002015180020FC170020C3
:10D25800EF180020F018002034180020F4480208C5
:10D26800064B1B7803F08003DBB233B1435C044800
:10D278002021C0180322F3F78DB87047B031002081
:10D28800F40100204328F8B504460D46174606D198
:10D29800104B00261A786FF3C3021A7000E00E468E
:10D2A8002046FBF773FB90B10A4B303C1A780A26EC
:10D2B80002F00801C9B2002918BF002506FB05467F
:10D2C8006FF3C30236B21A70BE42A8BF3E4630B2F0
:10D2D800F8BD00BF011900202DE9F3416E4F6F4ED4
:10D2E8003B7843F001033B70347844B94AF2033089
:10D2F80003F092FC6A4B6B491860204617E0012C3A
:10D3080002D10020684912E0022C02D100206749AE
:10D318000DE0032C02D10020654908E0042C02D15D
:10D328000020644903E0052C03D163490020FBF782
:10D3380071FA3178D9B9614B1B78312B01D10131A0
:10D3480001E0302B05D1564B4AF20330196003F047
:10D3580059FC5B4B1A785B4B02F08002D2B20AB1DF
:10D36800202202E04E4A12683032DA776EE0012954
:10D378000BD002290CD003290DD004290ED04AF273
:10D38800FF25052918BF00250AE04AF2EF2507E026
:10D398004AF2F32504E04AF2F72501E04AF2FB25B8
:10D3A8002946042201A803F048FC474B474A03F1E9
:10D3B800100153F8040B8B4242F8040BF9D10322F5
:10D3C80043489DF80410FBF74BFA032241489DF8A7
:10D3D8000510FBF745FA03223F489DF80610FBF7B6
:10D3E8003FFA3E4803229DF80710FBF739FA334B02
:10D3F8003B4C1878232804D12378022B22D80133F8
:10D4080004E02A2804D12378E3B1013B237019E012
:10D41800A0F13003DBB2092B01D9432812D194F8CB
:10D42800008002AA904418F8041CFF22FFF72AFF84
:10D4380008F8040C207802AA131813F8041C2818FA
:10D4480003F0E0FB27482178FFF70AFF1B4B1B7806
:10D45800532B1FD1224B00221A7033780133DBB2D1
:10D46800062B337004D0012B14D10D4B1B688BB1E4
:10D47800FDF71EF8002333703B781B4A43F0060380
:10D488003B701378013BDBB21370184A52F8232023
:10D49800174B1A60BDE8FC8101190020C118002053
:10D4A800D8180020EE0203081704030838040308FC
:10D4B800590403087A0403089B040308FC17002096
:10D4C800B0310020F40100205C2B03080402002086
:10D4D80005020020090200200D0200201102002090
:10D4E800CB180020F8480208EF180020F018002098
:10D4F8003418002070B5174C0D460646002120460A
:10D508004FF4C172F2F746FFFF2D0AD1B10001F5C1
:10D51800D84120466131042203F08FFB23789BB960
:10D5280070BDFE2D01D1173E02E0FD2D02D101365E
:10D53800267009E0B60006F5D8406130401903F0BE
:10D548006BFBC0B2207020B10248BDE8704015F0F6
:10D55800B7BB70BD241B00202DE9F04115F0E2FB9C
:10D5680060B110208F49FBF755F98F4B1B78432B7F
:10D5780040F0EE81BDE8F04115F0F6BB15F0E4FB94
:10D58800002826D0894C23786BB110208849FBF7F6
:10D5980041F988482D211030F2F77AFF002800F071
:10D5A800D781217810E010208349FBF733F98148AF
:10D5B8002D211030F2F76CFF0446002800F0C881D6
:10D5C80015F0DAFB014620468222BDE8F041FBF760
:10D5D80047B97A4C43F6CC2223689B68934250D0D3
:10D5E800774E744D307803EB800003F015FB03226F
:10D5F80001467448FBF734F92368986846F6C55322
:10D6080098422BD0203B984228D03378013000EB49
:10D61800830003F001FB0322014605F11500FBF727
:10D628001FF9236830789B68023303EB800003F00E
:10D63800F3FA0322014605F11900FBF711F92368F3
:10D6480030789B68033303EB800003F0E5FA03228C
:10D65800014605F11D00FBF703F90EE02D21032219
:10D668005948F2F797FE2D2103225848F2F792FE07
:10D6780057482D210322F2F78DFE20232B772B7696
:10D688002B75544B1B7813F0010F00F0BD802368F5
:10D6980043F6CC229B68444D934261D04E4E484F8E
:10D6A80032783878D31803EB800003F0B5FA4B4B87
:10D6B8000146186028789846A0F13002D2B2092AAB
:10D6C80001D943280FD109B2BA22FCF711FF236808
:10D6D80032789B680146C8F800003878D31803EB05
:10D6E800800003F08FFA2B782A2B04D1337813B1FA
:10D6F800394A013B13702B78232B0ED13378022B38
:10D708000BD8226846F6A55192688A4205D0203186
:10D718008A4202D0304A013313702B78552B01D03E
:10D72800442B0FD1236831789B68A3F5D843B3F114
:10D73800610248BFA3F15E023B7803EBA202D0B2BC
:10D74800FFF7D8FE264B1B7803F08003DBB23BB112
:10D758003278184B03EB820320225A749A74DA74D5
:10D768002B78532B06D023689A6843F6CC239A4229
:10D7780040F0EE80FBF712F9236846F661429B6899
:10D78800934203D10E4B0220197806E046F6C552A3
:10D79800934227D10A4B002019780131BDE8F041A6
:10D7A8000AF0E0BB1DEC0208FC170020D010002096
:10D7B800F4EA0208F40100203EEC020834180020C4
:10D7C800C118002005020020090200200D020020D7
:10D7D8001102002001190020CB180020D8180020C1
:10D7E800B031002046F6A552934204D1594B01208E
:10D7F80019780918D2E746F66152934240F0A8809A
:10D80800544B03201978C8E7236849F252629B6891
:10D8180093423ED14F4E10204F49FAF7FBFF317823
:10D828004E4D01EB011101F51641523110222846E7
:10D8380003F003FA2B4605F110012A461078474FEA
:10D8480078B94749FAF7E6FF3846E721F2F720FEAC
:10D8580078B13178401B381801310322FBF700F802
:10D8680007E013F8010B10B9203003F8010C8B42C4
:10D87800E4D13C4D2B782A2B03D13078FD21FFF7DA
:10D8880039FE2B78432B63D1307823680130C0B23E
:10D8980059E043F6CC229342324E1AD01020324936
:10D8A800FAF7B8FF33782A2B52D1304B1B689B68A4
:10D8B800A3F5D843B3F1610248BFA3F15E02254B3B
:10D8C800FF211B7803EBA202D0B2BDE8F041FFF7BD
:10D8D80011BE33781F4D552B04D12B78142B01D151
:10D8E800033B2B703378442B05D12B78122B02D1B4
:10D8F800184B15221A702B78DFF874805901C91853
:10D9080001F59041303100204144FAF783FF08F5D2
:10D918008E41102028312F78FAF77CFF3378112FA9
:10D928008CBF032700272A2B05D12878FE21C01B8E
:10D93800C0B2FFF7DFFD3378432B09D12B78173BB3
:10D94800DF1B2368F8B2997CBDE8F04115F0D2B925
:10D95800BDE8F081C1180020FCEB0208F4010020AA
:10D96800F3CD0208FC170020BAEB02083418002097
:10D97800D4A4020810B50E4B1B78452B17D10D4BBC
:10D988001A7842F006021A700B4A1378022B0ED846
:10D998000A490B4C086844F8230001331370836864
:10D9A8000B60FAF73FFEBDE81040FAF7F7BF10BD6D
:10D9B800FC17002001190020EF180020341800205F
:10D9C800F018002010B50C4B04462146D8790DF00C
:10D9D80076FA68B1094B1B5D543BDBB2012B09D8C1
:10D9E80020460DF063F9D0F1010038BF002010BDCA
:10D9F800022010BD022010BDCE180020DD3200200C
:10DA080008B50DF04BFAC0B208BD00002DE9F0478B
:10DA1800634B644C1A78994612F0010F624D65D039
:10DA28002078FFF7CFFF614A2B181178604F93F8E1
:10DA3800A831604E44293870336090460AD12D2BA6
:10DA480008D038B995F8A91101233B7031602078C6
:10DA5800FFF7D6FF98F80030552B10D133682D2BDF
:10DA68000DD03B785BB1013B514ADBB21370EB1828
:10DA780093F8A8114F4B20781960FFF7C1FF98F869
:10DA88000030232B19D14C4B20781B689B7C013B21
:10DA9800984212DA434B0130C0B21870FFF792FF78
:10DAA8003870281890F8A8313360444B9B7803F0FD
:10DAB8000203DBB20BB1FAF7A9FD98F800302A2B64
:10DAC80014D1207890B1374B0138C0B21870FFF7E5
:10DAD80079FF3870281890F8A8313360374B9B7855
:10DAE80003F00203DBB20BB1FAF790FD344EFCF7FA
:10DAF800DFFC237832789A4288BF337032780F324D
:10DB0800934202DD2E4A0F3B1370DFF8C4800027D2
:10DB180030783818C0B2FFF755FF281890F8A831A8
:10DB28000137102F08F8013F07D0254B1A78224BF0
:10DB3800BA181B689B7C9A42EADB99F8003013F00C
:10DB4800010F13D01F4B1A781F4B02F08002D2B27C
:10DB58002AB1227831781032521A5F2105E02278F2
:10DB680031781032521A134909689954134DAB7819
:10DB780003F00203DBB25BB12078E91D652246F6AB
:10DB88006153FAF793FD05200B212A46FAF7FAFDAF
:10DB980021780E4801310222BDE8F047FAF760BE4D
:10DBA80001190020CB18002054470208FC17002058
:10DBB80014180020D818002034180020101900204C
:10DBC800C3180020B0310020F4010020F501002026
:10DBD800030200202DE9F041074610460D46144681
:10DBE800F2F728FEC3B28046B3B1AB4214D80B4E4D
:10DBF80020212A46F019F2F7CDFB2046F2F71AFE4B
:10DC0800C8EB05056D08EDB2EF1902462146F0197B
:10DC1800BDE8F041F2F716BBBDE8F081F401002041
:10DC2800F0B5134B1A1894781F4604B30E780023E6
:10DC38003A1892781A4112F0010F4FF001020DD0F4
:10DC4800A6420D7803D09A4042EA050504E09A40BE
:10DC5800C2F10F0202EA05050D7005E09A400D7841
:10DC6800C2F10F022A400A700133042BE0D1F0BD43
:10DC7800CE180020312200230178194111F0010F3C
:10DC880002D00449C9188A7501330132042BD2B273
:10DC9800F2D17047F4010020034670B50846684A7F
:10DCA80031B11278532A40F0C980533A1A7070BDC6
:10DCB8001278302A24D163491C780A7822400FD080
:10DCC8000A78024112F0010F06D0012282401C7826
:10DCD800C2F10F0222401A7001300428F0D10CE082
:10DCE8000878104110F0010F04D0012090401C78F2
:10DCF800204318700132042AF2D1534800211AE057
:10DD0800A2F13100C0B2032825D84E4A1278024148
:10DD180012F0010F00F092801C7854FA00F212F011
:10DD2800010F4FF001020BD08240C2F10F0202EA4C
:10DD3800040445481C701322BDE87040F2F72ABB62
:10DD480082404149441C4C741C7822431A701022AA
:10DD580046F6A5536EE0132A0BD0552A17D13B4A35
:10DD68003B491278172000FB0212527912F0200F5B
:10DD780064D00024344D194620466C74FFF750FFD8
:10DD8800304B9B78002B59D0204629464FE0142A67
:10DD98000BD02A2A16D12D4A2D491278172000FBBC
:10DDA8000212527912F0200F48D0274C002219464F
:10DDB80062740120FFF734FF224BDB78002B3DD043
:10DDC800012033E0152A0BD0232A16D11F4A2049F7
:10DDD8001278172000FB0212527912F0200F2DD072
:10DDE800194C0022194662740220FFF719FF154BDF
:10DDF8001B79002B22D0022018E0162A0BD0442AC7
:10DE08001CD1124A12491278172000FB02125279CB
:10DE180012F0200F12D00C4C002219466274032015
:10DE2800FFF7FEFE074B5B7943B103202146102222
:10DE380046F6C553BDE87040FAF738BC70BD00BF60
:10DE4800FC170020CE180020FE170020C418002060
:10DE58007D3200202DE9F04F87B09DF84050804674
:10DE6800072D0E4605929A4637D100242746337867
:10DE7800234113F0010F2CD0012523B24FF00008E5
:10DE88000293512029462A462B460095CDF8048056
:10DE980002F040FF1B20414662194346CDF800803E
:10DEA800F4F72AFC37B9112039463A462B46009731
:10DEB800F4F722FC534B204613F8242001276FF374
:10DEC800000203F824201199F5F786FA2046F5F7A1
:10DED80087FC0134042CCAD1F7E1012D03780CD159
:10DEE8000BB90B7823B3FF2300930021464B019114
:10DEF8001B780C200133029316E0022D09D10BB9CF
:10DF08000B78ABB10021FF230093019102913420DB
:10DF18000AE0062D0CD10BB90B784BB10021FF2379
:10DF2800009301910291652004220B4602F0F2FE53
:10DF3800BAF1010F98F800302BD13BB1334B0020D8
:10DF4800D979024653460090F4F7D6FB33783BB1B3
:10DF58002E4B0120D979002203460092F4F7CCFB1E
:10DF68000020F5F72BFA98F80030002B5BD0284BEF
:10DF78001978002957D1274B5B78002B53D0FF2302
:10DF880000933A2001220B460191029102F0C2FE51
:10DF980049E063B1052D4FF0000102D100910F2037
:10DFA80001E000910B200A460123F4F7A5FB337822
:10DFB80083B1052D4FF0000106D110200A46012338
:10DFC8000091F4F799FB12E00C200A460123009116
:10DFD800F4F792FB022D25D0032D01D10E4B02E060
:10DFE800042D02D10D4B1F781DE0052D01D10C4BDE
:10DFF800F9E7012D01D1044BF5E7062D0CBFFF27EA
:10E00800002710E008150020D5150020CE180020A4
:10E01800F6140020670E0020D81A002027390020A7
:10E02800CF330020FF2798F80030002B00F09D80A8
:10E03800914C237803F02003DBB26BB18F4B197836
:10E0480011F0010108D1FF230093282001220B467B
:10E058000191029102F05EFE237803F01003DBB217
:10E0680073B1864B197801F00201C9B241B9FF2397
:10E078000093292001220B460191029102F04AFEE9
:10E08800E37813F0010F0ED07C4B197801F00401EE
:10E09800C9B241B9FF2300932A2001220B460191FE
:10E0A800029102F037FEE37803F00203DBB273B1AA
:10E0B800724B197801F00801C9B241B9FF230093E6
:10E0C8002B2001220B460191029102F023FEE378F6
:10E0D80003F00403DBB273B1684B197801F0100147
:10E0E800C9B241B9FF2300932C2001220B460191AC
:10E0F800029102F00FFEE37803F00803DBB273B17C
:10E108005E4B197801F02001C9B241B9FF23009391
:10E118002D2001220B460191029102F0FBFD0FF028
:10E1280075F970B1554B197801F04001C9B241B980
:10E13800FF230093492001220B460191029102F02E
:10E14800E9FDE37803F04003DBB273B14B4B197878
:10E1580001F08001C9B241B9FF2300934E2001228A
:10E168000B460191029102F0D5FD119B444A1978A2
:10E17800444B51B198F80010117032781A70337806
:10E188000BB1542005E0522003E01170327853207F
:10E198001A7003F09BF9119B00241A783A4B1A70F5
:10E1A80098F80030234113F0010F2DD0214605982F
:10E1B80014F00FF80122014628B923B20190009209
:10E1C8000293104605E0002123B2009201910293C8
:10E1D80024200B4602F09EFDBAF1010F05D12B4B0E
:10E1E8008020DA790521013208E0022D07F10102C9
:10E1F80002D18020072101E0802006212346F5F77F
:10E2080001FE2046F5F7C0FA3378234113F0010FD9
:10E2180057D000214FF0010B23B2029302205A4637
:10E228000B46CDF800B0019102F074FDDA45DFF835
:10E2380068900CD119F8243013EA0B0334D1134A2F
:10E248000520D1790093594404EB0B022AE019F810
:10E25800243013F0010327D1022D1FD10C4B1B785A
:10E2680003F02403042B04BF0A4B83F800B00023F7
:10E278000093072014E000BFB0310020971600205B
:10E288004015002041150020B4160020CE180020AB
:10E29800BE160020600E00200815002000930620FE
:10E2A800791C621CF4F728FA11992046F5F794F8BE
:10E2B8002046F5F795FA19F824306FF3000309F8AA
:10E2C80024300134042C7FF46BAF07B0BDE8F08F25
:10E2D8002DE9F04180460E46174646F28B7500241C
:10E2E8003846214613F075FF88B1294608220B48A5
:10E2F80002F0A3FC0948414613F018FF074813F041
:10E308003BFF20B90123A340327813433370013413
:10E318000835042CE4D1BDE8F08100BFAC1600201C
:10E328002DE9F04387B08046894604A847F2B51125
:10E33800082202F082FC002440462146E7B213F08E
:10E3480048FF002843D03846F3F712FF0025661C23
:10E358000246314611202B460095F4F7CDF90123EA
:10E3680021462A460420FF080095F4F7C5F94AF229
:10E37800B340381802F050FC04F00703C1B2194149
:10E3880011F001014FF002024FF001030AD0009290
:10E39800019336B27720294692182B46029602F04E
:10E3A800B9FC14E00092019336B2232004220B46F4
:10E3B800029602F0AFFCB9F1000F08D004A821467C
:10E3C80013F007FF18B10548214613F0ECFE01349D
:10E3D800402CB1D107B0BDE8F08300BF1D15002067
:10E3E8002DE9F74F174698463B7805460C469DF8A9
:10E3F80030909DF834B09DF83820DFF8B4A043B1D0
:10E4080002EA03033B7009789AF800208A18D31AA5
:10E418000370237883B121482146F5F78DF9204907
:10E428001E4813F083FE1D480121FFF779FF1B48A2
:10E4380041462246FFF74CFF1A4B00261E702978EA
:10E4480043F6F72002F0DEFB494646F2C96002F0C7
:10E45800D9FB204639464A46F4F774FF124B394631
:10E468009E7042464B462046CDF800B00195FFF716
:10E47800F1FC2846F7F700FE2B780C480C498AF87F
:10E488000030F5F759F988F800603E7026702E7054
:10E4980003B0BDE8F04F02F029BF00BFB516002059
:10E4A8003815002000190020670E0020981600205B
:10E4B800F614002010B50B4B0B4C024603CB206022
:10E4C80061600A48114613F052FE2146074813F0CE
:10E4D8002DFE064813F050FED0F1010038BF002091
:10E4E80010BD00BF70250020A2160020AC16002029
:10E4F80010B50A4CA37C4BB100200949FAF78AF9F8
:10E50800084B1B78432B01D1433BA374A07C20B953
:10E518000549BDE81040FAF77DB910BDFE17002087
:10E5280035CE0208FC17002014CE0208034B1A78D7
:10E5380001321A7001230370704700BF00190020D0
:10E5480010B50C48FAF70CF90B4A002414700B4A62
:10E558000B4B14700B4ADC7014700B4A9C701470CF
:10E568000A4A14700A4A1470FAF718FA094B1C6020
:10E5780010BD00BF10190020CE180020FD17002084
:10E58800670E0020021900200E19002038180020FC
:10E5980000190020341800202DE9F04F934B944EB9
:10E5A80093F800903368DFF894829C7C914BF022BA
:10E5B8001A7098F800308BB00C2B354647463DD181
:10E5C8008D4B93F803C0BCF1010F02D900208B4991
:10E5D8002FE01AD10024DC70894A8A4B8A498B487B
:10E5E8008B4D04701C7014700C70CDF800C0019431
:10E5F8002D780295FFF7F4FEFAF7D0F985483460D4
:10E608000BB0BDE8F04FFAF7ABB883487E49F5F791
:10E6180093F8824B824A03CB824B10601B7851607F
:10E62800532B57D198F800307F49013388F80030D0
:10E6380000200BB0BDE8F04FFAF7ECB8082B0FD16B
:10E64800784B1B78532B3DD1784B00221A700C2342
:10E6580088F80030764B1A7842F006021A707FE28A
:10E668000D2B37D16F4B1B78532B2BD171496A482F
:10E6780013F05CFD6848FFF71DFF044640B198F8A9
:10E6880000300522013B88F800305B4BDA7067E206
:10E69800082246F2CA61624802F0CFFA6049664829
:10E6A80013F065FD01230093594B01941B785748DB
:10E6B80002935549524A534BFFF792FEFAF76EF907
:10E6C80034604DE2232B40F04B820BB0BDE8F04F95
:10E6D800FFF736BF631E48BFA31DDB10013303FBE2
:10E6E80009F91FFA89F909F5CC46A9F5B649A9F13E
:10E6F8004D094F4BCDF81C901A78CA3612F0010F0D
:10E708004A4C00F01E81474B1A789946432A40F03C
:10E71800C7803B780C2B40F0C3803F48217813F02A
:10E7280058FD002800F0BC803D48217813F051FDC9
:10E73800002840F0B580079920780FFA81FB0BEB91
:10E74800D00002F069FA23784FF0010A03F00702BB
:10E758000AFA02FADFF8E8805FFA8AFA10EA0A0F82
:10E76800C8F8000027D0244B5B78002B40F0988035
:10E77800274BD879F7F7DEFB002800F09180D8F80E
:10E788000010CAF1FF0A20780AEA0101C8F800104F
:10E798000BEBD00002F036FA20780FFA86FB0BEB71
:10E7A800D00002F039FA00EA0A012078C8F800100F
:10E7B8000BEBD0005FE032B202EBD300059202F01F
:10E7C8002BFA10EA0A0FC8F800003BD140EA0A0108
:10E7D800059B2078C8F8001003EBD00002F012FA6D
:10E7E8002178154813F0DFFC5AE000BFC11800205B
:10E7F800341800200D190020670E0020DACE020818
:10E8080002190020FD1700200E19002038180020DA
:10E81800CE18002010190020B51600207025002001
:10E82800EC140020FC170020A0CF0208CB18002011
:10E83800011900202D15002038150020001900208E
:10E84800D8180020924B5B7823B9924BD879F7F708
:10E8580071FBB8B92078DDF814C0CAF1FF0A0CEBD7
:10E86800D00002F0D9F98C4A00EA0A01059B207809
:10E87800116003EBD00002F0C5F92178874813F046
:10E888009DFC0DE020780BEBD00002F0C5F940EAC2
:10E898000A012078C8F800100BEBD00002F0B2F99A
:10E8A80099F80030232B10D12A682378927C013AFA
:10E8B80093420ADA7A4A013313707A4B9B7803F051
:10E8C8000203DBB20BB1F9F7A1FE99F800302A2B4D
:10E8D8000CD1237853B1724A013B1370714B9B786A
:10E8E80003F00203DBB20BB1F9F790FE99F80030A0
:10E8F800552B12D129682278897C694B08398A42BC
:10E9080001DA083200E000221A70664B9B7803F0A7
:10E918000203DBB20BB1F9F779FE99F80030442B0A
:10E928000FD122785E4B072A9CBF2A68927C083A4E
:10E938001A705C4B9B7803F00203DBB20BB1F9F75A
:10E9480065FEFBF7B5FD584A23781178924699423F
:10E9580088BF137012780F32934202DD524A0F3B80
:10E9680013702B684FF0000B93F81280CDF818B095
:10E97800B8F10F0F9ABFC8F120085FFA88F84FF076
:10E98800100839784FFA8BF30C2905D19AF8002032
:10E998009B18DB10454A04E09AF800209B18444A6B
:10E9A800DB10D35C9AF8002005934FFA8BF39A1882
:10E9B8000C2902F007094FEAE20202D13D49895CBD
:10E9C8000691DDF81CC004930FFA8CF0101802F0C1
:10E9D80023F9C0B2049B08909AF8000032B21818C4
:10E9E80002EBE00002F018F939789AF80020049B4D
:10E9F800C0B209919A1846E0059BDDF824C043FA95
:10EA080009F12D4B01F0010100290CBFA521DB21E3
:10EA1800BCF10C0F03F8081014D128494FEAE20C96
:10EA280011F80C1041FA09F111F0010F08D0DDF8C6
:10EA380018C04CFA09F111F0010F03D0582110E069
:10EA48002D210EE0DDF820C04CFA09F111F0010F7C
:10EA580001D0502105E040FA09F111F0010F02D070
:10EA6800542103F8081009F101095FFA89F90BF13B
:10EA7800010B08F101080132B9F1080F5FFA8BFBAD
:10EA88005FFA88F81CD0B8F1200FB5D125E000BF97
:10EA9800670E0020CE180020D81800203815002056
:10EAA800CB18002010190020C31800202D150020B5
:10EAB8008D150020EC140020F4010020B51600206C
:10EAC800B8F1200F09D09AF800304FFA8BF2D2181B
:10EAD8002B689B7C9A42FFF654AF23490B7813F0BE
:10EAE800010F17D02B68214A9B7C12780F2B02F05C
:10EAF800800298BFC3F11003D2B294BFDBB20023E7
:10EB080042B122789AF800101032521A1849CB18DC
:10EB18005F219954174EB37803F00203DBB293B127
:10EB2800F11D652246F661432078F9F7BFFD2B6891
:10EB38009B7C102B02D905200B2101E00020072126
:10EB48003246F9F71FFE2B689B7C102B08D92178D9
:10EB58000948013102220BB0BDE8F04FF9F780BE39
:10EB68000BB0BDE8F08F00BF01190020B0310020C4
:10EB7800F401002010190020F50100202DE9F041D2
:10EB8800002386B08DF81730904B1B78012B00F0CE
:10EB980046828F4C227872B18E4B5B78002B40F006
:10EBA8003E828D4D2B78002B40F0A780F9F7F6FEBA
:10EBB80008232B70A1E0884B19781D46072900F21D
:10EBC8009C8086490978232913D11A70F9F7E6FE43
:10EBD8008349844A0B7853B18348013B0478DBB2FC
:10EBE80044F0060404700B70804951F82330136018
:10EBF800A8E27D4B1A7812F0010F04D101210A43D3
:10EC08008DF817101A70F4F7A9F928B92B781BB9E1
:10EC18000DF11700FFF78AFCF4F7AEF930B92B783D
:10EC2800012B03D10DF11700FFF780FCF4F7B2F9BF
:10EC380030B92B78022B03D10DF11700FFF776FCC2
:10EC4800F4F7B4F930B92B78032B03D10DF1170081
:10EC5800FFF76CFCF4F7B8F948B9F4F7D1F930B913
:10EC68002B78042B03D10DF11700FFF75FFCF4F7A5
:10EC780005FA30B92B78052B03D10DF11700FFF7F2
:10EC880055FCF4F7EFF930B92B78062B03D10DF1C9
:10EC98001700FFF74BFCF4F7A5F930B92B78072BD1
:10ECA80003D10DF11700FFF741FC9DF8173023B38E
:10ECB8002B78072B1FD8DFE803F004070C0F121579
:10ECC800181B00204A4901E04A490020F9F7A2FD33
:10ECD80013E000204849F9E700204849F6E70020FA
:10ECE8004749F3E700204749F0E700204649EDE7A8
:10ECF80000204649EAE7F9F751FE374F3B783D4691
:10ED0800082B40F0C380384B344F1978984611F0DF
:10ED180001013F4E23D113223046F1F73BFB01237B
:10ED2800B3743C4A2378137003B9B374B37C13B13A
:10ED3800394B00221A70FFF7DBFB3648B17CFEF72F
:10ED4800ABFF98F8003003F0FD0343F0010388F8A7
:10ED58000030324B1A7812B13A7000221A703B78A0
:10ED6800002B7FD0FFF7C4FB2A48B17CFEF794FF45
:10ED7800284B1A78984622B100201021244AFEF721
:10ED880029FF2378387898F80040254924EA0302B7
:10ED9800A0F152070A70FFB2224A23EA040E012F9B
:10EDA80082F800E042D854B9BEF1000F07D0012321
:10EDB80000931D4B01941B781648029392E1054B72
:10EDC8000422DA702B7801332B704BE00D190020E8
:10EDD800F6140020670E002000190020FC17002000
:10EDE800EF1800203418002001190020F018002026
:10EDF800C0D302089FD30208E1D3020802D4020854
:10EE080023D4020844D4020865D4020886D4020830
:10EE1800FE17002038180020600E0020C5180020BA
:10EE28000E19002002190020CE180020432819D1FD
:10EE3800C3B97C4C6778AFB97B4BD879F7F77AF8C8
:10EE480038B97A49F9F7E6FC0523E37007332B70E4
:10EE580004E038467649F9F7DDFCE770754A764BE9
:10EE68001A606FE17548FEF705FF737C002B00F010
:10EE78006981734A127802F08002D2B2002A00F047
:10EE88006181704AD31820225A755BE1092B31D170
:10EE98006D4808F09DF8C6B2624C36B3E378042B8F
:10EEA80002D10020694903E0022B04D168490020FF
:10EEB800F9F7B0FC02E00BB90433E37031460222E3
:10EEC8006048F9F7CDFC634B1E78232E00F0A7802D
:10EED8003046F9F75BFD002800F03481312E40F010
:10EEE80031812B7801332B7002E03B7801333B7082
:10EEF800042331E00A2B31D1534808F04FF8C6B249
:10EF0800484C2EB3E378042B02D10020524903E089
:10EF1800022B04D151490020F9F77CFC02E00BB91F
:10EF28000433E370314602224648F9F799FC494B0D
:10EF38001E78232E73D03046F9F728FD002800F0FC
:10EF48000181312E40F0FE802B7801332B7002E0D6
:10EF58003B7801333B700823E370F3E00B2B40F060
:10EF6800F1803948002107F0EFFFC4B2002C4CD0E3
:10EF78002C4FBB783E466BB92B4BD879F6F7DAFFA6
:10EF880010B903233B714AE0BE2013F00FFFBB7892
:10EF98000133BB70F378234A092B02D90020234997
:10EFA80015E010D1204B00241C70D4702C4B2D4A36
:10EFB8002549224801251C7014700C7004700095B6
:10EFC800019402948FE0082B04D127490020F9F717
:10EFD80021FC11E0062B02D100202449F7E7042B7D
:10EFE80002D100202249F2E7022B02D10020214958
:10EFF800EDE70BB90833D370F378082B0BD8114819
:10F0080021460222F9F72CFC05E001230093064B68
:10F0180001941B7862E00F4F3C78232C2CD1FFF72A
:10F028008FFA8FE0670E0020CE180020DACE020893
:10F0380056CE02080049020834180020381800206B
:10F04800B0310020F40100200E1900205ECF020824
:10F058007FCF0208FC1700201CCF02083DCF020812
:10F06800FD1700200219002077CE020898CE02086A
:10F07800B9CE0208FBCE02082046F9F787FC002823
:10F0880060D0303CE4B2631EDBB2012B3C7031D857
:10F09800022C2E4D1DD1E879F6F74CFF002830D010
:10F0A8002B48FFF707FA00282BD1082246F2CA613D
:10F0B800284801F0C2FD2649264813F042F82549A0
:10F0C80046F2CA60082201F0B2FD2348214913F034
:10F0D8004EF801230024009301942B781F482049FF
:10F0E800204A0293204BFFF77BF9F9F757FC1F4B97
:10F0F8001C6027E0032C25D1144BD879F6F71AFFAA
:10F1080010B90C23F3701DE000241148214613F0B8
:10F1180060F828B1E02013F049FE204613F082FE83
:10F128000134402CF1D1124A00231370F3702B786C
:10F13800104A01332B700D4B1A600F4B1A7842F0AE
:10F1480006021A7006B0BDE8F08100BFCE18002094
:10F15800B5160020EC1400203815002038180020BF
:10F168000E19002002190020FD1700203418002075
:10F17800CB18002000490208011900201FB50446D9
:10F1880011B100200B4901E008460B49F9F742FB91
:10F19800217810220139C9B201EB011101F5C241F0
:10F1A8004431684601F049FD102001466A46FEF7E1
:10F1B80011FD1FBDE4A6020826A702080B4B1B7809
:10F1C800442B06D0552B037801D013B17047013B6F
:10F1D80001E003780133037003780BB9203302E0B0
:10F1E800212B01D1203B0370FFF7C8BFFC1700207B
:10F1F8002DE9F74FDFF8C881DFF8D4A198F800307F
:10F20800554643F0010388F800309AF80130624C03
:10F2180023F07F039B46D3B100206049F9F7FAFA3F
:10F228005F482A21F1F734F918B121788222F9F7D9
:10F2380017FB2278002A40F0AB802B6862F3CF33AB
:10F248002B60584B1A7842F003021A70A0E0DFF8DE
:10F258005491237099F800304E4603F00202D2B25E
:10F268000192514F002A40D013F0010813D058469C
:10F278004E49F9F7CFFA3B78232B20D14C4B4D4A16
:10F288004D481A600121FFF779FF337803F0FE0338
:10F298006BF3410312E040464849F9F7BBFA3B7863
:10F2A800232B0CD1424B434A43481A600121FFF7F4
:10F2B80065FF337868F3000368F3410333703B78E4
:10F2C8002A2B65D1337803F0FE036FF341033370C3
:10F2D8002B6843F400432B600F232370364B1878B8
:10F2E80003B0BDE8F04F0DF015BB0DF057FA054619
:10F2F80000282DD001213048FFF760FF3B78532BC1
:10F3080012D13378019A03F0FD0362F300033370DE
:10F31800DAF8003043F40043CAF800300F232370B2
:10F32800254B18780DF0F6FA3B78232B30D133783B
:10F33800002203F0FD036FF3000333701E4B1A70B5
:10F34800F9F72CFB1E4A137843F00603137015E0F7
:10F358001C49F9F75FFA3B78232B19D199F800304B
:10F3680065F3410365F3000389F80030F9F716FBEC
:10F3780098F8003043F0060388F80030124A1378F2
:10F38800013BDBB21370114A52F82320084B1A6074
:10F3980003B0BDE8F08F00BF323A002068A702082A
:10F3A800F401002053330020FC17002089A702082D
:10F3B800341800201C490208CB180020AAA702080C
:10F3C80001190020CBA70208EF180020F018002030
:10F3D800B03100202DE9FF412C4D2D4C2B7843F006
:10F3E80001032B70217801F00401C9B211B9294831
:10F3F800FFF7E4FE284E3378232B21D12378274FBB
:10F4080013F004080AD0224A6FF382031370244BC6
:10F4180020483B600021FFF7B1FE11E0F9F7BEFA82
:10F428002B78204A43F006032B701378013BDBB29C
:10F4380013701D4A52F823303B60164B83F8008046
:10F448003378532B1FD12378052243F0040323700C
:10F45800104B16491C78013CE4B204EB840000F51B
:10F46800CA40843001F0E3FB00201149F9F7D2F9D2
:10F47800FF23002100930134162004220B4601913A
:10F48800029401F047FCBDE8FF8100BF011900208C
:10F4980053330020CB180020FC170020341800201C
:10F4A80038490208EF180020F018002054490208D3
:10F4B80047A702082DE9F041984B04469A7812F0C4
:10F4C800010F00F017811B88002B40F01381944D29
:10F4D80095F820303F2B40F2D780012C14D1914B66
:10F4E8001B7803F00203DBB2002B00F0C48095F810
:10F4F80020208B4B402A03D1013283F82020FBE0E7
:10F50800482283F82020B6E0022C03D1482385F84E
:10F518002030B0E0844E337803F02002D2B28AB1B2
:10F5280095F82020402A0DD1032C0BD07F4B804A20
:10F5380003F1100153F8040B8B4242F8040BF9D184
:10F54800412395E003F01003DBB28BB195F820302E
:10F55800412B0DD1032C0BD0764B754A03F11001CA
:10F5680053F8040B8B4242F8040BF9D142237FE095
:10F57800F37813F0010F0FD095F82020422A0BD111
:10F588006D4B6B4A03F1100153F8040B8B4242F8A0
:10F59800040BF9D143236BE003F00202D2B27AB133
:10F5A80095F82020432A0BD1644B614A03F11001DE
:10F5B80053F8040B8B4242F8040BF9D1442357E06B
:10F5C80003F00402D2B27AB195F82020442A0BD174
:10F5D8005B4B574A03F1100153F8040B8B4242F876
:10F5E800040BF9D1452343E003F00803DBB28BB1E8
:10F5F80095F82030452B0DD1032C0BD0514B4C4A9C
:10F6080003F1100153F8040B8B4242F8040BF9D1B3
:10F6180046232DE00DF0FAFEA0B14B4B1B788BB1C1
:10F6280095F82030462B0DD1032C0BD0474B404A80
:10F6380003F1100153F8040B8B4242F8040BF9D183
:10F64800472315E0F37803F04003DBB29BB195F84C
:10F658002030472B0FD1032C0DD03D4B344A03F1FA
:10F66800100153F8040B8B4242F8040BF9D14823DC
:10F6780085F8203078E095F820300133DBB2472B4D
:10F6880085F820307FF629AF95F82060472E04D9F9
:10F69800234B002683F8206001E00136F6B206F11C
:10F6A8004007FFB212E02B48314612F092FD08B134
:10F6B800032C04D1284B9B5D23B1032C02D185F880
:10F6C80020600FE00136F6B2BE4203D03F2EEAD9E1
:10F6D800402E07D1214B1E221A70402385F8203076
:10F6E800BDE8F08195F820001149652246F661438E
:10F6F800F8F7DCFF012C37D1194B0D4A03F1100143
:10F7080053F8040B8B4242F8040BF9D1044B93F8DD
:10F7180020303F2B3CD9002012493EE01019002030
:10F72800F4010020F7140020B03100201CAE0208BC
:10F73800171900203DAE02085EAE02087FAE02082F
:10F74800A0AE0208C1AE020830350020E2AE0208C1
:10F7580024AF02088D15002043150020CC18002086
:10F768002D0F0308DAAD0208104BD87800F02000FE
:10F77800C0B220B1022C06D000200D490DE0032CA8
:10F7880001D10C4909E00C4B93F820303F2B02D8EB
:10F7980000200A4901E00A490020F9F73BF8102047
:10F7A800084A0146BDE8F041F8F7ECBFB031002047
:10F7B800F5A40208FBAD0208F401002098AD020888
:10F7C80003AF02081019002010B5F9F7E7F8084B45
:10F7D8001B7803F00403DBB22BB106490020BDE817
:10F7E8001040F9F717B80220BDE81040FFF762BED5
:10F7F800F7140020CAAB020870B5224B06461B78E6
:10F80800214CF3B9257819E02048294612F0E1FC8B
:10F8180078B123689D4202D9FF2E02D007E0FF2E5F
:10F8280002D19D4208D202E036B91DB913B925604C
:10F8380012E00EB9013500E0AD19EDB23F2DE3D964
:10F848000AE0013B2021124810222360F0F7A2FDB4
:10F8580000201049F8F7DEFF0F48F8F781FF46F659
:10F86800614320780D496522F8F720FF084D21688B
:10F8780005F1100001310222F8F7F2FF2D23AB74D5
:10F8880070BD00BFC1180020D81800203A18002009
:10F89800F4010020A9ED0208101900201719002012
:10F8A800F8B5544BF02254481A700378044613F004
:10F8B8000E0518D1514A43F00203156000F8013BC8
:10F8C80012F02CFC2C464E4BE35C1BB14D482146F4
:10F8D80012F069FC0134402CF5D14B4B1A7842F0F8
:10F8E80001021A70F8BD13F00C0543D12E464548A5
:10F8F800294612F06EFC08B10136F6B20135402DEA
:10F90800F5D11EB9237843F0040331E000253F48C0
:10F918002946EFB212F05DFC68B1394BEB5C53B18C
:10F928003B4B01371F700020FFF766FF237843F039
:10F938000803237002E00135402DE8D1354D3A2106
:10F948002846F0F7A5FD38B1401BC0B20130281891
:10F9580031460222F8F784FF2F4B1B78532B47D1EF
:10F968002B4B00201870FFF747FF237843F008035C
:10F978002370F8BD6FF34103037003F00403DBB297
:10F98800254D23B100202549F8F744FF0EE02B78D8
:10F99800552B01D1FF2002E0442B02D10120FFF7B3
:10F9A8002BFF13200D211E4AF8F7ECFE2B78232B92
:10F9B8001ED1227802F00204D4B90F4902F0FB02EA
:10F9C80064F3C3020A700D4A1460F8F7E7FF0E4BA0
:10F9D8001A7842F006021A70124A1378013BDBB219
:10F9E8001370114A52F82320104B1A60084B1C70F0
:10F9F800F8BD00BF0D19002039180020D8180020C4
:10FA0800E02300203A18002001190020F8140020F3
:10FA1800C1180020F4010020FC170020EFFE0208A6
:10FA280010190020EF180020F018002034180020CA
:10FA380070B505460C4616463BB143004AF28D3078
:10FA480018184018114601F0DDF8054B172202FB83
:10FA58000535F3092C1906F07F066370E67070BD52
:10FA68007D32002038B510B3A0F14103DBB2432B3F
:10FA78001FD9C50900F07F040BD0052C19D9002126
:10FA8800601E0A460AF0C6FAD0F1010038BF00200D
:10FA980038BD082C0FD9601EC0B229462A4609F085
:10FAA80023FF50B9202C8CBF0020012038BD012035
:10FAB80038BD002038BD284638BD284638BD00006E
:10FAC800F7B5614C31232374604F01332376053B2E
:10FAD800637463763B784AF28D305B00181801F046
:10FAE8009BF8C0B220F07F0200F07F01D2B28DF8FF
:10FAF80004108DF8002004F1120359B9544A04F196
:10FB080015001188927861829A7020210222F0F7FC
:10FB180041FC0CE0D20904EB8202526A1088608230
:10FB2800927804F115009A700222F8F799FE387855
:10FB3800400000F5224000F5C77001F06DF8C0B232
:10FB480020F07F0300F07F01DBB28DF805108DF8FF
:10FB58000130404851B93E4B20311A889B78628366
:10FB6800837002220330F0F715FC0BE0DB0904EB8D
:10FB780083035B6A1A8862839B780222837003304E
:10FB8800F8F76EFE344B1B7813F0010F5AD0334D43
:10FB980002A92A788B1813F8041C13F8086C304B48
:10FBA8001B78232B04D1002A41D1223B2B703EE045
:10FBB8002A2B04D1002A3AD0013A2A7037E0552B73
:10FBC80046EA010611D10DE02B7802AAD318013EAE
:10FBD80013F8081CF6B23046C90913F8042CFFF7CD
:10FBE80041FF98B9002EEFD121E0442B19D115E03F
:10FBF8002B7802A9CB18013613F8081CF6B2304648
:10FC0800C90913F8042CFFF72DFF38B1134B3878C6
:10FC1800197832460123FFF70BFF08E0872EE7D952
:10FC280005E0532B03D1533B2B70FAF741FC0D4BE6
:10FC38001B7803F08003DBB223B12B782022023338
:10FC480004F83320FEBD00BFF4010020C1180020D5
:10FC5800EC0A03080E02002001190020CB1800202E
:10FC6800FC170020B0310020024800210922F0F7DB
:10FC780091BB00BFDD18002070B50A46002405E0DE
:10FC88001B19811A2A2501345D54E4B20E4D0F4B1D
:10FC9800295D09B19442F3D1801A0019181820215E
:10FCA800121BF0F777FB0A4B1E785EB1432E04D186
:10FCB8000CB1013CE4B200232B553046F8F766FE40
:10FCC80000B12E5570BD00BFDD180020F4010020E2
:10FCD800FC17002038B5184C184DA07800F010001B
:10FCE800C0B250B91649F8F795FDFFF7BDFF236874
:10FCF80043F4801323600F232B702A782AB92368D2
:10FD0800FF2062F31453236038BD0E48C5792DB91E
:10FD18001C200821FFF7B0FF284638BD23680A4990
:10FD28006FF3145308222360F0F7B4FD00280CBFCA
:10FD38000120FF2038BD00BFB03100200F1900207E
:10FD48002DAC0208DD1800202A2A0308F0B55B4C08
:10FD580085B0667806F01006F6B2002E3ED1584BF4
:10FD68001A78584B013A53F82230574A934204D133
:10FD7800564B1A7842F0020207E002F11C018B424E
:10FD880008D1524B1A7842F00402022161F3C702EB
:10FD98001A7019E03832934216D1FFF79BFF0028FA
:10FDA80000F08A800128494D06D12B78022243F0C1
:10FDB800010362F3C70306E030464549F8F72AFD18
:10FDC8002B7866F3C7032B70424B1A7842F0010276
:10FDD8001A70236843F4805323606DE03B4D2B7801
:10FDE80013F0F80606D03C49002005B0BDE8F04005
:10FDF800F8F710BD13F0070F3FD003F00202D7B297
:10FE08004FB1122031460EF06BFCFF230093019690
:10FE18000296432028E003F00406F6B296B139466C
:10FE280038460EF05DFC0DF0C3FE09F087FB0CF0C0
:10FE3800DDFCFF23009301970297442039460422F2
:10FE48003B4614E013F0010F13D0012143F61C6068
:10FE58000EF046FC3046F6F7D7F8204B45201E80BA
:10FE6800FF2300930196029631460422334600F0A0
:10FE780051FF00201A49F8F7CDFC2B7803F0FA035C
:10FE88006FF341032B70174B1B78232B14D1236876
:10FE98006FF30C332360F8F781FD0E4B1A7842F0AC
:10FEA80006021A70064A1378013BDBB21370054A42
:10FEB80052F823200C4B1A6005B0F0BDB031002079
:10FEC800EF180020F01800205C490208B537002020
:10FED8004EAC0208011900208B02030812180020FA
:10FEE8006A020308FC170020341800201FB50446D6
:10FEF800F6F776F9A8B14B2001F0E8FAFF23009352
:10FF08000121FF3B0193392004220B46013402945E
:10FF180000F000FF064B01205A7842F004025A70A4
:10FF280004E0044B1888003818BF012004B010BD45
:10FF380040330020483A0020F0B51E4E0024337AA2
:10FF48000546013385B00F46337210202146012241
:10FF580023460094F2F7D0FB45B9FF23009301959F
:10FF680002974F20294604222B4609E0012D09D18A
:10FF7800FF23009301940297502021460422234630
:10FF880000F0C8FE337A052B11D1FA330121002481
:10FF9800009327200B4604220194029400F0BAFE35
:10FFA800044B1C7205B0BDE8F04001F061BA05B021
:10FFB800F0BD00BFCE1800202DE9F04F974B87B059
:10FFC8001A78804699461AB1012A40F0E08130E05B
:10FFD800934B1A68934B9A4200F0DB81F5F77AFD50
:10FFE800914B5B7803F00203DBB253B98F4B5B781C
:08FFF80003F08003DBB223B922
:020000040801F1
:1000000001F060FA08B909F09DFA8B4B1A686FF39A
:1000100010421A60894B1878F8F7BCFC002800F0F1
:10002000BC81FFF725FE864B3C221A70F8F7FEFADA
:1000300099F80030013389F80030814B1C787CB985
:10004000804B08F101011A78204664F3C30264F37F
:1000500004121A70C9B2FFF773FF89F800409CE1DF
:10006000794D404609F08EFAF8F7D4FA0020774926
:10007000F8F7D4FB764F2B78AA46FB1813F8313CDF
:1000800023B91B200621FFF7FBFD86E16D4A0B21FA
:10009000137804A8C3F3C004C3F3001603F0F703F6
:1000A0006FF304131370002389F80030062200F068
:1000B000C8FD2A78394604A8303AF0F795F8074683
:1000C00020B100274FF012093D4629E049F23F6078
:1000D00000F0A6FD0028F4D05E4D2F72F5F75EFE0D
:1000E0000446002840F059815B4A4F4B21461A6074
:1000F000FF2300930190029004220820234600F081
:100100000DFE012223460E2021460094F2F7F8FA54
:10011000524B1A7842F004021A700123AB713CE191
:100120004946062204A800F08CFD9AF8002004A895
:100130004749303AF0F758F8002840F01D8128462A
:10014000FFF7D8FE002840F02881DFF808B1012130
:100150008BF808002846F5F72FFE8146F5F71EFEBE
:10016000DA46002840F0B18048463D49F0F71AFAD7
:10017000B0B901F0BFF82C4B14B916B9394A23E0D5
:1001800036B1394A1A60394B1A786FF3410205E0EB
:10019000374A1A60354B1A7866F341021A70D3E079
:1001A00048463449F0F7FEF920B148463249F0F7A5
:1001B000F9F958B9002C40F0F080002E40F0ED80A5
:1001C00001F098F82D4A184B1A60BDE048462C49BA
:1001D000F0F7E8F950B949F23D60012100F016FD51
:1001E000154A136843F400531360E3E74846254972
:1001F000F0F7D8F938B9002C40F0CF80002E40F04D
:10020000CC80214ADFE748462049F0F7CBF90028A7
:1002100040D1002C40F0C180002E40F0BE801C4A2E
:10022000D1E700BF3018002034180020B049020880
:100230009A2B00204F330020B0310020FC17002003
:100240000F190020DC18002018180020D4A4020880
:10025000DD180020CE180020CC490208192100200A
:10026000A12B0308184C0208A04D02080119002018
:10027000BC4D0208312B0308772D0308D84D020826
:100280006C2B03086E2B0308104E0208342D030854
:10029000644E020848464249F0F784F9002853D1D9
:1002A00001F028F83CB13F4A3F4B1A603F4B1A78A7
:1002B0006FF3410270E0002E6FD03D4A3A4B1A6056
:1002C0003A4B1A7864F3410266E048463449F0F745
:1002D00069F9064620B901F00DF8002C5DD01BE04D
:1002E00048463449F0F75EF9002856D0484632496E
:1002F000F0F758F938B9002C4FD1304A2A4B8BF817
:1003000007501A6049E048462D49F0F74BF9064678
:1003100050B9A4B100F0EEFF224A234B1A60234BE0
:100320001A7866F3410237E048462649F0F73AF971
:1003300020B148462449F0F735F900B96CBB234A8F
:10034000194B1A6000F0D6FF07F56A5078308AF82A
:10035000075000F065FC8AF800009AF8070000F5E5
:10036000D640353000F05CFC8AF801001848F5F7FB
:1003700067FE202D11D107E00135EDB20137202DA8
:1003800009F107097FF4CCAE08F101010020C9B2E0
:10039000FFF7D6FD01E000221A7007B0BDE8F08F2C
:1003A000702B0308BC4D02083418002001190020EE
:1003B000A04D02086E2B0308342D0308644E02087A
:1003C000A12B0308312B03086C2B0308804E020875
:1003D000CE18002010B52148214903680A789C7B7B
:1003E000944203D99C8914F0200F18D09A8912F0F6
:1003F000800F01D105E01C3B9A8912F0400FFAD022
:1004000000E01C33036000230B7003689B8913F02A
:10041000200F16D0134BDA79114B1A7011E001320C
:10042000D2B20A70986843F60553984209D101E0A8
:100430000132D2B2162A03D80B4853B29840F7D4EF
:100440000A700A4A136843F480731360F8F7EEF8F1
:10045000074B1A7842F006021A7010BD34180020BB
:10046000C1180020CE18002000060088B0310020FE
:100470000119002010B52349234A0B78D3B1106825
:10048000848914F0200F15D1013BDBB20B70846816
:1004900043F60552944228D104E013B1013BDBB28C
:1004A00000E0837B162B03D8184C5AB29440F4D446
:1004B0000B701AE01368988910F0400F01D106E024
:1004C0001C33988910F0800FFAD0136002E00E48B8
:1004D0001C3B036013689A7B0A709B8913F0200F02
:1004E00003D00B4BDA79074B1A700A4A136843F4AE
:1004F00080731360F8F79AF8074B1A7842F00602F7
:100500001A7010BDC11800203418002000060088A1
:10051000CE180020B031002001190020084B1A68C5
:10052000084B9A4204D003F580630C339A4205D1FC
:10053000054B1878003818BF01207047002070471D
:1005400034180020B0490208F6140020074B084A6E
:100550001B68934202D03832934205D1054B18787C
:10056000003818BF01207047002070473418002061
:10057000644E0208F61400202DE9F04F7F4B804DA9
:100580001970A0F11103DBB2012B87B00E46287061
:1005900006D8122801D1113800E00020F5F796FDA9
:1005A0002B78522B0DD1F2F7B9FD28B9F2F7AAFD3D
:1005B00010B9F2F7CBFD20B1724B1A7842F0080265
:1005C0001A70714B714C1B78002B2DD12168704A29
:1005D000914229D06F4A236013706F4A6F48117897
:1005E000037063F3C30163F3000163F30711117038
:1005F0006B4A117863F3010111706A4A117863F351
:10060000C5011170684A1370684A117863F341019B
:1006100063F3000163F382011170654A116863F3AB
:100620000C311160634A13702368002B40F056812F
:100630005F4F7B7803F02003DBB273B15E4B93F81E
:100640000080B8F1000F08D149F23D60414600F04A
:10065000DDFA3B6868F34D333B60584B187810F077
:100660001E0002D00020564907E0564B93F8048044
:100670009946B8F1000F05D0534907B0BDE8F04FD7
:10068000F8F7CCB8514F97F801B0BA46BBF1000F5C
:100690002DD0BBF1070F15D94D48F8F765F84D4936
:1006A000B878652246F66153F8F704F838780723DE
:1006B00010F003007B700EBF474940464749F8F7EA
:1006C000ADF80CE0BBF1020F09D84148437823B1E3
:1006D000F8F74AF887F8018078E202237B7010204F
:1006E0003B4A014607B0BDE8F04FF8F74FB83C4F22
:1006F000BB795BB187F806B000F0F4FB8E20594659
:1007000001225B46CDF800B0F1F7FAFF0020F2F7C6
:1007100059FE214A1F491378324843F006031370EB
:1007200000230B70304923600B7089F8013003708F
:10073000173303FB06FC2D49934611F80CC088467D
:100740001CF0080F04D130460593FFF739FC059BD8
:1007500003FB06835B7913F0100F04D02A78133A59
:10076000D2B2032A46D913F0200F79D02B78442B2C
:1007700040D03DD8232B3DD02A2B3AE0C41800208E
:10078000FC170020351500200D190020341800201A
:1007900000490208EF18002001190020CB180020A2
:1007A00015180020C6180020CD180020DC180020E5
:1007B000B03100200C190020F6140020313A00203E
:1007C00037A50208670E0020C8D40208C818002008
:1007D00010190020171900203FA602081EA60208C3
:1007E000CE180020C5180020C11800207D3200203E
:1007F000552B35D1794B1B78002B31D1784B93F8A1
:100800000080B8F1000F2BD143F6DB2000F008FA8E
:10081000012825D11F23FB7189F8010043F6173009
:1008200000F0FEF93870F87900F5D640353000F068
:10083000F7F978706B48F5F703FC9BF80030304609
:1008400068F341038BF8003008F09CFEF8F7AAF833
:10085000654B66482360664BC3F800802B780370B5
:100860002B78432B0AD15E4B1B783BB9013389F8B7
:100870000130604B3046236008F084FE287817383A
:10088000C3B2072B00F2A2815B49FF220AF062FB90
:100890009AF80010594B60F301018AF8001001F03A
:1008A0000301022900F092810122032041B100904E
:1008B00001929B7868309B1802930021033206E076
:1008C000009001929B786C200133029304220B4626
:1008D00000F024FAFF238AF8013077E1454A934279
:1008E00050D12878A0F14303DAB2122A22D8444A20
:1008F0005BB29A401ED5432840F06881374B1B7885
:10090000002B40F0638100F0FFFC3E4B48B11A78A9
:1009100003201109013191FBF0F000EB4000091AAE
:1009200004E01A781109013101F0070161F307129F
:100930001A704BE1F8F72EF8002823D0314F3A789F
:1009400012F0F00308D163F307123A7023602E4BC4
:100950001A7842F008020EE0102B13D100F0D4FCFC
:1009600080B13B786FF307133B7000232360264B65
:100970001A7842F0100230461A7007B0BDE8F04F06
:10098000FFF71EBB214B1E211A781E4E61F3460253
:100990001A70337813F0010F134B3DD022689A423E
:1009A0000CD0A3F5B0639A4208D0FFF7B7FD28B981
:1009B000FFF7CCFD10B9AA30F2F704FD2268144B02
:1009C0009A4202D10020F2F7FDFC2B78522B40F026
:1009D000C280104B53221A70BDE000BFF6140020F5
:1009E00030180020CE180020804E0208C5180020C4
:1009F000F0180020B0490208CA180020C8180020CA
:100A0000002000C001190020DC1800207E19002001
:100A1000B84E0208FC17002022689A420CD0A3F5B9
:100A2000B0639A4208D0FFF779FD28B9FFF78EFD31
:100A300010B9AA30F2F7C6FC2B78552B1ED1FFF760
:100A400019FD3378634843F0060333708378624FAF
:100A500003F00203DBB24BB1F7F786FE2368186898
:100A6000FBF7A8FD3B786FF341033B705B4883784D
:100A700003F00203DBB20BB1F7F776FE2B78442BC1
:100A80001ED1FFF7A7FC3378524843F006033370BA
:100A90008378514F03F00203DBB24BB1F7F764FEEA
:100AA00023681868FBF786FD3B786FF341033B70C2
:100AB0004A48837803F00203DBB20BB1F7F754FE28
:100AC0002B78522B09D13378002243F00103337085
:100AD000434B1A70434B45321A70434B00271F702B
:100AE0002B78232B37D1414B3A481F70404B1F7056
:100AF000F7F73AFE3948F7F737FE33783D4943F0C8
:100B0000060333700B78344AFBB13B4A013B177044
:100B10003A4ADBB20B7052F82330394A23609B68A3
:100B2000934202D109F0BEFC15E002F59A718B42A6
:100B300004D10120014606F0F9FE0CE002F5E07256
:100B4000934208D12F4B1F7005E0117863F3071112
:100B5000117023603AE02C4B5B7813B10020F2F760
:100B600031FC23681F7B17F00F0702D1FCF706FF4B
:100B70001BE0012F02D1F9F751FE16E0022F02D13E
:100B8000FAF7CCFD11E0082F05D84FF09C53BB407D
:100B900001D5FBF789F8042F03D123689B69984797
:100BA00003E0052F01D1FAF737FB337803F0020396
:100BB000DBB21BB123681868FBF7FCFC33786FF3DA
:100BC000410333702B780BB1074A137007B0BDE8AF
:100BD000F08F00BF101900200119002044180020D8
:100BE000CB180020FC17002016180020CD1800207C
:100BF0000C190020EF180020C1180020F018002068
:100C0000D44E020843180020670E002007B502AB3F
:100C100003F8011D19460122002305F005FB0EBD56
:100C200007B5002302A901F8013D012205F064FB8C
:100C30009DF807000EBD08B5002305F0F5FA002069
:100C400008BD034610B508461446194605F054FB86
:100C5000E0B210BD10B5034600248454084619467E
:100C600005F04AFB204610BD37B50546002400E0DC
:100C70001446012260190DF1070105F03DFB9DF8B6
:100C80000730621C203BDBB25A2BF1D920463EBD17
:100C9000F8B500252C461E4B1C21585D01FB043184
:100CA000400000F574506230043102220134FFF735
:100CB000C2FF1C355C2CEED14FF46F5420B20422DD
:100CC00005341449FFF7B7FFA4B243F6D4339C426E
:100CD000F4D1002548F63C472C4615E007EB4600CA
:100CE00004EB440100B259180222FFF7A4FF0136B9
:100CF000F6B2094B5A199278B242EFD801348037D4
:100D00000335142CBFB201D00026F2E7F8BD00BFB6
:100D100040790208332B0308508302082DE9F3477A
:100D2000044615468A46022243F61A610DF1060072
:100D30001E46BDF930909DF828809DF82C70FFF775
:100D400080FF2F4B2F499A78BDF906008A705A7898
:100D500000EBC000CA701A7900F578500A715A7910
:100D60001C304A719A791B7845EAC6158A710C7055
:100D700081F80190CB710D7200B20922FFF75BFF81
:100D80001EB1214B1A8801321A80BDF8063001339A
:100D90009BB2B3F57A7FADF8063002D30023ADF8ED
:100DA000063002220DF1060143F61A60FFF743FFF9
:100DB000BDF80600154B188000B200EBC00000F52E
:100DC000785000F11C05243000B2FFF729FF10F025
:100DD000800F03D00C4B1A88013A1A8028B20021E8
:100DE000FFF714FF0A4B03F8148003EB4404677009
:100DF000BAF1000F02D00120F5F70AF9BDE8FC872F
:100E0000BC370020E618002012180020982B002084
:100E1000332900202DE9F743314B1D78303DEDB2E9
:100E2000C5F10606F6B23EB305F11207202413E021
:100E300008F101080FFA89F000215FFA88F8FFF73E
:100E4000E5FE09F10109B0451FFA89F9F0D1013C2D
:100E50000737E4B2BFB21CB1B9464FF00008E7E76C
:100E60000B35013428B20021E4B20135FFF7CEFE84
:100E7000B442ADB2F5D131E0122425B2684629461C
:100E80000622FFF7DEFE9DF8003043B19DF80530E5
:100E90002BB99DF803308DF804308DF805300734F8
:100EA000062228466946A4B2FFF7C5FEF22CE4D11B
:100EB00068460B210622FFF7C4FE9DF8003043B1BF
:100EC0009DF805302BB99DF803308DF804308DF86E
:100ED00005300B2069460622FFF7ADFEBDE8FE8314
:100EE0001818002070B509F0DDFA0BF02BFD05F0A5
:100EF00039FF05F05FFEF2F7C5FCA648F5F7BAF832
:100F000043F6D120FFF78CFEA34BA44C187043F698
:100F1000D020FFF785FEA24B187043F6DC20FFF7C8
:100F20007FFEA04B187043F60350FFF779FE9E4BEF
:100F3000187043F60450FFF773FE9C4B187043F68D
:100F4000DA20FFF76DFE9A4B187043F6D920FFF7B1
:100F500067FE984B187043F6CF20FFF761FE964B63
:100F6000187043F6CC20FFF75BFE944B187043F6E5
:100F7000D220FFF755FE924B187043F6DF20FFF7A3
:100F80004FFE904B187043F6E820FFF749FE8E4B5A
:100F9000187043F6DD20FFF743FE237801280CBFCD
:100FA00043F001036FF30003237043F6E020FFF7E3
:100FB00037FE237801280CBF43F080036FF3C7137B
:100FC000237043F6E720FFF72BFE804B01281A68B9
:100FD00043F6ED200CBF42F000526FF35D721A60D1
:100FE000FFF71EFE7A4B18B91A7860F3000202E090
:100FF0001A7842F001021A7043F6EA20FFF710FE59
:10100000637801280CBF43F001036FF300036370A2
:10101000704843F66E210822FFF713FE6E4B002442
:101020001C705C706B48235C312B03D1103021465F
:1010300011F0BDF80134082CF4D1224643F6F61124
:101040006448FFF7FEFD224643F63A216348FFF766
:10105000F8FD47F2D71104226148FFF7F2FD47F28D
:10106000DB1104225F48FFF7ECFD0DF021F8F5F7E6
:1010700009FB43F6E120FFF7D3FD5B4C237860F3D7
:101080000003237043F6E220FFF7CAFD237860F3E4
:101090004103237043F6E420FFF7C2FD237860F399
:1010A000C303237043F6E620FFF7BAFD237860F30D
:1010B0004513237043F6E920FFF7B2FD237860F370
:1010C0008613237043F6E520FFF7AAFD237860F32B
:1010D0000413237043F6EB20FFF7A2FD237860F39F
:1010E000C713237043F6E320FFF79AFD237860F3DC
:1010F000820323703D48FFF793FD3D4B3D49052298
:1011000018703D48FFF79DFD3C48FFF789FD3C4BBB
:1011100018703C48FFF784FD3B4B18703B48FFF7C5
:101120007FFD3B4B18703B48FFF77AFD3A4B187038
:101130003A48FFF775FD3A4B18703A48FFF770FDD3
:10114000394B18703948FFF76BFD394B1870FFF7B2
:1011500061FE3848FFF764FD374B18703748FFF7DA
:101160005FFD374B18703748FFF75AFD364B187044
:101170003648FFF755FD364B18703648FFF750FDDF
:10118000354B18703548FFF74BFD354B002869D1BA
:10119000187069E02C180020620E00207E190020D3
:1011A000610E0020640E002069140020D61000207B
:1011B0004A3A002000000020AA160020171800203C
:1011C000630E002043320020F9310020B0310020AE
:1011D00018290020DD320020ED320020E532002009
:1011E000C0310020D831002097160020328CFFFF3C
:1011F00030350020AEA4FFFF98120020358CFFFF91
:101200002E350020368CFFFF61340020388CFFFF24
:10121000D5330020398CFFFFAC1A00204096FFFF29
:10122000311700209EA3FFFFB21700203E96FFFF5C
:10123000181800208AA3FFFF9831002007A3FFFFA2
:10124000902B002004A3FFFF292A002006A3FFFF04
:10125000972B002005A3FFFF912B00203A8CFFFF66
:10126000FA17002001221A704AF28D35002428B2A4
:10127000FFF7D6FC002102460B462046FEF7DCFBBA
:10128000681C00B2FFF7CCFC012102460023204677
:1012900001340235FEF7D0FB042CADB2E7D10E4885
:1012A000FFF7BEFC0D4B18700D48FFF7B9FC0D4B56
:1012B00001281A780C480CBF42F020026FF3451247
:1012C0001A70FFF7ADFC094B18700948FFF7A8FC2E
:1012D000BDE8704010F0DEB9EA8BFFFF4E3300200E
:1012E00020A4FFFF68400020E98BFFFF542100206D
:1012F000ADA4FFFF034B1E211A7861F346021A705A
:10130000704700BF7E190020024B187800F00100E2
:10131000704700BF7E190020014B1878C009704744
:101320007E19002008B5FFF7F7FF38B9044B1B788A
:1013300013F07E0F0CBF0020012008BD012008BD66
:101340007E190020F8B547F2CD042046FFF768FC6F
:101350002D2803DD20462D21FFF758FCA4F55C560F
:10136000353E3046FFF75CFC414FC0B207EBC00092
:101370000579C5F30015A5B90DE03D4B3D4953F87E
:101380003500EFF70FF920B930462946FFF73EFC4C
:1013900007E00135EDB207EBC5031B7913F0080F29
:1013A000EBD0013447F20D139C42CED143F6C42456
:1013B0002046FFF735FC2D2803DD20462D21FFF7C1
:1013C00025FC013443F6C8239C42F1D1012143F6A8
:1013D000E120FFF71BFC012143F6E220FFF716FC9A
:1013E000012143F6E420FFF711FC012143F6E6203A
:1013F000FFF70CFC012143F6E920FFF707FC012170
:1014000043F6E520FFF702FC012143F6E320FFF756
:10141000FDFB012143F6EB20FFF7F8FB002143F62B
:10142000E020FFF7F3FB002143F6EA20FFF7EEFB95
:10143000002143F6EC20FFF7E9FB012143F6DC2015
:10144000FFF7E4FB002149F23F60FFF7DFFB48F6BE
:10145000A8300121FFF7DAFB47F2B5142046FF213F
:10146000FFF7D4FB013447F2BD139C42F6D1F8BD1F
:1014700014040020E30D030810B508F043F80BF046
:1014800025FA074B4FF416721A80012147F2C51056
:10149000FFF7BCFB4C20BDE8104000F01BB800BFBC
:1014A000483A002010B508F04DF80BF0A3F9044BB2
:1014B000002147F2C5101980BDE81040FFF7A6BB18
:1014C000483A0020024B1888003818BF01207047A6
:1014D000483A0020542873B5044663D83D4BDB7866
:1014E00003F02003DBB2002B72D13F2801D811F0AA
:1014F00089FC394D35F81460002E69D1E10001F501
:10150000DA416846D5310822FFF79BFB3348214674
:1015100010F063FE50B1F3B2072B07D03F2C05D873
:101520000122B240D243D2B22D4B27E01DF8063043
:101530000122542B08D0562B03D0532B284B1AD101
:1015400000E0284BB24007E0B240254BD2B2195D13
:1015500042EA01011955234B195D0A431A55FFF759
:10156000D3FE98B1204B1B7883B13F2C0ED81E338D
:1015700025F814300AE0B240D243D2B2195D02EA33
:1015800001011955174B195D0A401A550136082EED
:10159000BCD1134B1A5D134B1B5D134318D125F8B7
:1015A000143015E0C10001F5DA416846D531082252
:1015B000FFF747FB00231DF803202D2A05D001214A
:1015C0009940074A105D014311550133082BF2D1B0
:1015D0007CBD00BFB03100208219002068250020AA
:1015E0004E1E0020A91C0020281700201FB501F066
:1015F00015F910B901F026F948B10021FF23009335
:101600000B2004220B4601910291FFF787FBAD22CC
:101610000023D9B24D2909D0012A07D90D4800214C
:1016200019540D4819540D4820F813100133013294
:10163000552BD2B2EDD1074B002183F85510084B42
:1016400008481970084B0822197005B05DF804EBC2
:10165000EEF7A4BE4E1E0020A91C00208219002017
:101660000D1B0020EC1A00208019002059B1064BF8
:101670000C2202FB0030437AC918837A4172083089
:101680000BB93C3383707047B4250020072813B58D
:10169000044624D9124B1B5C022B20D10DF107010B
:1016A0000DF1060208F024F958B19DF8061001204A
:1016B00010FA01F19DF807300A4AD05C0143D15479
:1016C0000DE0083CE4B2E308012104F0070411FA3C
:1016D00004F4054A0133D15C41EA0404D4541CBD2E
:1016E000E02300201432002010320020044B0C2292
:1016F00002FB00330C3A5A729A72FFF7C7BF00BF61
:10170000B425002010B50446FFF7F0FF034B0C2270
:1017100002FB0434FF23637210BD00BFB425002018
:1017200070B5104D002410482146E6B210F055FD6A
:1017300098B96B7A8BB10D4AA318A25C93F88030EC
:10174000022A0AD0413BDAB2122A06D8084A5BB212
:101750009A4002D53046FFF7C9FF01340C35402CC2
:10176000E1D170BDB425002098160020E0230020B0
:101770000020008810B50A4B0C2203EBD00393F82D
:101780008011084B02FB00331C7A3CB900F00700C3
:1017900051FA00F010F0010F18BF1A7210BD00BF0F
:1017A000E0230020B4250020044B0C2202FB003370
:1017B0001A7AFF2A01D1FF3A1A727047B425002025
:1017C000104B1B7813F0010F02D10F4B187818B192
:1017D0000E4B03F540720CE00C4B03F54072197A86
:1017E0000C330139C9B2FD2998BF01209342F6D1CB
:1017F0007047197A09B1FF2119720C339342F8D15D
:1018000000207047BE16002028170020B4250020B5
:1018100030B504461048007800F00200C0B2C8B1EC
:101820000C2060430D4D285C904201D1994207D0B5
:10183000984201D1914203D0052A0BD1052B09D141
:101840000C2303FB0455064821462B72BDE83040AB
:1018500010F0B8BC30BD00BF39180020B4250020FE
:101860003A1800201FB504462146144810F0B5FC74
:10187000002821D00122022300210093A318029303
:101880005C200B460192FFF749FA21460B4810F005
:1018900099FC21460A4810F095FC2146094810F0B1
:1018A00086FC074BE40804F5CC40195DCA3004B04F
:1018B000BDE81040FFF7AAB904B010BD1D15002007
:1018C000381500209816002010B50D4C0021082274
:1018D0002046EEF763FD43F6F120FFF7A1F92071F2
:1018E00043F6F220FFF79CF943F6F42160710222DF
:1018F0002046FFF7A6F9A37943F00203A37110BDB8
:101900002C1A00200A4B1B781D2B0A4B0BD89A79F6
:1019100012F0010F03D05A880AB1013A5A809A791D
:101920006FF3000202E09A7942F001029A71704767
:10193000BC3700202C1A00202DE9F0436F4885B0F9
:1019400010F0F0FBDFF8D0816D4E0024E5B22846A0
:1019500005F0A6FA18F8019F074618F8403C13B1A5
:10196000022B3ED10FE02846FFF7C0FE2146654816
:1019700010F028FC2146644810F024FC21466348FE
:1019800010F020FCDAE028464946F3F7B7FE10B124
:101990002846FFF79FFD737AFF2B01D1FF3B73723F
:1019A000737A4B4501D2F37A9BB15448214610F02B
:1019B000FEFBF37A002B40F0C180204605F0BCFD11
:1019C000052128460A460B46FFF722FF2846FFF767
:1019D0008DFEF37A002B40F0B1802846FFF742FFDE
:1019E000ACE090B92846FFF781FE2146434810F04D
:1019F000DEFB28463946F2F72FFA002800F09780E0
:101A00003378002B00F093803AE0022814D13B4851
:101A1000214610F0CCFB3378012B01D0737A1BB92F
:101A200028460121FFF722FE28464946F3F766FEC5
:101A300000287CD0284626E003280FD12846FFF74F
:101A400055FE21462D4810F0B2FB28460121F2F741
:101A500003FA00286BD03378032B10E0042815D14B
:101A60002846FFF743FE2146244810F0A0FB2846F5
:101A70000221F2F7F1F9002859D03378042B56D01F
:101A8000052B54D04520FFF725FD50E001284ED10D
:101A9000737A4B4502D32846FFF728FE21461948A2
:101AA00010F090FB2146184810F08CFB2146174897
:101AB00010F088FB2846FFF777FE3378012B36D0ED
:101AC000052B34D02846FFF7CDFE33780BB1032B1E
:101AD00007D10F48214610F080FB40B3204601217A
:101AE00008E0042B1AD10B48214610F076FBF0B128
:101AF00020460221F0F700FF19E000BF461E00203B
:101B0000B4250020C4230020CC230020D4230020AF
:101B1000F8140020201700201F24002036482146FA
:101B200010F05BFB18B120460021F0F717FF2846A4
:101B3000394601220223FFF76BFE377021462F48FA
:101B400010F04BFB013401462846F4F723FA0C361B
:101B5000402C7FF4FBAE0CF05FF843F6F220FFF769
:101B60005FF8274EC0B27578264C854224D143F6E3
:101B7000F120FFF755F8B378C0B283421CD16279E7
:101B8000AA4213D122799A4210D1A37903F0040317
:101B9000DBB25BB902220DF10E0043F6F421FFF730
:101BA00050F8BDF80E2023889A4201D0FFF78CFE32
:101BB000A3796FF38203A3716488124DCCB92B888B
:101BC000B3B1AB7903F00203DBB293B14320FFF76B
:101BD00081FC21460122234608200094F0F790FD65
:101BE00001230E20214622460094F0F789FD2B8820
:101BF0006B8005B0BDE8F083C8160020461E0020AB
